:020000040800F2
:1000000000500020F5160008A517000891290008E7
:10001000A5170008A5170008A51700080000000094
:10002000000000000000000000000000A51700080C
:10003000A517000800000000A517000809460008E1
:10004000A5170008A5170008A5170008A5170008A0
:10005000A5170008A5170008A5170008A517000890
:10006000A5170008A5170008A5170008A517000880
:10007000A5170008A51700081D450008A5170008CA
:10008000A5170008A5170008A5170008A517000860
:10009000A5170008A5170008A5170008A517000850
:1000A000A5170008A5170008A5170008A517000840
:1000B00079110008A5170008A51700089D3E000843
:1000C00085400008A13E000881400008A5170008EF
:1000D000A5170008514500088D450008A517000820
:1000E000A5170008A5170008A517000800000000C4
:1000F0000000000000000000000000000000000000
:0C01000000000000000000005FF808F1A3
:1001100010B5054C237833B9044810B10448AFF347
:1001200000800121217010BDD405002000000000D6
:100130002002010808B5064B1BB106480649AFF37B
:1001400000800648016811B1054A02B1904708BD18
:100150000000000020020108D8050020D40500207E
:100160000000000081F0004102E000BF83F0004386
:1001700030B54FEA41044FEA430594EA050F08BF42
:1001800090EA020F1FBF54EA000C55EA020C7FEA06
:10019000645C7FEA655C00F0E2804FEA5454D4EB83
:1001A0005555B8BF6D420CDD2C4480EA020281EA4D
:1001B000030382EA000083EA010180EA020281EA85
:1001C0000303362D88BF30BD11F0004F4FEA0131D7
:1001D0004FF4801C4CEA113102D0404261EB4101E6
:1001E00013F0004F4FEA03334CEA133302D052426C
:1001F00063EB430394EA050F00F0A780A4F1010428
:10020000D5F1200E0DDB02FA0EFC22FA05F2801861
:1002100041F1000103FA0EF2801843FA05F3594147
:100220000EE0A5F120050EF1200E012A03FA0EFCC6
:1002300028BF4CF0020C43FA05F3C01851EBE371F0
:1002400001F0004507D54FF0000EDCF1000C7EEB0D
:1002500000006EEB0101B1F5801F1BD3B1F5001F4B
:100260000CD349085FEA30004FEA3C0C04F101046A
:100270004FEA445212F5800F80F09A80BCF1004F93
:1002800008BF5FEA500C50F1000041EB045141EA15
:10029000050130BD5FEA4C0C404141EB010111F416
:1002A000801FA4F10104E9D191F0000F04BF0146C1
:1002B0000020B1FA81F308BF2033A3F10B03B3F19F
:1002C00020020CDA0C3208DD02F1140CC2F10C022F
:1002D00001FA0CF021FA02F10CE002F11402D8BF8D
:1002E000C2F1200C01FA02F120FA0CFCDCBF41EA59
:1002F0000C019040E41AA2BF01EB0451294330BD28
:100300006FEA04041F3C1CDA0C340EDC04F1140404
:10031000C4F1200220FA04F001FA02F340EA0300DB
:1003200021FA04F345EA030130BDC4F10C04C4F121
:10033000200220FA02F001FA04F340EA0300294601
:1003400030BD21FA04F0294630BD94F0000F83F44B
:10035000801306BF81F480110134013D4EE77FEA2E
:10036000645C18BF7FEA655C29D094EA050F08BF7A
:1003700090EA020F05D054EA000C04BF194610465B
:1003800030BD91EA030F1EBF0021002030BD5FEA9F
:10039000545C05D14000494128BF41F0004130BDC7
:1003A00014F580043CBF01F5801130BD01F000451B
:1003B00045F0FE4141F470014FF0000030BD7FEA8E
:1003C000645C1ABF194610467FEA655C1CBF0B4689
:1003D000024650EA013406BF52EA033591EA030FA0
:1003E00041F4002130BD00BF90F0000F04BF002198
:1003F000704730B54FF4806404F132044FF00005CB
:100400004FF0000150E700BF90F0000F04BF002143
:10041000704730B54FF4806404F1320410F00045A9
:1004200048BF40424FF000013EE700BF42004FEAA4
:10043000E2014FEA31014FEA02701FBF12F07F4321
:1004400093F07F4F81F06051704792F0000F14BF1E
:1004500093F07F4F704730B54FF4607401F0004562
:1004600021F0004120E700BF50EA010208BF7047B9
:1004700030B54FF000050AE050EA010208BF7047AE
:1004800030B511F0004502D5404261EB41014FF417
:10049000806404F132045FEA915C3FF4DCAE4FF01B
:1004A00003025FEADC0C18BF03325FEADC0C18BF02
:1004B000033202EBDC02C2F1200300FA03FC20FA53
:1004C00002F001FA03FE40EA0E0021FA02F11444A0
:1004D000C1E600BF70B54FF0FF0C4CF4E06C1CEAB5
:1004E00011541DBF1CEA135594EA0C0F95EA0C0F2A
:1004F00000F0DEF82C4481EA030621EA4C5123EA9D
:100500004C5350EA013518BF52EA033541F48011CB
:1005100043F4801338D0A0FB02CE4FF00005E1FB7E
:1005200002E506F00042E0FB03E54FF00006E1FBC8
:1005300003569CF0000F18BF4EF0010EA4F1FF040B
:10054000B6F5007F64F5407404D25FEA4E0E6D414B
:1005500046EB060642EAC62141EA55514FEAC5205C
:1005600040EA5E504FEACE2EB4F1FD0C88BFBCF5D8
:10057000E06F1ED8BEF1004F08BF5FEA500E50F189
:10058000000041EB045170BD06F0004646EA01014F
:1005900040EA020081EA0301B4EB5C04C2BFD4EB81
:1005A0000C0541EA045170BD41F480114FF0000E7A
:1005B000013C00F3AB8014F1360FDEBF002001F0E8
:1005C000004170BDC4F10004203C35DA0C341BDC62
:1005D00004F11404C4F1200500FA05F320FA04F034
:1005E00001FA05F240EA020001F0004221F0004168
:1005F00010EBD37021FA04F642EB06015EEA430EDB
:1006000008BF20EAD37070BDC4F10C04C4F120050A
:1006100000FA04F320FA05F001FA04F240EA0200BD
:1006200001F0004110EBD37041F100015EEA430E8E
:1006300008BF20EAD37070BDC4F1200500FA05F2AE
:100640004EEA020E20FA04F301FA05F243EA02032D
:1006500021FA04F001F0004121FA04F220EA02003C
:1006600000EBD3705EEA430E08BF20EAD37070BD82
:1006700094F0000F0FD101F00046400041EB010162
:1006800011F4801F08BF013CF7D041EA060195F044
:10069000000F18BF704703F00046520043EB0303FE
:1006A00013F4801F08BF013DF7D043EA06037047EB
:1006B00094EA0C0F0CEA135518BF95EA0C0F0CD0F6
:1006C00050EA410618BF52EA4306D1D181EA03013C
:1006D00001F000414FF0000070BD50EA410606BF36
:1006E0001046194652EA430619D094EA0C0F02D17B
:1006F00050EA013613D195EA0C0F05D152EA0336C0
:100700001CBF104619460AD181EA030101F00041DD
:1007100041F0FE4141F470014FF0000070BD41F026
:10072000FE4141F4780170BD70B54FF0FF0C4CF400
:10073000E06C1CEA11541DBF1CEA135594EA0C0F1F
:1007400095EA0C0F00F0A7F8A4EB050481EA030E6C
:1007500052EA03354FEA013100F088804FEA033353
:100760004FF0805545EA131343EA12634FEA022221
:1007700045EA111545EA10654FEA00260EF00041E2
:100780009D4208BF964244F1FD0404F5407402D234
:100790005B084FEA3202B61A65EB03055B084FEAC5
:1007A00032024FF480104FF4002CB6EB020E75EBC2
:1007B000030E22BFB61A754640EA0C005B084FEAEA
:1007C0003202B6EB020E75EB030E22BFB61A754667
:1007D00040EA5C005B084FEA3202B6EB020E75EBB2
:1007E000030E22BFB61A754640EA9C005B084FEA2A
:1007F0003202B6EB020E75EB030E22BFB61A754637
:1008000040EADC0055EA060E18D04FEA051545EA25
:1008100016754FEA06164FEAC30343EA52734FEACE
:10082000C2025FEA1C1CC0D111F4801F0BD141EA47
:1008300000014FF000004FF0004CB6E711F4801FAC
:1008400004BF01430020B4F1FD0C88BFBCF5E06F8C
:100850003FF6AFAEB5EB030C04BFB6EB020C5FEA9C
:10086000500C50F1000041EB045170BD0EF0004EF1
:100870004EEA113114EB5C04C2BFD4EB0C0541EA23
:10088000045170BD41F480114FF0000E013C90E620
:1008900045EA060E8DE60CEA135594EA0C0F08BFE4
:1008A00095EA0C0F3FF43BAF94EA0C0F0AD150EAE3
:1008B00001347FF434AF95EA0C0F7FF425AF104676
:1008C00019462CE795EA0C0F06D152EA03353FF49E
:1008D000FDAE1046194622E750EA410618BF52EA1B
:1008E00043067FF4C5AE50EA41047FF40DAF52EAEF
:1008F00043057FF4EBAE12E74FEA4102B2F1E04369
:1009000024BFB3F5001CDCF1FE5C0DD901F0004CF6
:100910004FEAC0024CEA5070B2F1004F40EB830046
:1009200008BF20F00100704711F0804F21D113F172
:100930003872BCBF01F00040704741F480114FEAAB
:100940005252C2F11802C2F1200C10FA0CF320FA34
:1009500002F018BF40F001004FEAC1234FEAD32351
:1009600003FA0CFC40EA0C0023FA02F34FEA4303BB
:10097000CCE77FEA625307D150EA01331EBF4FF044
:10098000FE4040F44000704701F0004040F0FE405F
:1009900040F40000704700BF80F0004002E000BF5C
:1009A00081F0004142001FBF5FEA410392EA030F5A
:1009B0007FEA226C7FEA236C6AD04FEA1262D2EBA4
:1009C0001363C1BFD218414048404140B8BF5B42A9
:1009D000192B88BF704710F0004F40F4000020F042
:1009E0007F4018BF404211F0004F41F4000121F058
:1009F0007F4118BF494292EA030F3FD0A2F10102A2
:100A000041FA03FC10EB0C00C3F1200301FA03F1DF
:100A100000F0004302D5494260EB4000B0F5000F02
:100A200013D3B0F1807F06D340084FEA310102F1C1
:100A30000102FE2A51D2B1F1004F40EBC25008BF73
:100A400020F0010040EA03007047490040EB00003D
:100A500010F4000FA2F10102EDD1B0FA80FCACF16C
:100A6000080CB2EB0C0200FA0CF0AABF00EBC2506B
:100A700052421843BCBFD0401843704792F0000F59
:100A800081F4000106BF80F400000132013BB5E7AC
:100A90004FEA41037FEA226C18BF7FEA236C21D022
:100AA00092EA030F04D092F0000F08BF0846704787
:100AB00090EA010F1CBF0020704712F07F4F04D155
:100AC000400028BF40F00040704712F100723CBF68
:100AD00000F50000704700F0004343F0FE4040F492
:100AE000000070477FEA226216BF08467FEA236350
:100AF0000146420206BF5FEA412390EA010F40F43B
:100B0000800070474FF0000304E000BF10F0004386
:100B100048BF40425FEA000C08BF704743F096436D
:100B200001464FF000001CE050EA010208BF704788
:100B30004FF000030AE000BF50EA010208BF70470F
:100B400011F0004302D5404261EB41015FEA010C24
:100B500002BF84460146002043F0B64308BFA3F11C
:100B60008053A3F50003BCFA8CF2083AA3EBC253FE
:100B700010DB01FA02FC634400FA02FCC2F120021D
:100B8000BCF1004F20FA02F243EB020008BF20F054
:100B90000100704702F1200201FA02FCC2F12002BA
:100BA00050EA4C0021FA02F243EB020008BF20EAAF
:100BB000DC7070474FF0FF0C1CEAD0521EBF1CEADD
:100BC000D15392EA0C0F93EA0C0F6FD01A4480EACB
:100BD000010C400218BF5FEA41211ED04FF00063B4
:100BE00043EA501043EA5111A0FB01310CF00040E0
:100BF000B1F5000F3EBF490041EAD3715B0040EA06
:100C0000010062F17F02FD2A1DD8B3F1004F40EBD5
:100C1000C25008BF20F00100704790F0000F0CF0A8
:100C2000004C08BF49024CEA502040EA51207F3A6C
:100C3000C2BFD2F1FF0340EAC250704740F4000047
:100C40004FF00003013A5DDC12F1190FDCBF00F038
:100C500000407047C2F10002410021FA02F1C2F1E6
:100C6000200200FA02FC5FEA310040F1000053EA82
:100C70004C0308BF20EADC70704792F0000F00F0D0
:100C8000004C02BF400010F4000F013AF9D040EAD6
:100C90000C0093F0000F01F0004C02BF490011F46A
:100CA000000F013BF9D041EA0C018FE70CEAD15368
:100CB00092EA0C0F18BF93EA0C0F0AD030F0004CE8
:100CC00018BF31F0004CD8D180EA010000F000409C
:100CD000704790F0000F17BF90F0004F084691F05A
:100CE000000F91F0004F14D092EA0C0F01D1420294
:100CF0000FD193EA0C0F03D14B0218BF084608D15D
:100D000080EA010000F0004040F0FE4040F40000A6
:100D1000704740F0FE4040F4400070474FF0FF0C39
:100D20001CEAD0521EBF1CEAD15392EA0C0F93EA80
:100D30000C0F69D0A2EB030280EA010C49024FEAD2
:100D4000402037D04FF0805343EA111143EA10138B
:100D50000CF000408B4238BF5B0042F17D024FF443
:100D6000000C8B4224BF5B1A40EA0C00B3EB510F1E
:100D700024BFA3EB510340EA5C00B3EB910F24BF07
:100D8000A3EB910340EA9C00B3EBD10F24BFA3EB8C
:100D9000D10340EADC001B0118BF5FEA1C1CE0D154
:100DA000FD2A3FF650AF8B4240EBC25008BF20F007
:100DB000010070470CF0004C4CEA50207F32C2BF5B
:100DC000D2F1FF0340EAC250704740F400004FF0F8
:100DD0000003013A37E792F0000F00F0004C02BF29
:100DE000400010F4000F013AF9D040EA0C0093F0F3
:100DF000000F01F0004C02BF490011F4000F013B4D
:100E0000F9D041EA0C0195E70CEAD15392EA0C0FB4
:100E100008D142027FF47DAF93EA0C0F7FF470AFEC
:100E2000084676E793EA0C0F04D14B023FF44CAF2F
:100E300008466EE730F0004C18BF31F0004CCAD1C4
:100E400030F000427FF45CAF31F000437FF43CAF00
:100E50005FE700BF4FF0FF3C06E000BF4FF0010C22
:100E600002E000BF4FF0010C4DF804CD4FEA400204
:100E70004FEA41037FEA226C18BF7FEA236C11D04E
:100E800001B052EA530C18BF90EA010F58BFB2EB01
:100E9000030088BFC81738BF6FEAE17018BF40F081
:100EA000010070477FEA226C02D15FEA402C05D135
:100EB0007FEA236CE4D15FEA412CE1D05DF8040BBA
:100EC000704700BF844608466146FFE70FB5FFF74D
:100ED000C9FF002848BF10F1000F0FBD4DF808ED05
:100EE000FFF7F4FF0CBF012000205DF808FB00BFF6
:100EF0004DF808EDFFF7EAFF34BF012000205DF850
:100F000008FB00BF4DF808EDFFF7E0FF94BF01209C
:100F100000205DF808FB00BF4DF808EDFFF7D2FF99
:100F200094BF012000205DF808FB00BF4DF808EDDC
:100F3000FFF7C8FF34BF012000205DF808FB00BFA9
:100F40004FEA4002B2F1FE4F0FD34FF09E03B3EBD6
:100F500012620DD94FEA002343F0004310F0004F16
:100F600023FA02F018BF404270474FF0000070476C
:100F700012F1610F01D1420205D110F0004008BF0B
:100F80006FF0004070474FF00000704742000ED2F3
:100F9000B2F1FE4F0BD34FF09E03B3EB126209D4B4
:100FA0004FEA002343F0004323FA02F070474FF06A
:100FB0000000704712F1610F01D1420202D14FF0DF
:100FC000FF3070474FF00000704700BF034BDA88D6
:100FD0000280198941805B8983807047F005002079
:100FE000054B1A88510001805A88510041809B8826
:100FF0005A008280704700BFF00500207047000053
:10100000074B084A0360426007480B60074A4FF0ED
:101010007E534860CB604FF4BC711180704700BFB5
:10102000FD0F0008CD0F0008E10F00084800002068
:1010300038B504460D46002D14DD052003F017FBDE
:10104000204608F07DFE204608F07FFE0028FAD1F9
:10105000204608F07EFE204608F080FE0028FAD1E7
:10106000013DE8E738BD000070B53E4D90B0284620
:1010700009F076FC3C4880213C4B06900A912020E8
:101080004FF40051002409264FF4807205930D900F
:101090004FF480630E91284605A90C930B92079498
:1010A00009940F94089609F0D3FC2846012109F011
:1010B000FCFC009403942E4C01254FF46022204642
:1010C000694602928DF804508DF805508DF8106035
:1010D00008F000FE20460A212A46032308F04BFEB2
:1010E00020460B210222032308F045FE032220465E
:1010F0000C21134608F03FFE20460D210422032355
:1011000008F039FE20460E210522032308F033FEA5
:1011100020460F210323062208F02DFE204605213C
:101120000722032308F027FE204606210822032376
:1011300008F021FE324603232046072108F01BFE5B
:101140002046294608F0F3FD2046294608F0E6FD32
:1011500020460221FFF76CFF2046294608F002FED8
:1011600010B070BD08000240F00500204C24014082
:1011700000240140002070475E4B2DE9F0411C78AF
:10118000002C58D002214FF0804009F060F901286E
:1011900008D1594C594B21884FF08040198009F0F3
:1011A00049F9208002214FF0804009F05BF9524854
:1011B000524902880B889A4201D9D21A01E0D843D9
:1011C000121893B2B3F57A6F4D4A03D90023137006
:1011D000BDE8F081A3F2EF2188B240F2DA518842F3
:1011E0001ED81278072A1BD84648032A00EBC201F2
:1011F000CB80454909D840F2D930834205D9012333
:1012000003FA02F2087802430A7009780F2907D11D
:101210003E483D4B016800221A700A68536898479F
:1012200037483A4B01784A1C0270186801680A680E
:101230009047BDE8F0812546354850F8347000EB02
:10124000C402B7F1804F9688B2F806804DD1384677
:10125000414609F0FCF8012847D13846414609F0DB
:1012600001F90C2E1CD8DFE806F0071B1B1B0C1B1A
:101270001B1B111B1B1B16004FF0804009F0DAF8F6
:101280000DE04FF0804009F0D8F808E04FF08040C2
:1012900009F0D6F803E04FF0804009F0D4F8054695
:1012A000184AE00012F83410131839B9012019490E
:1012B00002F8340002225D804A8011E05F889D8040
:1012C000BD4201D9EF1B01E0F9436F18DF80002711
:1012D00017540E4A10680368196888470D494F80F3
:1012E0004FF080400E8009F009F80134082CA3D19A
:1012F000BDE8F0810D060020100600200E0600203B
:1013000054060020140600200C060020C8100020FF
:1013100000000020020600202DE9F04300248FB0D9
:101320000A2706460D463A46214604A801940BF0CA
:101330007FFC214610220AA80BF07AFC844B854AD8
:101340001D6085487578337840F2DC510570D18096
:10135000D181D182D183D184D185D186D187002B0F
:1013600000F0948007A821463A460BF061FC0394F4
:101370002820002D42D0012502A98DF80B004FF046
:1013800002087648ADF808508DF80A8008F0EAFBAC
:101390001C2203A88DF80C208DF80D408DF80E50FE
:1013A0008DF80F5008F03EFD07A808F027FF4FF614
:1013B000FF704723ADF8200007A94FF08040ADF83B
:1013C0001C30ADF81E4008F0D1FD65494FF080405B
:1013D0004C80CC800C810C808D80624C08F08EFF9C
:1013E0004FF0804041462A4608F02BFF4FF08040E6
:1013F000294608F00CFFA946277047E002221F2467
:101400008DF80B0002A955488DF80A20ADF8084068
:1014100008F0A8FB01241C2103A88DF80C108DF8FE
:101420000D508DF80E408DF80F4008F0FBFC07A81A
:1014300008F0E4FE4FF6FF704723ADF8200007A93F
:101440004FF08040ADF81C30ADF81E5008F08EFD16
:10145000434A55809480D5801581434C4049631997
:10146000988808802859083508F048FF202DF4D1C5
:101470004FF080401E21012208F0E3FE01214FF0D1
:10148000804008F0C4FE374904250D7018254FF43C
:101490007071ADF804108DF8075001A9022533488A
:1014A0008DF8065008F05EFB04A808F0A7FE33890B
:1014B0002F48472290FBF3F4611EADF814102D481D
:1014C00004A9ADF8102008F051FD4FF47A704FF4E4
:1014D0008071702200230124ADF82E00ADF8341085
:1014E00024480AA9ADF82820ADF82C30ADF82A40E0
:1014F000ADF8305008F084FD0AA91E4808F0C4FD7C
:101500000AA91C4808F004FE0AA91A4808F042FE7D
:101510000821184808F09EFE0821164808F0A2FE8F
:101520000821144808F0A8FE0821124808F0ACFE73
:101530002146104808F06BFE21460E4808F073FE65
:101540000C48082108F086FE0FB0BDE8F08300BF0C
:10155000C8100020140600200D06002000080140DD
:10156000020600201206002000000020000C0140AE
:1015700040420F0000080040044B1A78824203D911
:10158000034B53F820000180704700BF1206002073
:1015900040DC000870470000024B03EBC000C0882D
:1015A000704700BF14060020F8B5134B05469B8911
:1015B0000E461446ECB116B116F8017B00E0FF2789
:1015C0000D48022108F080FB0028F9D00A4839466E
:1015D00008F075FB0848012108F076FB0028F9D0D7
:1015E000054808F06EFBC0B20DB105F8010B013CD7
:1015F000E0E70120F8BD00BF003800402DE9F047CA
:10160000012188B04FF4804009F0A6F8374C012141
:101610004FF4804009F0B8F803214FF4204018231C
:10162000ADF800008DF80310204669468DF80230B1
:101630004FF0040802F02EFD2D4E4FF4804220465C
:101640006946ADF800204FF480554FF0100A8DF830
:10165000028002F01FFD69462046ADF800508DF86B
:1016600002A002F017FD304608F0CCFA07214FF433
:10167000007000230222ADF81600ADF81C104FF0E8
:101680000109304603A94FF48277ADF80C30ADF86C
:101690001030ADF81A30ADF81220ADF80E70ADF87C
:1016A00014901F46ADF818A008F0DEFA30464946FF
:1016B00008F0F9FA9F238DF804308DF805708DF845
:1016C00006708DF807700DEB08014246656102A8AF
:1016D000FFF76AFF25619DF80900B0F1EF014A426A
:1016E00052EB010008B0BDE8F08700BF000C0140DC
:1016F000003800401D481E49026800608A4200F020
:101700001F80002100F004B81A4B5B58435004318D
:1017100019481A4B42189A42FFF4F6AF184A00F0E3
:1017200003B8002342F8043B164B9A42FFF4F9AF8A
:1017300008F0FAF80BF084F901F00CF8FFF7FEBF9F
:10174000114E124830601248016821F0706101604A
:10175000410201600F4C182020600F490F480860BB
:101760000F48D0F800D0406800470000F04F00203C
:10177000EFBEADDE4402010800000020D4050020C9
:10178000D405002020170020181002400900000096
:1017900004000140140C0140000C01404434434457
:1017A00000F0FF1FFFF7FEBF014B186802F0ADBC51
:1017B000101700200149002000F076BEA91700088C
:1017C00010B5FFF7A3F90A49FFF7F4F90949FFF744
:1017D000A5FA094B044618680078FFF797F9014607
:1017E0002046FFF7E7F9FFF7D1FB80B210BD00BF3D
:1017F0003333534000F07F456806002038B50D4C68
:1018000000202578FFF7B6FC0B4A05F0070322F805
:1018100013000135002325701846D15A02334018B1
:10182000102B80B2F9D1C008FFF7CAFF034A10702D
:1018300038BD00BF5506002056060020CC10002001
:10184000074B084A19781088884207D3064B1A6854
:10185000907888428CBF002001207047002070479C
:10186000CC100020CE10002068060020124B70B56E
:101870001860202400250020FFF77CFC2D180A208A
:1018800002F0F5FE013CF6D1C5F34F10FFF798FFCB
:10189000094902230A6851784D006619B04203D302
:1018A0000133062B0C44F8D104489278037053435B
:1018B00003490B8070BD00BF680600204000002077
:1018C000CE1000202DE9F04F0446008885B048B9BD
:1018D000B4F9023043B9B4F90420D2F1010138BFA0
:1018E000002102E0002100E0014611F0010377D160
:1018F0003D4D00B22B7000F007FD0646B4F9020022
:1019000000F002FD0546B4F9040000F0FDFC0446B9
:10191000304609F0EDF80746304609F05DF980469B
:10192000284609F0E5F80646284609F055F9054627
:10193000204609F0DDF88246204609F04DF9394687
:1019400081465046FFF736F9394683464846FFF749
:1019500031F9514601904046FFF72CF94946029073
:101960004046FFF727F9314603905046FFF722F92A
:101970001E4C4946206006F10040FFF71BF929463E
:101980006060A5600298FFF715F901460198FFF71E
:1019900009F82946E0600398FFF70CF9014658461C
:1019A000FEF7FEFF3146206108F10040FFF702F923
:1019B000294660615846FFF7FDF801460398FEF797
:1019C000EFFF2946A0610198FFF7F4F8014602985D
:1019D000FEF7E8FF3946E0613046FFF7EBF820629A
:1019E00005B0BDE8F08F00BF410000206C0600206C
:1019F0002DE9F8434D4B0C460168013A1960808887
:101A00009880072A30D8DFE802F004080F14191E66
:101A10002226188820805A8803E0598821801A8855
:101A2000524262809A881EE01988484220805A8873
:101A3000F6E75988484220801A88F2E71988484218
:101A4000208058880CE05A882280188808E019887D
:101A500021805A8803E05988484220801A885042E1
:101A600060809B885A42A280314B1A78002A5AD152
:101A7000B4F90000FFF74AF88046B4F90200FFF716
:101A800045F80746B4F90400FFF740F8294D06462B
:101A900029684046FFF78EF8E96881463846FFF727
:101AA00089F801464846FEF77DFFA9698146304620
:101AB000FFF780F801464846FEF774FF09F04CF83E
:101AC000696820804046FFF775F8296981463846E5
:101AD000FFF770F801464846FEF764FFE969814662
:101AE0003046FFF767F801464846FEF75BFF09F00E
:101AF00033F8A96860804046FFF75CF86969804662
:101B00003846FFF757F801464046FEF74BFF296A73
:101B100007463046FFF74EF801463846FEF742FFCB
:101B200009F01AF8A080BDE8F88300BF90060020F5
:101B3000410000206C060020F8B5154C06462378BD
:101B4000274663B902F082FD124D2A683232904274
:101B500005D30123237002F079FD2860F8BD3878A1
:101B6000A0B102F073FD0B4C2168731898420DD39D
:101B700007480022027002F069FD074920600B78D7
:101B80000BB15A1E0A70054901200870F8BD00BF4C
:101B900096060020A0060020990600209A06002044
:101BA00037B58DF805101F498DF807300B788DF883
:101BB000040002A88DF80620C21812F8044C0D4645
:101BC000443CE0B20A2828D81749022B31F81040CB
:101BD00003D814B12046FFF7AFFF2B78022B0BD9A7
:101BE000124D2D6802F032FD021B954204D20D49C0
:101BF0000F4B0020087018700E4802780146012A29
:101C000000D074B9074B1878022801D8421C1A700A
:101C100000230B7008490B7003E03224022BD9D942
:101C2000DBE73EBD9706002060DC0008A006002030
:101C3000990600209A06002096060020014B1860A5
:101C4000704700BFC810002070B53D4B04465A7B5A
:101C50003C4802B1012202704FF4007000F052F9CA
:101C6000002828D0384E394B316858780D6800303C
:101C700018BF0120AA68904748B13368344D1868EE
:101C8000012102692970904708B1022129702E4D67
:101C90002B681868C268904728B12C494B7813B953
:101CA0002B4A0220107029680B689869804710B190
:101CB000274900220A70202005F070F860B1204802
:101CC000244B827A0AB9C17A21B12048C27A0AB972
:101CD000012100E0002119701D4B1878022802D163
:101CE0004C204E211DE0012807D14D2153204C22CC
:101CF0000B46BDE87040FFF753BF164A1178012923
:101D000003D1532001464E2206E00E4B18780128DD
:101D100004D15320014602464D23EAE724B1532063
:101D20004D210A464423E4E70B4A117821B13220C1
:101D3000BDE87040FFF700BF084B1C7070BD00BFCE
:101D40009C1600209B060020C81000208B16002047
:101D5000980600209C060020990600209606002088
:101D60000E4B1A78402A16D15888B0F5667F12D1EA
:101D70001979BE290FD193F895230020EF2A0CD1B1
:101D800013F8011B064A48409342F9D1D0F10100F3
:101D900038BF0020704700207047704700F80108E6
:101DA00098FB010810B50C4C204605F0ABF80B4B26
:101DB0002046B3F8D010B3F8D2201F3C05F0BCF891
:101DC00014F8B40B01F0ACF903F0BEFF2046BDE8F7
:101DD000104000F06DBC00BFF3100020A0110020E7
:101DE00010B5FFF7BDFF10B90A2002F0E3FC0E4C5E
:101DF0000E4920464FF466720AF06CFE94F8943354
:101E0000022B02D9002084F8940394F89413CC2276
:101E100002FB0143064803F598710AF05BFEBDE83A
:101E20001040FFF7BFBF00BFA011002000F801085D
:101E3000D410002008B5FFF7D3FF0F201421012292
:101E4000BDE8084007F050BD08B5054BCC2202FBA9
:101E50000030044900F598700AF03CFE08BD00BF50
:101E6000A0110020D4100020224A38B5402313705E
:101E70004FF466700023BE21EF245080117182F868
:101E8000954382F896331D461A4A985C0133B3F5A0
:101E9000667F85EA0005F7D182F8965308F06EFB5D
:101EA00004250024691E11F0FF0516D0342008F027
:101EB00079FB114808F0CCFB0F4C04280BD10F4ADA
:101EC0002046A15808F09AFB0D4B04349C42F4D1F3
:101ED0000428044601D00446E4E708F05BFB042C28
:101EE00002D1FFF73DFF20B90A20BDE8384002F0DB
:101EF00061BC38BDA011002000F80108A019FE1730
:101F000098FB0108034B996808420CBF0020012090
:101F1000704700BFA0110020024B9A6810439860E0
:101F2000704700BFA01100202DE9F347B74AB84D14
:101F300010685168B74C6B4603C34FF466720021BA
:101F400028460AF075FECC22002120460AF070FED9
:101F500040200321287002206971FFF7DDFFFA227B
:101F6000A5F8F2202A236E22A5F8EE304FF4FA707D
:101F700085F804212B2340F24C42A5F8F60085F8A1
:101F80000531212002F54873202185F80601A5F8C6
:101F9000163140F27E404FF47A7300274FF001096A
:101FA0004FF4167685F8F410A5F8142140F2DC51B0
:101FB00000F52F72A5F8D00003F5CB70A5F8F060FE
:101FC000A5F81211A5F8D22085F89473A5F8F87039
:101FD000A5F8FA70A5F8FC7085F8E27085F8E37052
:101FE00085F8E470A5F8E670A5F8E870A5F8EA7041
:101FF00085F8ED7085F8EC9085F8077185F82C71FF
:1020000085F82D7185F82E7185F8107185F8187195
:1020100085F8197185F81A91A5F8D430A5F8D6007D
:102020006C30A5F8D8004FF4C870A5F8DE004FF466
:102030001650322340F2B452C5F8240140F6AC5099
:10204000A5F8DA20A5F8DC301A46A5F8E030A8811A
:102050004FF4E1331E20C5F82031E0725223207383
:10206000552085F82A31E07017230B204FF02808FF
:102070006375A37560712D2314204FF0080E6373F0
:102080002271A07185F81C7185F81D7185F8287181
:1020900085F82971AF7385F81B71277084F801806A
:1020A00084F80280E775A7732776E773677684F86C
:1020B00010E060745020E076E1845A200421A37679
:1020C00020722375E077412384F82E10524853493B
:1020D0004FF00E0A84F82030514B84F807A04FF0DF
:1020E000640C4FF00A0A4FF0780E84F821206063E8
:1020F0001522E1634B4805F5847184F83120A36310
:1021000084F812A084F81CC084F8098084F80AE0DE
:1021100084F81E9084F8237084F8247084F8257065
:1021200084F822706785A785278584F82F8084F836
:10213000308084F8409004F03DFF4FF44872C8208E
:102140004FF4966340F2D9313E4684F86C7084F8BF
:102150006D7084F86E8084F86F9084F87270A4F8C3
:10216000702084F8B4A084F8B500A4F8B630A4F8C0
:10217000B8104FF47F724FF4FA601DF80710A4F8FE
:102180007420A0F5FA73FF220137A4F87600A4F8B2
:10219000783084F87A1084F87B200834082FE8D14E
:1021A0001C4C0120C823142184F8BA0084F8BB0019
:1021B00084F8BC00A4F8BE3084F8C01084F8C200D3
:1021C0001E2264204FF49673282184F8C120A4F8BD
:1021D000C400A4F8C630A4F8C81000240C4A002398
:1021E000A0181034C02C0361F8D100240E49CC2271
:1021F00060180849CC340AF06DFCB4F5197FF5D1AC
:1022000002B0BDE8F047FFF72FBE00BF28DC000892
:10221000A0110020D41000209A99193F3D0A773F61
:10222000F6287C3F76DC0008D012002008B5FFF7C6
:1022300097FD18B9BDE80840FFF776BE08BD00005D
:10224000024B9A6822EA000098607047A0110020B3
:10225000014B9868704700BFA0110020884203DB43
:102260008242B4BF1146014608467047002303610D
:1022700070472DE9F041066904460136012E0D46EE
:10228000066105D10023616021608360BDE8F081B3
:10229000D0F8008008464146FEF782FB07463046EC
:1022A000FEF734FC01463846FEF738FD014640464D
:1022B000FEF778FB0646606031462846FEF770FB65
:1022C00001463846FEF776FCA168FEF76BFB2660F8
:1022D000E060A060BDE8F08110B504460069012807
:1022E00007DD0138FEF712FC0146E068FEF716FD37
:1022F00010BD002010BD08B5FFF7EEFFBDE8084097
:1023000008F0F8BC0000000008B5FEF77DF804A353
:10231000D3E90023FEF7DEF8FEF7EEFA08BD00BFB2
:10232000399D52A246DF913F2DE9F041069C0646B9
:102330000F46002B0CBF4FF020084FF0300820460E
:1023400010F8013B0BB9154603E0002AFBDD013A0A
:10235000F6E7002D04DD30464146B847013DF8E779
:1023600014F8011B11B13046B847F9E7BDE8F08118
:102370002DE9F04389B006460F4603921C46039AA6
:10238000134613F8011B0393002900F08A802529C6
:1023900001D0304683E0002004905578911C302D08
:1023A000039105D19578033203924FF0010800E0C4
:1023B0008046A5F13003D8B2092806D8284603A9DB
:1023C0000A2204AB00F00CF905466C2D05D10399E7
:1023D000012211F8015B039100E00022642D2FD04F
:1023E00010D8582D3AD006D8002D5AD0252DC6D158
:1023F0003046294653E0632DC1D130462178251D52
:10240000B8474AE0752D0DD0782D27D0732DB6D161
:10241000251D2468304600943946049A0023FFF7AE
:1024200083FF3AE0251D20680A2122B1002205AB76
:1024300000F060F802E005AB00F08CF82C4623E0D9
:1024400005AD04F104092068294612B100F077F8BF
:1024500001E000F0A4F84C46009517E004F10409EF
:102460002068102142B1B5F15804634253EB0402D5
:1024700005AB00F03FF806E0B5F158035A425A4167
:1024800005AB00F067F84C4605A800903046394689
:10249000049A4346FFF748FF71E72C466FE7B847B9
:1024A0006DE709B0BDE8F083024B1960024908608E
:1024B000704700BFA4060020A80600200FB407B58F
:1024C000094904AB0868094953F8042B09680193CA
:1024D000FFF74EFF064B186801F036FE0028F9D0D2
:1024E000BDE80E4004B07047A8060020A4060020F6
:1024F00010170020F0B50124B0FBF4F58D4201D394
:102500004C43F9E70026C4B1B0FBF4F504FB150019
:10251000B4FBF1F41EB9002D01DC002CF4D1092D1F
:10252000EFB204DD002A0CBF5725372500E0302527
:10253000ED1903F8015B0136E5E71C70F0BD0028DA
:102540000B4603DA2D22404203F8012B0A21002218
:10255000FFF7D0BFF0B50124B0FBF4F58D4201D3F5
:102560004C43F9E70026C4B1B0FBF4F504FB1500B9
:10257000B4FBF1F41EB9002D01DC002CF4D1092DBF
:10258000EFB204DD002A0CBF5725372500E03025C7
:10259000ED1903F8015B0136E5E71C70F0BD00287A
:1025A0000B4603DA2D22404203F8012B0A210022B8
:1025B000FFF7D0BFA0F13003DAB2092A01D81846DC
:1025C0007047A0F16101052901D857387047A0F183
:1025D0004103052B01D8373870474FF0FF30704763
:1025E0002DE9F8430D6804460F46904699460026AB
:1025F0002046FFF7DFFF002806DB404504DC08FB30
:10260000060615F8014BF3E73D602046C9F8006067
:10261000BDE8F883014B00229A807047AC06002089
:10262000034BB3F90400D0F1010038BF002070471C
:10263000AC0600200649074B0A68B3F9040013787A
:1026400005214B439842D4BF00200120704700BFB2
:10265000B4060020AC06002010B50446FFF7EAFFE0
:10266000002814BF2046002000F0010010BD00002B
:10267000074B084A1968B2F904004B780A78D11858
:10268000052251438842D4BF00200120704700BF7B
:10269000B4060020AC060020044B9A8811B214291D
:1026A00001DD143A00E000229A807047AC06002059
:1026B000024B00221860024882807047B406002056
:1026C000AC060020034B0449186004480022016056
:1026D000C2807047B806002080DC0008AC060020ED
:1026E00008B502F099F8024B00221A7008BD00BF2D
:1026F0008B16002010B5FFF79DFFE0B1104B5C7802
:10270000201C18BF0120FFF7A7FF70B10D480E4B2A
:1027100001680E484A8901681A805A809A804A885E
:10272000DA800B4BD888411CD980FFF7A1FF00B994
:102730000CB9FFF7D5FF064B9A88501C988010BD46
:102740008B160020B8060020CC160020B40600200E
:10275000AC06002070B57F4C86B0A07B003018BF5F
:10276000012001F08FFFFFF725F8FFF75FFDFFF76E
:1027700037FB94F8073133B1012B01D0092B02D17B
:102780008DF8003004E000218DF8001084F8071166
:102790006846FEF769FC7048FFF794F8022004F0E1
:1027A00007FB02F0F9FC6B4A55790E2D01D0082D7C
:1027B00001D1012600E000264FF480708DF80A60F8
:1027C000FFF7A0FB18B90820FFF79CFB00E00120F1
:1027D00000F0010440208DF80640FFF793FB8DF8D0
:1027E00007000120FFF78EFB8DF805000820FFF79A
:1027F00089FB80F001008DF8040003F01DF9574BB0
:10280000544D93F8BC108DF80800B5F8DE604FF415
:102810007A70B5F8E040C1F38002ADF810004FF4D3
:1028200080408DF80920ADF80C60ADF80E40FFF740
:1028300069FB18B1B5F8DA30ADF81030BDF80C10FE
:10284000B1F5FA7F02D90022ADF81020434CB5F85B
:10285000126195F80751B4F8B800012DADF8126077
:10286000ADF8140004D0092D01D1072500E00025A2
:102870003B488DF80B50FFF725FF3A4E3060FFF7CD
:10288000DDF901A83168FEF747FD3548316804F0ED
:10289000BFFA4FF48070FFF735FB40B10820FFF717
:1028A00031FB20B92B4B93F81D0103F09FFA2E4CFE
:1028B0004FF400414FF4805261610A26C4F8102899
:1028C000294C013EE06880F40045E560274D192061
:1028D000EB6883F48051E96001F0C9FE192001F032
:1028E000C6FE16F0FF06EBD14FF400404FF48052C5
:1028F0002A61206101F03CF902F012F80220FFF792
:1029000001FB10B11A48FEF7B1FF1A4805F01EF995
:102910004FF40060FFF7F6FA10B1174804F006FE16
:1029200001F07AFE0B4D154C6B792060052B03D11D
:10293000134E4FF4C87131801248134D134B4FF4AE
:102940007A72C824012102802C80597300F0F6FBB2
:10295000FCE700BFA011002086120020D410002048
:10296000A8120020C81000200008014000100140FB
:10297000A4120020C0120020101700200007002021
:102980006007002080070020680B00208B160020C5
:1029900008B5034BB3F9D40002F01AFDFEE700BFFF
:1029A000A01100202DE9F04F794B0024B3F902A0CB
:1029B000B3F9000087B0BAF1000FB8BFCAF1000A3E
:1029C0000028B8BF40428245B8BF82462546A0468F
:1029D00027460594A14626466E49CA7812B90B7956
:1029E000002B40D0022E3ED06B4B6C486849B0F8AB
:1029F000F620685EE95EDFF8B4B101EB40005142B9
:102A0000FFF72CFC664A05EB0B0335F902C0B3F95E
:102A10002A10CCEB00009BF8082000EB010902FB18
:102A200009F09BF81C30642190FBF1F005226FF057
:102A3000040159435A43CDF81090FFF70FFC594B4E
:102A4000DDF810C0E258584981460CEB020042F212
:102A500010720493FFF702FC04999BF81230605047
:102A60005843001305904B49CA781AB10B790BB93A
:102A7000022E30D1464F4D48EF5F5021794306EB8F
:102A8000000B9BF801204A4BDFF83C8191FBF2F0F0
:102A9000E95E54F80820401A801846494FF47A52EB
:102AA0000493FFF7DBFB049B48F80400E95E002970
:102AB000B8BF4942B1F5207F02DD002048F804008C
:102AC00058F804207D239BF80B1092FBF3FE01FBCA
:102AD0000EFC4FEAAC182F480279A2B1022E12D098
:102AE0000AFB07F1CAF5FA7303FB09104FF4FA71F8
:102AF00090FBF1F20AFB08F0DDF814B003FB0B03C6
:102B000093FBF1F308E0C3780BB1022E02D14346E8
:102B10003A4601E0059B4A462549DFF8B0C0695AAC
:102B200016F80CB008B20BFB00FB6FF04F0C9BFBD0
:102B3000FCFB9344204ACDF804B035F902C0A952F9
:102B4000CCEB00001D4ADFF888C0029054F80C104E
:102B5000A0584018029903904018A15844F80C104E
:102B60000299A150164A0434B15C202201FB00F006
:102B700090FBF2F15B1A134A9B44013625F802B030
:102B80000235032E7FF428AF07B0BDE8F08F00BFF9
:102B90006C1500208B16002028070020A0110020B3
:102BA000780B002048070020F0D8FFFFD410002049
:102BB0009A0B002080C1FFFFDC0600203C070020AC
:102BC000BA15002074150020BC060020BD15002099
:102BD0001C0700202DE9F74F002425462646A24673
:102BE000474BDA780AB91879C8B1022E19D0454B8B
:102BF00045484649B0F8F6206F5EE85E514200EB6A
:102C00004700FFF72BFB424A424F35F902A0EB1970
:102C1000CAEB0001B3F92A0001EB000A0BE0022E17
:102C200009D13C49394B91F82470B3F904201B3782
:102C300057437B1116E03249364ACF7877B933488B
:102C400092F823702B5E1B375F4309793B1149B122
:102C5000927C02FB0AF703EB272303E0137A03FBC2
:102C60000AF003112C48DFF8C8B0295EBBF8000059
:102C70005F1A284B784306EB030898F80120DFF829
:102C8000B4907A4398F80B104FEAE21C54F80920EC
:102C9000C31201FB0320214944F809004FF400123C
:102CA000CDF804C0FFF7DAFA1D4B4FF6FF72E1587A
:102CB000E750791ABBF8007044F809003B09B2FBF1
:102CC000F3F74F43174A184B54F80290E158BF11DD
:102CD000A750494498F81520C9194A43DDF804C0A3
:102CE00012490CEB603044F80390013600EB2223CC
:102CF0006B5204340235032E7FF472AFBDE8FE8FB1
:102D00008B16002028070020A01100206C15002041
:102D1000780B0020D41000209A0B00200000E0FF68
:102D2000D0060020F0060020300700207415002097
:102D30002C070020BC0600200B4B0C481A8852B907
:102D4000817841B142786AB9012141700848094B44
:102D500002881A807047437823B90220FF2101229C
:102D600006F0C2BD704700BF800700208B16002010
:102D7000F6150020B81500202DE9F04FB54BB64AE6
:102D8000B3F90600D18C85B088420FDBB0F5FA6F3D
:102D900092F8254007DA451A6C43A1F5FA6694FBD0
:102DA000F6F4643403E0C4F1640400E06424AB4A44
:102DB000A94BB2F8127192F9EC2093F82310009706
:102DC000574293F86C50019193F86D60B9B293F843
:102DD00024300291002103930A469E4FDDF80080C3
:102DE00031F907C040F2E637C8EB0C0303F2F31EDB
:102DF000BE4503D8002BB8BF5B4201E04FF4FA7325
:102E0000022ADFF864822CD025B1AB42CCBFC5EBDF
:102E1000030300236427DFF880A293FBF7FE6FF023
:102E2000630B3AF81E900BFB0E3B0EF1010E3AF9C4
:102E30001EA00FFA89FECEEB0A0E0EFB0BFE9EFBC8
:102E4000F7FEF14428F80190DDF8048003FB08FE4A
:102E5000834B9EFBF3F3DB199BB2634393FBF7F7C2
:102E600012E026B1B342CCBFC6EB03030023029F9E
:102E70005F43A8F80470039F002BB8BF5B427B43FD
:102E8000774F93FBF7F76437734B02EB030E9EF813
:102E90000190642307FB09F898FBF3F9DFF8FC8144
:102EA00002F808909EF80B909EF815E007FB09F8D1
:102EB00007FB0EF798FBF3F9DFF8E48197FBF3F3D8
:102EC00002F80890DDF80080664FC445D35503DA58
:102ED000654BCF5A7F42CF5201320231032A7FF431
:102EE0007CAF5E4C4FF4FA62B4F81411FFF7B6F9F8
:102EF000B4F814614FF47A75801B4543C6F5FA6344
:102F0000B5FBF3F56421594895FBF1F36FF06306C7
:102F100030F8132006FB0355013330F9130013B2C8
:102F2000C01A4543524B504C95FBF1F1587A8A1820
:102F3000E280002838D04F4F4F4D3E882988721AC2
:102F400010B2FFF7E1F9074607F0D2FD0646384612
:102F500007F042FE0546B4F90200FDF7D7FD07462B
:102F6000B4F90000FDF7D2FD31468046FDF722FEA0
:102F7000294681463846FDF71DFE01464846FDF7C5
:102F80000FFDFDF7DDFF314620803846FDF712FECC
:102F9000294606464046FDF70DFE01463046FDF740
:102FA00001FDFDF7CDFF60800220FEF7ABFF90B181
:102FB000324806220378591CCBB20370B3FBF2F0FF
:102FC00002FB103111F0FF0F05D1FEF717FCFEF7E1
:102FD00037FC2B4B18702A4A1078003018BF01209C
:102FE000FEF732FE27490B881BB9274A108828B9FB
:102FF0000AE0022003F0D2FE0028F6D0234BDA6864
:1030000082F48051D9600EE0194B997819B11F4AAA
:103010004FF4805010615B781BB11C484FF4805115
:10302000416104F05FFA1A481A4A01681368C81A25
:10303000002839DB0E4B587BA0BB9870134B01F571
:10304000F421D86880F48050D86001F59073136043
:103050002AE000BFCC160020D4100020A0110020D0
:103060000CFEFFFFBA1500206C150020B4160020DE
:103070008B160020F6150020B815002051070020FF
:10308000FD0600206007002080070020001001409E
:1030900054070020E4060020F0160020BD15002093
:1030A000B01500200121997004F05CFD154A1078DC
:1030B00030B94FF40060FEF725FF08B104F04EFA76
:1030C000202003F06BFEA0B10F49104B0A6818686E
:1030D000111A00290DDB0E480178042909D902F5DF
:1030E000123202F5F87018600A4BD96881F4004278
:1030F000DA60094883680BB10848984705B0BDE815
:10310000F08F00BF30100020540700201807002067
:10311000B615002000080140E41500204C150020E1
:103120000128034B14BF034A034A1A60704700BFCB
:1031300044000020A5290008D52B000838B5082038
:10314000FEF7E0FE90B1A04B93F8100103280CD8D5
:10315000DFE800F00202050804F072F906E003F06F
:10316000BBFF03E004F076F800E000209749984A9E
:103170000B681168591A002902DA002800F0B3829E
:1031800003F59C44934820349349146003F062FE95
:103190004FF48040FEF7B6FE20B1904D2B780BB96E
:1031A00001F03AFB884A92F81B11B1B18C4CC81C53
:1031B00034F910504FF47A720021A5F57A70FFF7B8
:1031C0004DF8FDF7A3FC8749FDF7A8FD8649FDF7FB
:1031D000F1FCFDF7DBFE854B18804FF40070FEF725
:1031E00091FE20B1824A116808684469A047764D73
:1031F0000022B5F81401B5F81641134678499B082A
:10320000555E8542C4BF63F07F03DBB2A542B8BF01
:1032100043F040030232082AF0D17648764A047817
:1032200005469C4204D11078F92803D8411C00E0DF
:10323000002111704FF480402B70FEF763FE68B1DF
:10324000614D674BB5F81211B5F8DC20B3F90640B3
:10325000881A844202DD8B189C420CDB4FF48040BC
:10326000FEF750FEF8B95E4C5749B4F90650B1F874
:103270001421954217DA614D6148624CB5F842104D
:1032800000230360436083602360636059B1534A45
:103290005D4B1078002800F08D821C78002C00F027
:1032A0008982FFF749FD54490A78142A40F0DD80ED
:1032B00055484478ECB1514AB2F842502DB94D49C5
:1032C00008785F2801D101F0A7FA3F4C94F8183133
:1032D000002B00F0CA80494AB2F84250002D40F05D
:1032E000C480444908787D2840F0BF8001F094FAFA
:1032F000BBE0404D2B78572B18D1444C4FF47A72D9
:103300004FF480702280FEF7FDFD08B102F0CAFC88
:10331000042003F043FD10B13D490A250D8008202B
:1033200003F03CFDD8B93B4B188018E00420FEF7B1
:10333000E9FDA0B129785A2911D1374802781AB18C
:103340000470364B012009E0354C364B257885F06A
:103350000101217009B1022000E003201870254806
:1033600002785D2A00F02D825B2A00F02C825E2A12
:1033700000F02B822148B0F8422032B91D4C25784C
:103380006F2D02D1FFF7D8FC15E00F49194B91F8CA
:10339000180118B112B91A787E2AF3D01C78972C2C
:1033A00004D1214B4FF4C870188004E0A72C02D13F
:1033B000154901258D730F4A1478BB2C36D10F4C5B
:1033C000A18D8D1C37E000BFA01100205407002004
:1033D00014070020A8120020B21600209C1600201E
:1033E000CC16002000007A4400C07F44B4150020B1
:1033F000C81000205007002004070020D41000202F
:10340000BC060020480700208B1600208007002003
:10341000680B0020F6150020C8060020CC0600200E
:10342000E80600209906002060070020B72C04D190
:103430008C4CA28D951EA5850BE0BE2C03D1894D29
:103440006B8D981C04E0BD2C0FD1864D698D881EB4
:1034500068858548002490F89403FEF7F5FCFEF794
:1034600003FDFEF7E7FC814B1C700420FEF74AFDCC
:1034700000282CD07E4C23788BB17E4A557875B1CC
:103480007D49794BB1F90600B3F81421904206DD6D
:103490007A4D2B781BB97A49322008802370774CFB
:1034A000627C52B1774D2A782AB9774B187810B9D7
:1034B000734C32212180012408E0734D2B7833B105
:1034C0006C48417819B92970704D01242C70002383
:1034D0006F4C1A4634F8020F40F2135501B2A9425C
:1034E000CCBF0025012505FA03F5A0F21550B0F573
:1034F000C77F8CBF002001202A435D1C00FA05F025
:10350000024340F2A4608142D4BF00210121981CF3
:1035100001FA00F103330A430C2B92B2DAD10023F3
:103520005048564900EB4300B0F8420002420CBF3D
:103530000020012058540133152BF1D14A7822B1D3
:10354000022003F02BFC68B915E04FF40070FEF781
:10355000D9FC80B14F4908680368DA6890470028B1
:10356000EED108E0434AD37843B94B4901200B60C0
:103570004B60D07002E03F480021C1703F4A3D4B94
:10358000917839B118790021D97020B9424A0121C6
:10359000106050601971394B3649187808B901220A
:1035A0000A70C8783D4B10B932490A791AB14FF404
:1035B0000041596102E04FF400401861202003F0FF
:1035C000EDFB00287FD02B4BD87A1A46002875D007
:1035D00033490878042871D92848817A79B1DA7991
:1035E000002A70D12F480121D9711A722E4B011D6A
:1035F0001A7002F06BFC2D4A0220107063E0C27A50
:10360000D97122B317482A49B0F8C820B1F900008F
:103610000028B8BF4042904219DAB1F902100029DF
:10362000B8BF4942914212DA187A00284BD10124DE
:103630001C721D4B1F4918701F480A684B68011DFA
:103640000260436002F042FC184804703BE01648F8
:10365000084B017800221A72A9BB0122027002F005
:1036600045FB30E0D4100020A0110020040700200A
:10367000E80600208B160020CC1600209C160020A7
:103680000607002010070020C8060020CC060020F6
:10369000D2160020C8100020480700200008014072
:1036A000B61500207C1500204200002008070020ED
:1036B0006C150020981500205C1500200023D371A4
:1036C00013724A4A13704A494A4B087B00B10120E1
:1036D000494A98725179082901D00E2927D1454BC2
:1036E0000020587223E045480368042B1FD8DFE808
:1036F00003F00305080B17000122026001684B1C50
:1037000003600268511C01603C4803685A1C026057
:103710004FF48070FEF7F6FB10B102F071FC06E08A
:103720003648002101604FF40050FEF7EBFB00F03B
:1037300073FF334A304910608A89324B1AB11968D5
:10374000411A002951DB8018186001F0F9FAFFF7DF
:1037500013FB00F061FF2C4B294A196810601860B8
:10376000421A2A482A4990F872300A8053B12149F6
:10377000CA780AB9087928B1264B2749DA88088817
:103780008118D980202003F009FB40B1194BD8796A
:1037900008B91A7A1AB1197B09B103F079FA1F4BEB
:1037A0001868804701F026FE01F0A2FDBDE8384010
:1037B00001F0FABD5D78002D3FF475AD01F02CF8F5
:1037C00071E5012402E0022400E003240A4BE5B283
:1037D000691E83F89413FEF747FBFEF701FB0220F6
:1037E00028212A4606F080F8C4E538BD08070020E5
:1037F0009C1600208B160020A01100200C07002032
:1038000054070020EC06002000070020D410002000
:103810002C0700206C150020980B0020440000208D
:10382000F8B5664B1D88002D40D000231946B5F52C
:10383000C87F634A01D100205050624E50589F5FAC
:103840005F4CC0195050604A002098539E180233B4
:103850000431062BA6F8F800E9D1012D22D1216808
:103860004FF4C87301F1C80191FBF3F1A2F8F8100D
:103870006168C83191FBF3F1A2F8FA10A168C83170
:1038800091FBF3F3514909885B1A5149A2F8FC30C6
:103890004885888592F89403FEF7D6FAFEF7E4FA95
:1038A000FEF7C8FA45480288531E03800420FEF73D
:1038B00029FB00286FD047490A88322A11D1424D8E
:1038C000454CB5F8F860B5F8FA00B5F8FC30404959
:1038D00026806080A3804D8D404C8E8D2580668033
:1038E00001E0002A32D000231946322A3C4801D197
:1038F00000244450334D44585E5FA6194650324868
:1039000000245C531D1802330431062B2646A5F80B
:10391000F840EAD1012A16D1324B33491A70334BA1
:103920000C70022119702C4B1988A0F8F8105988D6
:103930009B88A0F8FA102949A0F8FC30244B08888D
:10394000498858859985234B013A1A80284801787F
:1039500009B30022027022481B4B0468322194FBF9
:10396000F1F4A3F8F8404468806894FBF1F490FB0C
:10397000F1F11648A3F8FA400088091A1448A3F890
:10398000FC104285828593F89403FEF75DFAFEF7FA
:103990006BFAFEF74FFA0B4B0B4A1888B2F8F81087
:1039A000401A1880B2F8FA105888B2F8FC20401A71
:1039B00099885880881A9880F8BD00BF6007002059
:1039C0007407002014160020A011002048000020D9
:1039D000D4100020060700205A07002062070020AC
:1039E00068070020C8060020100700209906002064
:1039F000CC06002010B5074B074C59682046884775
:103A0000064A204621461278FDF7F2FFBDE8104035
:103A1000FFF706BFD015002014160020580700201D
:103A20002DE9F84F414B188800286ED00024254618
:103A300026463E490A88B2F57A7F08D13C4B3D497B
:103A400000271420EF5000FB0610FEF70FFCDFF8F4
:103A5000F0A0374F3AF90400EA59DFF8D89013186C
:103A6000EB51FDF753F84FF0140B0BFB069B01468F
:103A70004FF000085846FEF7FCFB24F80A80DFF8F8
:103A8000ACA02D48BAF8001024F80080012933D1E9
:103A90005846FEF730FC294A834692F8F400E0B11C
:103AA000FDF734F801465846FDF740FAA8B14FF447
:103AB0007A714846AAF80010FEF7D8FB09F1140005
:103AC000FEF7D4FB09F12800FEF7D0FBC7F8088009
:103AD000C7F80480C7F800800EE0154B4FF47A72E7
:103AE000E858154B00F5FA7191FBF2F0E0520F2106
:103AF0000A20012205F0F8FE013604350234032EB7
:103B000097D10A480288531E03800D4B0A4A188831
:103B10001188401A1880518858889288401A9988CC
:103B20005880881A9880BDE8F88F00BF8007002071
:103B300084070020900700206A0B0020A0110020BD
:103B4000FC15002010B5074B074C596820468847E4
:103B5000064A204621461278FDF74AFFBDE810408C
:103B6000FFF75EBFE4150020FC150020CC07002005
:103B700001480249FDF744BAD0150020E4150020A1
:103B80002DE9F84F9C4C2068838A9BB213F0010208
:103B900039D0018821F400631A04110C018001213D
:103BA00006F0BCFE954A964B117800201870D9B1EA
:103BB000944803781BB9944A1178FF2914D1012342
:103BC000037092480278022A06D18B490B68188844
:103BD00082B242F4006119808D4B874819780068E1
:103BE000012206F0B5FE2FE18948834B01780022BF
:103BF000186806F0ADFE844A1178FF2900F0248190
:103C0000FF207F4BDEE003F00201C9B200293DD066
:103C1000BFF35F8F7D4D2E78012E354616D1774943
:103C20000B789BB177490B7883B1114606F076FE8D
:103C3000BFF35F8F20683146038B06F063FE754A41
:103C4000206816704FF480613246FBE0038BBFF3AF
:103C50005F8F6E490A78022A09D1684B1A7832B10F
:103C6000684B1A781AB1002106F058FEE5E0097891
:103C7000032907D1614B1A7822B162490B78002BD6
:103C800040F0DD804FF480610122DBE003F00406A8
:103C9000F6B2002E71D0594BDFF878811A780126E0
:103CA00088F80060574B002A4DD01A78002A4AD075
:103CB000564D2F78524D022F574F29D906F02EFE20
:103CC000206895F80090D7F800A006F03EFE4FFA65
:103CD00089FB0AF80B0009EB0600314628702068C2
:103CE00006F010FE206888F800603F6895F80080B4
:103CF00006F02BFE4FFA88F907F80900B044206857
:103D00004FF48061324685F8008006F013FE2BE008
:103D1000314606F0F7FD20682E78D7F8008006F0CF
:103D200014FE4FFA86F9731C08F80900D9B220680E
:103D30004FFA81F83F68297006F007FE033607F84E
:103D400008002E7010E01B78012113B9334A137854
:103D50002BB106F0D7FD2A480278511C03E006F08B
:103D6000C5FD284801210170234A11680B8803F41E
:103D7000807082B2002AF9D166E003F040010F465C
:103D80001F4D09B3244B2F78D3F8008006F0DDFDDA
:103D90004FFA87F908F80900781CC1B229701B4D49
:103DA0004FB22A780337BA4205D120684FF48061B8
:103DB000324606F0BFFD124B28781A7851B288427D
:103DC00042D1501C18703FE01B063DD52B785EB2E7
:103DD000721C27D0124901330A682B70915D06F0DE
:103DE000B2FD0A4895F90020017891422CD1206853
:103DF0004FF480613A4625E0E4070020E207002006
:103E0000E0070020E1070020D1070020D2070020B2
:103E1000E9070020D0070020D4070020D8070020A1
:103E2000DC070020154A2970117806F08CFD144833
:103E3000017811B9134B1A7832B9134800684FF45E
:103E40008061002206F076FD0E4A104B117893F93E
:103E500000004A1C90420ED10D4B0E4918780022EA
:103E60000A7028B1084908684FF4407106F062FDF5
:103E7000094B00221A70BDE8F88F00BFD10700205F
:103E8000E2070020D2070020E4070020E00700201E
:103E9000D0070020E1070020E8070020FFF770BEF0
:103EA000FFF76EBEF0B5484C89B04FF440651C2357
:103EB00007460226204602A9ADF808508DF80A30C0
:103EC0008DF80B6000F0E6F84048142107608DF88B
:103ED0000E10204603A9ADF80C508DF80F6000F0CD
:103EE000D9F825610825384CA268520503D40A2068
:103EF00000F0B2FBF7E74FF480660A20666100F03D
:103F0000ABFB6F1E0A20266100F0A6FB17F0FF0531
:103F1000E9D14FF4006767610A2000F09DFB6661FC
:103F20000A2000F099FB26610A2000F095FB022090
:103F300027611C218DF80F002046244C4FF440636C
:103F40008DF80E1003A9ADF80C3000F0A3F820682E
:103F500006F02EFC04A806F0AFFC20682A464FF4B9
:103F6000407106F0E7FC1A484FF480434BF6FF72AD
:103F7000049001212068ADF81C30ADF81620ADF892
:103F8000145006F0A7FC04A9206806F02BFC4FF49F
:103F9000A06005F03DFF2221012201A88DF8041048
:103FA0008DF805508DF806508DF8072005F03AFF82
:103FB000212301A82E468DF804308DF8055005F018
:103FC00031FF09B0F0BD00BF000C0140E407002044
:103FD000801A0600274B37B51868818A8AB2019289
:103FE000019B13F4706F02D0234A01211170019BD1
:103FF00013F4E06F31D04FF480610022038B06F0A0
:1040000099FC0198810528D41A4D2868018801F48B
:10401000007293B20BBB048804F480718CB29CB123
:10402000028802F4807399B20029F9D1012106F0C7
:1040300069FC10480068028802F4007399B20029F4
:10404000F9D1FFF72FFF08E0012106F05BFC28689B
:104050004FF44071224606F06DFC06480268938AD0
:1040600023F470610804030C0449938200220A704F
:104070003EBD00BFE4070020D9070020E80700206C
:10408000FFF7A8BFFFF7A6BF014B188880B27047A3
:10409000CE0700202DE9F0410F88002347FA03F2F4
:1040A000D2072DD58A7803F00705DC08AD0012F0A1
:1040B000100F18BF91F803C002F00F0618BF46EAB0
:1040C0000C064FF00F0C0CFA05FC06FA05F550F83B
:1040D0002480282A28EA0C0C45EA0C0540F82450D4
:1040E00006D1012202FA03F2C46824EA020206E0C1
:1040F000482A05D1012202FA03F2C4682243C260B1
:104100000133102BCAD1BDE8F08108B503681A68E5
:10411000904708BD38B505460C4614F8011B19B187
:104120002846FFF7F2FFF8E738BD08B5036859687D
:10413000884708BD08B503689968884708BD08B571
:104140000368DA68904708BD08B5036819698847AD
:1041500008BD08B503685A69904708BD7047036BEE
:1041600013B15A68006C01E0026AC069101A18BFE6
:1041700001207047436B13B190F844007047826A86
:10418000406A111A4B4253EB01007047836A816900
:10419000426BC918D160416A994203D9CB1A536066
:1041A000816204E00169CB1A53600022826200211F
:1041B00080F84410406B012106F077BC30B504460E
:1041C000007985B000230D460091C107ADF8043099
:1041D000ADF80630ADF80830ADF80C30ADF80A3067
:1041E00002D50422ADF80A20820705D5BDF80A10D1
:1041F00041F00803ADF80A30A06C694606F036F9C4
:10420000A56005B030BD026B034610B5406942B1F0
:104210001A6CD9688C1A013A18BF1146005D1964EE
:1042200010BD196ADA68405C0131B1FBF2F402FB9F
:104230001411196210BD10B5426A8469A154416A13
:1042400002690131B1FBF2F402FB1411426B4162CD
:1042500032B11368DB070BD4BDE81040FFF796BFFF
:10426000806C40F227710122BDE8104006F062B96F
:1042700010BD0000214B13B5986021480C465861D1
:104280002048214A2149186314381A6099614FF473
:104290008072586301214FF48040DA601A6106F0A1
:1042A0004FFA4FF4007102231822ADF80010A10755
:1042B0008DF803308DF8022003D515486946FFF7C5
:1042C000E9FE48234FF48060E207ADF800008DF866
:1042D000023003D50E486946FFF7DCFE01220E21AD
:1042E00001A88DF804108DF805208DF806208DF8B2
:1042F000072005F097FD01481CBD00BFAC0A002057
:10430000AA090020580002409CDC00082A0800206E
:10431000000801401F4B13B51F4A98600C468020CF
:104320004021D86019611D481D491A601D4A9861D5
:1043300099644FF4003001215A6106F00DFA02230E
:10434000042218208DF80330A307ADF800208DF863
:10435000020003D514486946FFF79CFE0821482354
:10436000E007ADF800108DF8023003D50E4869461D
:10437000FFF790FE012026228DF8050002218DF81E
:10438000070001A88DF804208DF8061005F04AFDFD
:1043900000481CBDF80A00209CDC0008EA07002049
:1043A000004400402A090020000801402DE9F041A6
:1043B0001E46584B90B0984205468846174604D191
:1043C00010463146FFF756FF07E053480024854268
:1043D00004D110463146FFF79DFF0446002106F048
:1043E00004022671A7600197A5642162E161A162C0
:1043F0006162C4F82C80ADF8081002F0FF0732B1FA
:104400004FF40053ADF80A304FF4806701E0ADF887
:104410000A700020ADF80C7016F00107ADF810001E
:1044200002D1ADF80E7002E00421ADF80E1006F0D6
:10443000020606F0FF082EB1BDF80E2042F0080378
:10444000ADF80E30284601A906F010F801212846E3
:1044500006F064F805A806F01BFB0023281D4FF4A6
:104460008051802205900E910F9309930B930A922D
:104470000C9317B3206BD0B16269E16807932023D6
:104480000D930692089106F06BFA206B05A906F0D1
:10449000DFFA206B012106F008FB284640210122AB
:1044A00006F062F8206B06F015FB206405E0284654
:1044B00040F22551012206F03DF8B8F1000F24D05A
:1044C000606BE0B1266910210896002607910D96D1
:1044D00006F046FA606B05A906F0BAFA0122606B95
:1044E000022106F0EDFA606B314606F0F1FA606BDE
:1044F000802146600122284606F036F805E028466D
:1045000040F22771012206F015F8204610B0BDE8F0
:10451000F08100BF003801400044004010B50B4C52
:104520004FF4005006F0DAFA0021606B06F0BDFA95
:10453000626AA36A9A4204D02046BDE81040FFF7A1
:1045400025BE012084F8440010BD00BFAC0A002045
:104550000D4B986C028802F080018AB29AB19A6A77
:10456000596A8A420AD09969895C01328180196945
:10457000B2FBF1F001FB10229A62704740F2277102
:10458000002205F0D7BF7047AC0A00201C4B10B5C5
:104590009A6C1488A4B204F0200188B290B1D96A50
:1045A00019B1938898B288470CE09288D969586904
:1045B000D2B24254D869DA68411CB1FBF2F002FB76
:1045C0001011D96104F08004A4B2C4B10C4B9A6AF2
:1045D000586A82420BD09869996C805C013288805D
:1045E0001969B2FBF1F001FB10229A6210BD986CC0
:1045F00040F227710022BDE8104005F09BBF10BDBE
:10460000F80A002070470000024B1A68501C18601E
:10461000704700BF440B002010B5094A09491368D0
:104620008C6810688342F8D1074A106811684FF40B
:104630007A725043001BB0FBF1F102FB031010BD76
:10464000440B002010E000E0480B0020014B1868EC
:10465000704700BF440B002038B50446FFF7DCFF6D
:104660000546FFF7D9FF401BA042FAD338BD10B56D
:1046700004462CB14FF47A70FFF7EEFF013CF8E7E7
:1046800010BD000070B53E4B8AB0054601AC0FCBA3
:1046900084E80F00284605F0A7F90121394806F003
:1046A0005BF8012144F61D2006F04AF8012001467E
:1046B000354D06F039F806F073F800214FF6FF701B
:1046C000ADF800008DF80210284669462F4EFFF71E
:1046D000E1FC2F486946FFF7DDFC69463046FFF7ED
:1046E000D9FC2C4B5A6842F000705860FFF78AFFE3
:1046F0004FF480514FF40043274A31612B61106819
:104700002649884206D19DF80A30142B02D1102286
:104710008DF80A20211D0198FFF7BCFC1E481F4B95
:104720000168994206D19DF81220142A02D1102066
:104730008DF8120004A90398FFF7ACFC05A805F05A
:10474000A5FF059B1649174AB3FBF1F01649106007
:1047500008684FF47A73B0FBF3F2511E1348144A01
:10476000F023416082F82330002107238160036039
:10477000FCF744FF6420FFF77AFF0AB070BD00BF6A
:1047800030DC000807004000000801400010014034
:10479000000C01400000014084010020001BB70014
:1047A00040420F00480B00208801002010E000E08C
:1047B00000ED00E010B540F2DB1460430D4B4FF408
:1047C00000424FF480515A61841EC3F81018094802
:1047D000C26882F40043C360D0F80C1881F48052A0
:1047E000C0F80C282046FFF742FF1920FFF73FFFD3
:1047F000EDE700BF0008014010B1034A034B1A6007
:1048000003480449C8607047EFBEADDEF04F00209A
:104810000400FA0500ED00E0024B5A780AB10020CE
:10482000587070478B1600202DE9F84F384E04461B
:104830003768384606F05CF90546384606F0CCF98C
:1048400076688046304606F053F98346304606F0D7
:10485000C3F9D4F80490064629464846FCF7AAF95D
:10486000A768824641463846FCF7A4F901465046FF
:10487000FCF796F8216882465846FCF79BF94146BA
:1048800004464846FCF796F93146FCF793F9014691
:104890002046FCF787F8314604463846FCF78AF98B
:1048A0002946FCF787F901462046FCF77BF80146CC
:1048B000504606F01DFA1749FCF77CF9FBF7B6FDE8
:1048C00011A3D3E90023FBF72FFF134B044618680D
:1048D0000D46FBF7ABFD02460B4620462946FBF78B
:1048E00047FC00220D4BFBF71FFFFCF705F806F015
:1048F00033F981B20A0444BF00F5B47189B208B239
:10490000BDE8F88FAFF30080182D4454FB21094017
:104910005C0B00200000E144A00B002000002440BC
:1049200010B5194C2088FCF7F1F81849FCF742F94A
:1049300006F012F9164B18802088FCF7E7F80146BC
:104940001448FCF7EBF91449FCF7E8F9134908603F
:104950001348B0F87000FCF7D9F801461148FCF78D
:10496000DDF9FBF763FD06A3D3E90023FBF7B2FDF6
:10497000FBF7C2FF0C4A106010BD00BFAFF3008010
:104980003B597E90A9E7814048000020C903683F59
:104990004C0B00200AE81C4100401C461016002069
:1049A000D4100020000061442C160020AFF30080DA
:1049B0002DE9F041044600680D460146FCF7FAF87F
:1049C000D4F80480064641464046FCF7F3F8014619
:1049D0003046FBF7E7FFA768064639463846FCF73E
:1049E000E9F801463046FBF7DDFF06F083F90021C8
:1049F0000646FCF773FA70B920683146FCF78EF969
:104A0000314628606068FCF789F931466860A06823
:104A1000FCF784F9A860BDE8F0812DE9F04F0C683F
:104A2000836889B0D0F800A0D0F8048006462046FC
:104A300003938B4606F05CF80746204606F0CCF858
:104A4000DBF804408146204606F052F80546204631
:104A500006F0C2F8DBF8082004461046019206F082
:104A600047F88346019806F0B7F839460290584651
:104A7000FCF7A0F8394604900298FCF79BF85946D9
:104A800005904846FCF796F8029906904846FCF7D0
:104A900091F8294607905846FCF78CF80146504695
:104AA000FCF788F8214683460698FCF783F8014610
:104AB0000598FBF777FF01464046FCF77BF8014677
:104AC0005846FBF76FFF214683460498FCF772F8BF
:104AD00001460798FBF764FF01460398FCF76AF864
:104AE00001465846FBF75EFF3060029905F1004031
:104AF000FCF760F801465046FCF75CF82146834617
:104B00000798FCF757F801460498FBF749FF014660
:104B10004046FCF74FF801465846FBF743FF214655
:104B200083460598FCF746F801460698FBF73AFFDE
:104B300001460398FCF73EF801465846FBF732FF62
:104B4000214670605046FCF735F82946044609F1C5
:104B50000040FCF72FF801464046FCF72BF80146D1
:104B60002046FBF71FFF394604462846FCF722F88B
:104B700001460398FCF71EF801462046FBF712FF9A
:104B8000B06009B0BDE8F08F1FB50B684A6889684E
:104B90000193039101A90292FFF73FFF05B000BD09
:104BA00080EAE073A3EBE0738B4206DB002801DDB3
:104BB000401A704702D0401870470020704700002C
:104BC0002DE9F041524B86B01A685B6802F1004251
:104BD00003F1004301934F4B0646B3F900000092E6
:104BE000FBF794FF00F10040FBF720FC46A3D3E95C
:104BF0000023FBF76FFCFBF77FFE474C0290B4F9F4
:104C00000000FBF783FF0390B4F90200FBF77EFF7F
:104C10000490B4F90400FBF779FF6946059003A8F6
:104C2000FFF7FBFE3D4B93F84030012B16D13C487B
:104C3000417869B93B4C4025226892FBF5F7D01BBF
:104C4000FBF764FF0599FBF7ADFEFCF779F92060EF
:104C5000344B4021186890FBF1F001E0324B18888A
:104C6000FBF754FF01460598FBF79AFE0590304686
:104C7000FBF748FF2D490746FBF794FE01463846EF
:104C8000FCF74CF82A4D07462C6805982146FBF79F
:104C900087FE01463846FBF78DFF01462046FBF7AD
:104CA00081FE244C28601D4D07460398D4F80080EF
:104CB00005F052FF95F83010FFF772FF08EB000285
:104CC00004982260D4F8048005F046FF95F830106F
:104CD000FFF766FF08EB000338466360D4F80880EE
:104CE00005F03AFF95F82F10FFF75AFF1249134BC2
:104CF0000A684044A0601868B6180E60411C19602C
:104D000006B0BDE8F08100BF399D52A246DF913F59
:104D10005C0B0020F615002024160020D410002083
:104D20008B160020700B0020480000203661823C6A
:104D3000940B002004160020740B0020900B002020
:104D40002DE9F04F87B0FEF7FDFE022002F026F8B5
:104D5000002800F0A781FEF74DFEFFF75DFCAA4C8E
:104D600005462768C71B3846FBF7CCFEA749C9682C
:104D7000FBF720FF8346A648256090F82E8000258B
:104D80002C462E46A34A105FFBF7C0FE5946FBF7A0
:104D900011FF03AB5851B8F1000F27D04046FBF785
:104DA000B5FE01464FF07E50FBF7B8FFDFF8A49246
:104DB000824651464FF07E50FBF7F2FD55F8091040
:104DC000FBF7F8FE94490346085F0193FBF79EFE4C
:104DD0005146FBF7EFFE01460198FBF7E3FD49F86A
:104DE0000500FCF7ADF88D4A105303E08A498B4A61
:104DF000605AA052894B0435E15E0234062C01FB57
:104E00000166BFD1864A6420138846435B438548C8
:104E100003A996FBF3F6FFF7B7FE082001F0BEFFEB
:104E200020B1814803A9FFF7AFFE07E07F4803A93F
:104E3000FFF7AAFE7D480146FFF7BAFD493EB1B231
:104E40003B2904D9082001F0A9FF48BB50E0784C69
:104E5000B4F8F000FBF756FE4FF07E518046FBF7AA
:104E6000A1FD01464FF07E50FBF758FF0024064697
:104E70006C4D404655F81410FBF79CFE8146674880
:104E8000005FFBF743FE01464846FBF78BFD3146CA
:104E9000FBF790FE45F814000234062CE8D1D1E768
:104EA000634A0024B2F8F200FBF72CFE4FF07E516B
:104EB0008046FBF777FD01464FF07E50FBF72EFF53
:104EC0000646594D404655F81410FBF773FE594BF2
:104ED0008146185FFBF71AFE01464846FBF762FD64
:104EE0003146FBF767FE45F814000234062CE8D182
:104EF00051494C4DB1F90000FBF708FEAC68014682
:104F000020460126FCF712F800B906464B48214618
:104F10004673686805F0ECFE494C2A6820606868B2
:104F200002F100460146FBF745FED5F8088005462C
:104F300041464046FBF73EFE01462846FBF732FD60
:104F400005F0D8FE0146304605F0D2FE60602068CC
:104F5000FBF76CFA2AA3D3E90023FBF7BBFAFBF7B4
:104F6000CBFC05F0F9FD374D28806068FBF75EFA51
:104F700023A3D3E90023FBF7ADFAFBF7BDFC05F053
:104F8000EBFD6880082001F009FF2F4C08B126488E
:104F900000E02648FFF748FC1D4D20803846FFF70B
:104FA0000FFE95F87230002B00F080801D490868D4
:104FB0008C684F680146FBF7FDFD394606463846CA
:104FC000FBF7F8FD01463046FBF7ECFC21460646B0
:104FD0002046FBF7EFFD01463046FBF7E3FC05F00A
:104FE00089FE01462046FBF799FE18490446FBF767
:104FF00089FF88B3164A0020108057E0AFF3008085
:105000003B597E90A9E78140640B0020E415002005
:10501000D4100020FC1500201416002024160020B7
:105020004800002030160020500B00204C000020CB
:10503000A0110020DC1500204C0B00208B16002056
:105040005C0B0020780B0020F61500208FC2753C09
:10505000980B0020800B0020204605F0F9FD264B20
:105060001968FBF7A7FD05F077FDB0F5617FA8BFD4
:105070004FF46170FBF7C8F91DA3D3E90023FBF7D8
:1050800053FBFBF739FC05F0A7FD044695F87200C9
:10509000FBF73CFD2146FBF78DFD05F05DFD174B51
:1050A000188003E0164B188058809880154B59796A
:1050B000154B012907D015481A8859889B8802800A
:1050C0004180838011E01249B3F90420B1F9000056
:1050D00002EB4000032290FBF2F080B20B4A088002
:1050E00019885B8890801180538007B0BDE8F08FED
:1050F000A2EB0FE5DD1696402C160020980B002041
:1051000014160020A0110020FC1500209A0B00208E
:105110008C0B0020AFF3008010B5054C00202188D7
:10512000FCF738FA61880120BDE81040FCF732BA7C
:10513000580000200A4A02EBC00393F87B10FF29B5
:1051400004D019B1074830F8110007E00728DABF8A
:1051500002EBC000B0F8780040F2DC5000B27047BB
:10516000D4100020CC16002010B500244FF480404D
:10517000FCF7C8FE064B10B1B3F8DA0001E0B3F853
:10518000D400044AA0520234182CEFD110BD00BF45
:10519000A011002054160020F8B53B4D3B4E6B7912
:1051A0003B4C06EBC300417820202160FCF7AAFEAF
:1051B000324608B1012626606B79162B1CD10024DB
:1051C000314E0021A6193069FBF788FE28B14FF453
:1051D0008040FCF797FE50BB23E02E4B06F11000F9
:1051E0001D190FC885E80F002B4910340A78531C8D
:1051F000C02C0B70E4D1EAE7274F12F8336002EBC2
:10520000C3003E704768002FE1D00024B442DEDACC
:10521000204D21016D187A180FCA013485E80F005E
:10522000F4E719481D4B4179082923D124E01A4E8F
:105230003678012EF5D91A4C00251034B542F0DA33
:1052400054F8100C4FF07C51FBF7B4FC4FF07C513C
:1052500044F8100C54F8140CFBF7ACFC4FF07C51E4
:1052600044F8140C54F80C0CFBF7A4FC013544F87A
:105270000C0CE2E70E2901D1012200E000221A7491
:10528000BDE8F840FFF770BFA011002024DE000841
:10529000AC0B0020B00B0020A80B00208B160020C8
:1052A000B80B0020F0B50023461C0E4A00219818C8
:1052B0001033C02B0161F8D10B4F07EBC6035F68B9
:1052C00007B9F0BD0024084A12F83600844208DA13
:1052D000064D21014D197B180FCB013485E80F00D5
:1052E000F1E7F0BDA011002024DE0008B01100207D
:1052F000284B10B5186800284AD027494A79531E10
:10530000142B3DD8DFE803F00B3C3C24403C3C1C14
:105310003C3C3C3C3C2C3C3C3C3C3C242C001F4852
:1053200090F8BB1031B11E4B00205989BDE81040E8
:10533000FCF730B91B4A50780028F4D10146F5E754
:10534000174C0020E188FCF725F901202189EDE7C1
:10535000134C00202189FCF71DF901206189E5E744
:105360000F4C0020E188FCF715F901202189FCF79A
:1053700011F902206189FCF70DF90320A189D5E715
:105380002020FCF7BFFD18B1BDE81040FFF7C4BEF8
:1053900010BD00BFAC0B0020A0110020D4100020D5
:1053A000580000208B16002010B50024064B1878FA
:1053B000A04208D90549204631F814100134FCF701
:1053C000DBF8E4B2F2E710BDA80B00203C16002089
:1053D000064B1A780023D9B2914204D2044921F82D
:1053E00013000133F7E7FFF7DFBF00BFA80B002072
:1053F0003C1600202DE9F84FB24B187803280FD93E
:10540000B149B24CB1F904206FF06305002AB8BF6E
:105410005242A91AB4F904006432FCF71FFFA080BD
:10542000A84A1678012E1DD8A94EAA4C75796A1E75
:10543000142A00F2F981DFE812F0C200F701F70147
:105440008400D500F701F7017101F701F701F701B9
:10545000F701F701F100F701F701F701F701F70193
:105460005E00C7019B48994B90F9BA90964FB3F9EB
:105470000440C9F10001B7F806A004FB01F95F88F8
:10548000B3F80080944C00251034B542CCD20FFA0A
:105490008AF0FBF73BFB54F8101CFBF78BFB8346B1
:1054A00038B2FBF733FB54F8081CFBF783FB0146CB
:1054B0005846FBF777FA83460FFA88F0FBF726FB8E
:1054C00054F80C1CFBF776FB01465846FBF76AFACA
:1054D00083464846FBF71AFB54F8041CFBF76AFBAB
:1054E00001465846FBF75EFAFBF72AFD7B4B23F893
:1054F00015000135C8E794F89A20744D12F0010F99
:105500006B880CBF01264FF0FF365E43744CB7B278
:1055100004202781FFF70EFE29886E4D381895F874
:10552000A230208113F0010F0CBF01224FF0FF3297
:105530004A43052096B26681FFF7FCFD3718678164
:1055400072E194F89A50614805F002084FFA88F623
:10555000002E0CBF01214FF0FF3115F0010F4588DF
:105560000CBF01224FF0FF326A438688042001FB02
:1055700006F497B2FFF7DEFD1FFA84F808EB00038C
:105580005448F91890F8A270554C07F0020253B233
:105590002181002B0CBF01214FF0FF314E4317F04A
:1055A000010F0CBF01204FF0FF3045430520FFF7EE
:1055B000C1FDB6B2ADB23718EA19628134E1434990
:1055C00094F8A2408E8814F0010F0CBF01234FF015
:1055D000FF3305205E43FFF7ADFDB5B2404F2818FD
:1055E000788121E10020FFF7A5FD3E4F94F97A3044
:1055F000B7F902603A4D7343322693FBF6F1401837
:1056000028800120FFF796FDB7F9002094F9824029
:10561000544394FBF6F3C7186F8005E1324C607871
:1056200020B9B6F8D4202E4BDA810AE02649B6F824
:10563000D220B1F90600B6F8D010FCF70FFE284DC5
:10564000E881274E254CF7892780214F97F81901CB
:1056500030B3204D0220FFF76DFDB5F98410B5F988
:105660008620FCF7FBFD214BB7F812111A880C1AA3
:1056700016B220B2864203DA97F81961B41803E033
:1056800003DD97F81971D41B1C8095F98A50B3F982
:10569000003064226B43124F93FBF2F00918B9807B
:1056A000114C0F4DA67A56B1074B1A880324EA8095
:1056B0002A81988868815988A981094D18E0034B8F
:1056C000F3E700BFA80B00206C1500207415002024
:1056D000A0110020D4100020B00B00203C160020A8
:1056E00058000020780B00208B160020AA0B002009
:1056F000AA4FB5F9062007EBC40696F97A30642064
:105700005A4392FBF0F7EF802046FFF713FD013478
:105710003918E9800235072CEAD185E0A04B5A7888
:1057200022B9B6F8D4709F49CF810AE09E48B6F8F6
:10573000D010B6F8D220B0F90600FCF78FFD994ED4
:10574000F081964E974B964A96F89270974DDC8969
:10575000907A17F0010F2C800CBF01254FF0FF3518
:1057600008B1914900E09249488807F00204454396
:1057700096F89A60098862B2002A0CBF01274FF0A0
:10578000FF3716F0010F0CBF01244FF0FF3407FB69
:105790000155604306F0020257B2DD80002F0CBFB6
:1057A00001254FF0FF3505FB010018810320FFF7AD
:1057B000C1FC7C4EF388C1180420F180FFF7BAFCCD
:1057C0003489021932812FE0794F0324BF88734B4B
:1057D00003EBC40090F87A60C4F1060306F00201FE
:1057E0004DB2002D0CBF01224FF0FF327A437049B9
:1057F000580831F8105016F0010F0CBF01264FF079
:10580000FF3606FB0522674D96B225F81460204648
:10581000FFF790FC331825F814300134072CD6D14B
:10582000614F6249F88808802020FCF76BFB002854
:1058300041D00020FFF77EFC5A4C05462080012015
:10584000FFF778FC5B4A6080137AA3B3534F5A4A40
:1058500097F8BC1001F00206F3B2CBB1B2F90030F8
:1058600097F9821097F97A70B2F9022059437B4276
:105870005343322691FBF6F16FF0310789B293FB67
:10588000F7F28F187D1993FBF6F625808E1910E03C
:1058900097F97A10B2F9026097F982704E43B2F923
:1058A00000203221574396FBF1F3ED18258097FB3A
:1058B000F1F680196080414C384D04F11006B4F9BE
:1058C0000200B5F97410B5F97620FCF7C7FC24F88E
:1058D000020F0835B442F2D1304991F8BC3003F0E0
:1058E0000402D7B22FB93148354B07881C78012202
:1058F0001CE0344D68790E280AD0082808D0324CB4
:1059000004EBC0014B78002B14BF0225002500E0FA
:10591000042500242D4F621907EB4401D0B20989F8
:105920000134FBF737FE042CF4D1DCE7A24209D2A4
:105930001E483FB230F912100132B942A8BF0F46DB
:10594000BFB2F3E70024A0461D4A1178884567D20C
:105950001C4D3BB2B5F8D200834204DD134DC21B8F
:10596000615B501860534FF48040FCF7CBFA0F4D49
:1059700070B3164B40F2DC51B3F90620114B8A424A
:10598000285FC7BFB3F8D810B3F8D220B3F8D4104B
:10599000B3F8D620FCF762FC285336E0D410002080
:1059A0008B160020580000206C1500203C160020AB
:1059B000741500209C160020780B00205600002053
:1059C000A80B0020A011002024DE0008CC16002027
:1059D000144E285FB6F8D010B6F8D220FCF73EFC83
:1059E000114BB6F81411B3F9062005EB04098A42ED
:1059F00028530ADA1020FCF785FA10B9B6F8D0005F
:105A000001E0B6F8D400A9F80000084A507818B9A7
:105A10000749084B625AE25208F10108023493E741
:105A2000BDE8F88FA0110020CC1600208B160020B6
:105A3000541600203C160020024B1868003018BF96
:105A400001207047AC0B002044F25063984203DD04
:105A5000A0F50C40A038704703498842BCBF00F550
:105A60000C40A030704700BFB0B9FFFF10B5FBF786
:105A70004DF800210446FBF759FA08B1204601E031
:105A800004F100400549FBF749F90549FBF792F895
:105A900005F02EF8034B186010BD00BF8096184B20
:105AA00035FA8E3C6800002010B5044C00232070AD
:105AB0002361FEF7CBFD606110BD00BF70160020B2
:105AC000F8B51D4614460E46FBF720F86968FBF74B
:105AD00071F83146FBF76EF82168FAF763FF206032
:105AE000FBF72EFAED68074605F10040FBF728FAB0
:105AF00006462846FBF724FA314602463846FCF7AC
:105B0000ADFBFBF703F82060FBF71AFAF8BD0000C5
:105B1000F8B5101A0C461F46FAF7F8FF0546381B71
:105B2000FAF7F4FF174B079E1968FBF743F829466D
:105B300004462846FBF73EF8214607462046FBF779
:105B400039F801463846FAF72DFF05F0D3F80E492B
:105B5000FBF730F8FBF71AFA06990860214605F1C1
:105B6000004005F0C5F80949FBF724F80849FAF7A1
:105B700019FFFBF7E5F90028BCBF00F50C40A03089
:105B80003060F8BD680000202C7D8E3FA00CB3452E
:105B900000A00C4610B50446002003460D49CA5C1F
:105BA000A2B12E2A04D1013394B1C91800220A559A
:105BB000084A0A21D25C4843A2F13001092901D8E0
:105BC000303880180E2B02D80133E7E710BD0020D3
:105BD00010BD00BF980C0020F8B52D4B93F81C01A8
:105BE00010B1012850D10AE02A4B2B4A58782B4B90
:105BF00002EB001149685868FEF7A1FA41E0274D11
:105C00006868FEF7A1FA00283ED0224C217826468B
:105C100001291ED1FEF71AFD06466069321A632A71
:105C200035D92169042912D81B4F686807EB011385
:105C30005968FEF784FA607807EB0017B96868685E
:105C4000FEF768FA22696661511C21611CE002209E
:105C500018E022693AB964780F4B686803EB0411C5
:105C60004968FEF76CFA33690A4C8B2B09D80C4A49
:105C70000A48D15C4068FEF748FA21694B1C236151
:105C800002E00320FFF710FF024A00205060F8BD39
:105C9000A01100207016002044E300081017002017
:105CA000B6E2000810B50B4CE37A8BB10A480178D4
:105CB00004290DD9094A0A4B1068516818605960C7
:105CC000FFF7D4FE0748084B028801211A80217390
:105CD00010BD00BF8B160020B615002098150020BF
:105CE0007C150020F6150020380D0020002370B52B
:105CF0001C460F4800211952142060430D4A0E4ED5
:105D00000E4D995200223250595335180C4E69608D
:105D1000AA60325035180B4E01346960AA60023314
:105D20003518022C32506960AA60E2D170BD00BF04
:105D30005015002028070020F80C002054150020E2
:105D4000B00C0020780D002070B5204C204D6079FB
:105D5000FAF7D8FE1F49FAF7E1FF2860E07BFAF76F
:105D6000D1FE1C49FAF7DAFF1B4E6860EE60A0799D
:105D7000FAF7C8FE1949FAF7D1FF194D2860207CBF
:105D8000FAF7C0FE1349FAF7C9FF6860A07EFAF778
:105D9000B9FE1449FAF7C2FFEE60A860E079FAF79D
:105DA000B1FE0E49FAF7BAFF0F4D2860607CFAF792
:105DB000A9FE0849FAF7B2FF6860E07EFAF7A2FE92
:105DC0000849FAF7ABFFEE60A86070BDD410002060
:105DD000240D00200000C8420000FA4400002041C9
:105DE0005C0D002000007A44E80C002070B5124CD5
:105DF00005460020FFF758FE6570FEF727FC0F4BA5
:105E0000A06093F81C0100266660B0420CBF01241C
:105E10000324FFF799FF0A49234601EB05156A6839
:105E200031460848FEF7C2FA074A50600120BDE833
:105E30007040FFF739BE00BF70160020A01100208F
:105E400044E300080044004010170020F8B51B4B45
:105E5000187803282ED11A494FF480524FF4004489
:105E6000A1F500650A612C61164C6068FEF75DF9CA
:105E700060B1134D4FF480566E6160682768FEF77D
:105E800059F901463846FEF740F92E610D4C20685D
:105E9000FEF74BF90028E7D00B4D4FF4004694E88D
:105EA00081006E61FEF746F901463846FEF72DF98E
:105EB0002E61D9E74FF0FF30F8BD00BF701600200B
:105EC000001001401017002000080140F7B50368DA
:105ED000164C174D23600968164E61600068FFF785
:105EE000C5FD94E80C0014480196009095E8030065
:105EF000FFF70EFE6B68114A61683668C81A1660B3
:105F0000FAF704FE0E4A0F4F1168FAF753FEFBF73B
:105F100017F82968786020680B4A431A0B483B60E1
:105F2000B0F8C4100A4B16601980FEBD400D002069
:105F300098150020A00D0020AC0D00203C0D002085
:105F400068000020D00D0020B40D0020D4100020E7
:105F5000CE0D0020264BF0B51D68024600F1100161
:105F600016781446AB195B78013203F00403DBB2F8
:105F700063B18A42F4D10020F0BD13B10A22534329
:105F8000DBB210F8011B30395B18DBB2211A022991
:105F9000F3DC0021844209D911B10A225143C9B26C
:105FA00010F8012B303A8918C9B2F3E72E2E11D11F
:105FB0000134042000220A2672432678AF197F7824
:105FC00007F00407FFB217B1303A921901340138D3
:105FD000F1D100E00022074C6420614300FB021174
:105FE00006240548B1FBF4F200FB0320F0BD00BF1E
:105FF000A401002040420F0080969800000000009D
:106000002DE9F04F9A4B91B05868C0B9994C21785E
:106010004A1E032A00F20286DFE812F0C605C60512
:10602000DF05C9056068FEF785F89349044691F8D5
:106030001C31012B00F0DF8008D3022B06D08C4CE2
:106040006068FEF772F80028ECD1DFE7242C07D156
:106050008A4B8B4A8B4C0021197011702170C5E05E
:106060002C2C02D02A2C40F08280854D834A29783E
:10607000854B157800205854844AB5B918781570A6
:10608000472868D15978502965D19878472840F039
:10609000B385D978472940F0AF851B79412B40F073
:1060A000AB850120107000F0A7BD117801293AD10D
:1060B000022D05D11846FFF74DFF754908604AE0EB
:1060C000032D07D11978532945D1714802685342ED
:1060D000036040E0042D05D11846FFF73BFF6C4BF1
:1060E000586038E0052D07D11B78572B33D168490C
:1060F0004A68504248602EE0062D07D1197865485D
:10610000302994BF00210121C17224E0072D04D160
:10611000FFF740FD604A10701DE0092D1BD1FFF70D
:1061200039FD5E4B16E0022915D1072D0CD1012057
:10613000FFF730FD41F2184250434FF47A71584B4B
:10614000B0FBF1F0188006E0082D04D10120FFF724
:1061500021FD544B1880494B4949013500202A2C18
:106160001D70087039D15048012404703EE00D2C98
:106170004D4A01D00A2C26D11478FCB1424C21782A
:106180006478A1F13000C3B2092B84BFA1F13703B9
:10619000DBB2A4F1300003F00F02C3B21101092BEE
:1061A00084BFA4F13703DBB2364C03F00F02891829
:1061B0002078CBB2C21A514251EB02043A4B002074
:1061C00018707CB912E02E490B780E2B03D82E489C
:1061D000C45401330B70127842B92A4B1A785440D8
:1061E0001C7003E0294A1078012800D00020C00765
:1061F00000F1338123E72D4B0022197808293FF65F
:106200001EAFDFE801F00A051119275F7C96A00098
:10621000622801D1022105E01A70B52C7FF40FAF7E
:106220001C78611C19700AE72149224A03261E7056
:1062300008701070204B0BE01E4E0421197032784C
:106240001D4BA1181878CAB2101818701B4B327069
:106250001C70F4E605211970164B174E1A78307829
:10626000A118CAB210183070154E1A703480E6E6C4
:106270001017002070160020A0110020B00D002083
:10628000D90D0020B90D0020980C0020CD0D002064
:10629000981500208B160020B61500204E15002002
:1062A00058150020CA060020700D0020370D002070
:1062B000B80D0020340D0020350D0020AC0C00205E
:1062C000E60C00206C4906261E700A786B4BA61857
:1062D0001878F2B210181870694B0A70198801EB1F
:1062E0000424A6B2B6F5007F01D81E8003E0002288
:1062F0001A80644B1A700024634B00F052BC5E4954
:106300005E4E0A783078A318DAB2101830705E4EFC
:106310000A7033885A4AC72B98BF5C49108898BFC7
:10632000CC545C1CA1B2884231807FF488AE072136
:1063300007E0514A08261E70137883423FF47FAE6F
:106340000021504B6EE74D4E1A70337883427FF434
:1063500076AE4F4C207806283BD005D8022813D0C3
:1063600003287FF46CAE23E0122847D030287FF456
:1063700066AE464A474C1679444A102E88BF10260E
:1063800026702178002347E0404C434E6368A068A4
:1063900021697360414B4FF47A723060404C91FB3D
:1063A000F2F618783F492680C87201223E4923E060
:1063B00036494A7912F0010004D00E79F41E634286
:1063C00053EB040035490870002839D1354AD072A2
:1063D00036E02E4EF47A14F0010104D0B07AC21ED9
:1063E000534253EB02012D4E317009B92D4CE1722D
:1063F00026482E4990F82F200A7021E023482C4986
:106400008669426942F210742A4B96FBF4F00A80C6
:10641000188001222849EFE70C328B4210DA12F87B
:10642000046C264812F8034C1E54254E25489C55F2
:1064300012F8014C16781C54234C1E550133EBE71F
:1064400019490A78002A3FF4FAAD1B4B1E78002E3A
:106450003FF4F5AD00240C701C701C4CA068E0608B
:10646000FEF7F4F8A060202000F0A2FC18490A789A
:10647000012A2FD100232EE0340D0020350D0020FD
:10648000E60C0020370D0020200D0020DC0D002040
:10649000AC0C0020B715002098150020CC0D002072
:1064A0004E1500208B160020360D0020B61500205A
:1064B00058150020CA060020BA0D00203C15002007
:1064C00086150020A0150020C015002070160020A1
:1064D000FC06002001237E4C0B70E07A00283FF47C
:1064E000AEAD7C490A78042A7FF6A9AD677807B972
:1064F0002773257B15B90FB1FFF7D4FB764E052125
:106500003378764F5C1C94FBF1F001FB1042327043
:10651000734E97F800C0734D06EB82020023724C55
:1065200072491F59DFF810E27148724E5F5097FBB5
:10653000FEF1195006FB0170DFF8009203EB040A2C
:1065400042F2107490FBF4F71668BCB253F809706D
:106550001060C6EB07084044052643F8090090FB8D
:10656000F6F00EFB01016448BCF1010F25F8024F63
:10657000195005D1023CB4F5797F98BFCAF80010D4
:1065800004331432082BCAD1FEF760F85B4D5C4C23
:106590002A68801AFAF7B6FA5A49FAF7BFFB206060
:1065A000FEF754F8286025684FF07E512846FAF728
:1065B0009FFC08B94FF07E5525600CA90DAC4A48E8
:1065C000514B0194009103C80CCBFFF7A1FA0C9A30
:1065D00064234E49B2FBF3F008800D9A3C4892FBCD
:1065E000F3F34B4C027B23800AB90A80228049498D
:1065F0000C78002C36D0424F4FF07E503968FAF7B5
:106600008DFB454D384E2B6804463068C01AFAF7AA
:106610007DFA2146FAF7CEFAFAF792FC72686968B9
:106620003E4D0746501AFAF771FA2968FAF7C2FA8E
:106630002146FAF7BFFAFAF783FC04B2384802257C
:10664000B0F902303FB2E21892FBF5F1B0F9002048
:106650008BB2B918334C91FBF5F291B26380218073
:10666000438001802B4B01201F4C1870184B616830
:10667000294A20681C7A516010601CB9DA79002A16
:106680003FF4DDAC284E294D294C01960095164F5C
:1066900094E80C00FFF73CFA61687868254E081A08
:1066A000FAF734FA1D4B1968FAF784FAFAF748FC3E
:1066B00070600A48226890F900303C68012BC4EBF6
:1066C000020131603CD0022B7FF4B9ACF2E000BF94
:1066D0008B160020B6150020D80D002008070020DA
:1066E000700C0020560D002098150020C40D0020CD
:1066F0004C0D0020806967FFDC0C0020540D002049
:106700006C0D002000007A447C1500207A150020D2
:1067100084150020480D0020BC0D002068000020DA
:10672000A80C0020720D0020A00D0020AC0D002050
:10673000400D0020D00D002080969800A40D002070
:10674000002634463546DFF874B28B4F5BF825805F
:10675000DFF864924046FAF7D9F93968FAF72AFA6D
:10676000FAF7EEFB34F80910844B421A90B2E0526B
:1067700007B2CDF80890DFF8489238460397FAF749
:10678000C5F9D9F80010FAF715FAFAF7D9FB81B272
:106790007B48142202FB0507DFF800A2039B089147
:1067A00003EB0800DAF800104B463A46FFF788F989
:1067B0000899DFF810820A185BF82500DAF800B0B3
:1067C00024F8082008905846F9F730FED7F808A0BA
:1067D000CDE904015046F9F729FE6A4BCDE90601DF
:1067E00093F8C000FAF78EF9F9F720FE60A3D3E919
:1067F0000023F9F76FFE02460B4600206249F9F7C5
:1068000093FFDDE90423F9F7B3FC0B460246DDE90B
:106810000401F9F789FF089ACDE904017968013587
:10682000501AFAF773F95946FAF778FA5146FAF717
:10683000B7F8F9F7FBFD02460B46DDE90401F9F76D
:1068400049FE0B460246DDE90601F9F791FCFAF72D
:1068500053F8089938617960B860D9F80810FAF7E8
:10686000A9F9FAF76DFB49494FF4FA62FBF7F6FC18
:10687000DDF808C034F8081034F80C20313293B237
:10688000622B98BF0020401882B224F8082010B272
:106890003F4940F6B832FBF7E1FC394B28F80400D9
:1068A00099593C48023431501436022D7FF44BAFD5
:1068B000FFF7C5BB2F68334D374CB5F9C6807E084E
:1068C000B04528BFB04625881FFA88F80FFA88F22D
:1068D00029B28A420BDD314831490068FAF76AF97A
:1068E000FAF72EFB43191FFA83F8A4F800802D4E07
:1068F0002D4D34682A68A61A3046FFF7A5F80028FF
:10690000D8BF404241F293118842CCBF0020012001
:10691000002859D03046FAF7F9F82449FAF74AF92D
:1069200004F05AF905463846FAF7ECF801462846CD
:10693000FAF740F9FAF704FB1D4B1549188040F6A9
:10694000B83200B2FBF78AFC201848F6A044A042F7
:1069500003DDA0F50C40A03804E00028BCBF00F522
:106960000C40A030134A106030E000BFAFF300804D
:10697000182D4454FB211940240D0020D80C002070
:10698000B00C0020D41000200000F03F30F8FFFFD2
:1069900048F4FFFF780D0020CE0D00206C0D002084
:1069A0000000C842A00D0020B40D0020D3023739EA
:1069B000E40C00203C0D0020720D0020D00D0020C2
:1069C0005C0D002054150020994F3C60984E002526
:1069D00031682C46C1F50C502830FAF797F89549E4
:1069E000FAF7E8F8074604F083F80F90384604F009
:1069F000F3F82F460E900FFA88F0FAF787F80EABEF
:106A000053F82710FAF7D6F806468B48DFF86CA241
:106A1000005FFAF77BF801463046F9F7C1FFFAF755
:106A20008FFA864924F80A004FF47A7200B2FBF715
:106A300015FC82B211B2DFF8489224F80A20084609
:106A40000391FAF763F8D9F80010FAF7B3F8FAF7F8
:106A500077FA83B27A48142606FB0706DFF824B2D9
:106A6000039ADBF80010069310464B463246FFF7B8
:106A700027F8DBF800C034F90A1009906046D6F810
:106A800008A00891CDF808C0F9F7D0FCCDE90401C1
:106A90005046F9F7CBFCDFF8F0B1CDE90A019BF8DD
:106AA000C000FAF72FF8F9F7C1FC5FA3D3E9002380
:106AB000F9F710FD02460B4600206249F9F734FE53
:106AC000DDE90423F9F754FB02460B46DDE9040136
:106AD000F9F72AFE089BCDE9040170680137181AFE
:106AE000FAF714F8DDF808C06146FAF717F95146CD
:106AF000F9F756FFF9F79AFC02460B46DDE9040167
:106B0000F9F7E8FC02460B46DDE90A01F9F730FB2C
:106B1000F9F7F2FE089A099B72603061B060069E38
:106B2000D9F80810F618FAF745F8FAF709FA301804
:106B3000454E81B2A15308B240F6B8324349FBF743
:106B40008DFB3F4A3053424BA8580234E85014356D
:106B5000022F58467FF44FAF90F8C21031B1344A3B
:106B6000642413683B4A93FBF4F111803A4BB0F86C
:106B7000BE001C6884420ED9384939480A68036847
:106B800042F21074D01AFEF75FFF0028B8BF4042EF
:106B9000A0427FF754AA3348334A012104882D4B81
:106BA00011701C80FFF74BBAFFF716F836E06268E9
:106BB0006078531C411CCAB263600523B2FBF3F03A
:106BC00003FB10216170FDF741FD284AA0602848B1
:106BD0000023C372137001200BE0FDF737FDA3689B
:106BE00040F6C411C01A884218D9202000F0E8F8F5
:106BF0000420FEF759FF11E01E498A78522A7FF4DB
:106C0000AAAACB784D2B7FF4A6AA087943287FF453
:106C1000A2AA194A02211170FFF79DBA11B0BDE86E
:106C2000F08F00BFAFF30080182D4454FB211940B2
:106C30003C0D0020D3023739720D002018FCFFFFF5
:106C4000780D00200000F03F5415002048F4FFFFAD
:106C5000B00C0020F4150020AC0D0020A00D002089
:106C6000B40D0020380D002008070020B6150020C4
:106C70008B160020980C0020CD0D0020D80C002091
:106C8000E80C00206C0D0020D4100020AFF3008031
:106C90003B4B2DE9F047B3F90000F9F737FF3949CD
:106CA000F9F788FF044603F097FF0646204603F0F5
:106CB0001FFFDFF8E490054699F8C180324FB8F124
:106CC000000F29D0314CB7F90200B4F802A00FFA36
:106CD0008AF1401AFEF7B8FEC8F100014246FBF700
:106CE000BDFAB4F80080B7F900700FFA88F300EB32
:106CF0000A02F81A6280FEF7A7FE99F8C1205142F5
:106D0000FBF7ACFA404487B22780B4F90200F9F7E8
:106D1000FDFE804638B206E0B7F90200F9F7F6FE4C
:106D20008046B7F90000F9F7F1FE294607464046CC
:106D3000F9F740FF314681463846F9F73BFF0146F7
:106D40004846F9F72DFE1249F9F7E8FFFAF7F8F887
:106D5000104C314620804046F9F72CFF2946064664
:106D60003846F9F727FF01463046F9F71BFE084978
:106D7000F9F7D4FFFAF7E4F86080BDE8F08700BFC8
:106D8000F615002035FA8E3C5415002050150020D1
:106D90000000204128070020D4100020034B196870
:106DA00008420CBF00200120704700BFA40E002045
:106DB000024B1A6810431860704700BFA40E0020F1
:106DC000024B1A6822EA000018607047A40E0020E7
:106DD000014B1868704700BFA40E0020037A0A46D2
:106DE000032B0FD8DFE803F00202060A0649074B1F
:106DF00000F0ECBA0449054B00F040B90249034BDE
:106E000000F00ABA704700BFB2160020EC0E002056
:106E100038B504460D46002361890B4A9952023366
:106E2000242BF9D10820FBF76DF828B1204629461C
:106E3000BDE83840FFF7D2BF0448054A2946BDE8FF
:106E4000384000F0D9B800BFCC160020B2160020A0
:106E5000EC0E00202DE9F843074608208846FBF792
:106E600051F870B10024224A414613683846E2B214
:106E70009847204921F814000134082CF3D1BDE8CB
:106E8000F8831D4A1D4D1378591CCCB204F003063B
:106E9000147005EB4609044606461548414603684A
:106EA00032463846984729F824002A886988AB88F2
:106EB0005018EA88C118881803B2991C042291FB63
:106EC000F2F00C4A0E4BA15EE052CB1E984201DA62
:106ED000811CA152135FD91C884201DD0238105376
:106EE0000136F6B202340835082ED6D1BDE8F88353
:106EF000EC0E0020CC160020A80E0020AA0E0020C8
:106F0000F00E002010B544780078002303FB03F155
:106F10001939614301F6C4115943414340F6C41283
:106F200091FBF2F1034A22F813100133072BEDD144
:106F300010BD00BFF01600202DE9F04F85784FF00E
:106F40000A0C0CFB05FCC778C5F164086E425FFAB9
:106F500088F8C7F16409B6B2002330B2002804DC17
:106F6000B8BF2C4602DB012400E0444600FB00FBD6
:106F700064430BFB07FB9BFBF4F44C4444434FF08E
:106F80000A0B94FBFBF00CEB000420B2C1EB020AED
:106F900000FB0AF44FF47A7094FBF0F404480C19E7
:106FA0001C5202335E44182BB6B2D6D1BDE8F08F26
:106FB000B4160020F8B505460F46441E14F8011F0C
:106FC00049B1054E304605F0EFFE0028F6D0861B8D
:106FD000631BBB55F2E7F8BD94E3000810B5044607
:106FE000805CFAF7D9FAA0F2EE2291B240F2DC53BB
:106FF000994288BF608910BD024B0821136001705F
:10700000704700BFDD6F0008825C044B53F822001C
:10701000410801F5777290B2704700BF040F00205D
:1070200038B50446FDF7F8FA104B40F6C4111A685B
:10703000821A8A421A460E4B01D9002119701B7818
:1070400010600BB90F2C10D10A4800210170084ABA
:107050004BB1094D182B1D4405F8014C03D10123F8
:107060000370117038BD0133137038BD240F002038
:10707000280F0020000F0020290F002038B540897C
:107080001C460E4B0D461A60A0F577710C4A4B005A
:10709000136053609360D360136153619361D36154
:1070A00008490948094A0523FDF780F90849C860DD
:1070B0000CB10848206008232B7038BDC810002090
:1070C000040F00202170000800440040A086010049
:1070D000101700200970000870B5294D2878002885
:1070E0004CD0284CA67DC6F3C006002E44D1264BBA
:1070F000186801680A68904761782278234B01F08C
:10710000070042EA00221A60A2782E7002F03F00C7
:10711000400140EAD1015960E078810041EA9211D2
:10712000227902F0010041EA80219960617901F041
:107130000F00C00140EA5202DA60A27902F07F003B
:10714000000140EA11111961E079410041EAD212CF
:10715000217A01F0030042EA40225A61627A02F089
:107160001F00800140EA91019961A07AC10041EAC3
:107170005212DA61012070BD0020287070BD00BF7E
:10718000000F0020290F0020C8100020040F00204D
:10719000825C034B53F82200C0F3CF00704700BF5E
:1071A000600F002010B50446FDF736FA154B1A683B
:1071B000811AB1F57A6F1A46134B01D90021197063
:1071C0001060187820B9A82C1AD1104B187006E05E
:1071D000022802D10E4A147001E0142801D80D498A
:1071E0000C540B490130C3B20878074A4100481DCE
:1071F0008342137004D100230449137001220A70E2
:1072000010BD00BF580F0020800F0020570F002036
:107210005C0F0020420F002038B51C46084B0D467D
:107220001A60084908484FF4E1320123FDF7BEF81F
:107230000649C8600CB10648206008222A7038BD93
:10724000C8100020A571000800440040101700205D
:1072500091710008154B10B51A780AB9002010BDBD
:107260001349002018704B78012BF7D1114A106890
:1072700001680B68984710480278082A01D908214C
:10728000017001780D4A0023D8B2023288420AD236
:1072900012F8010C12F8024C40EA0424084840F8A5
:1072A00023400133F0E7012010BD00BF570F00203D
:1072B000420F0020C81000205C0F0020450F002066
:1072C000600F00201F4B2DE9F0431B7823B31E4CA9
:1072D0001E4D277891F800C095F8008002231C4CC1
:1072E00003F10109E65C46FA07F606F00F05EEB277
:1072F00066450BD20B2E09D8E65C14F8094006EA65
:10730000080604EB0626134C44F825600233102BC4
:10731000E5D10C4B00241C700978914202D90E4B28
:10732000197811B94089BDE8F0830C4B825C19785B
:10733000084B53F8220001B1400800F5777188B27C
:10734000BDE8F083820F0020810F00208A0F00200B
:10735000FE160020940F0020880F0020890F0020C7
:10736000134B012210B51A700446FDF755F9114A66
:107370000146106811600B1A0F4841F288318B42A8
:1073800003600E4B01D900221A7018780C49E4B240
:107390000F280C5408D10B4B0B491A6801200870B8
:1073A00010680168884710BD044A431C137010BD63
:1073B000880F0020840F00208C0F0020900F0020E9
:1073C000FE160020C8100020820F002010B51C46B9
:1073D000134B1A60027A5AB1012A13D1114B0320C0
:1073E0001870114B07201870104802700C2208E02A
:1073F0000C4B022018700C4B032018700B480270C5
:1074000007220A700A490B484FF4E1320123FCF7C6
:10741000CDFF0949C8600CB1084B236010BD00BF07
:10742000C8100020810F00208A0F0020890F002043
:10743000617300080044004010170020C572000866
:10744000014B1878704700BF820F002008B54FF439
:107450000060FAF757FD08B9002008BD4020FAF790
:1074600051FD094B20B993F82D21501E0128F3D965
:1074700093F82C01012805D1034991F82D31002BF7
:10748000EAD008BD012008BDA0110020084B93F8E8
:107490002D215AB993F82E0110B9064A537801E00C
:1074A00005490B7D181C18BF01207047012070474B
:1074B000A01100208B1600209C16002010B5084B50
:1074C00093F82C211C460AB900F0A0F894F82C017E
:1074D000012803D1BDE8104000F056BA10BD00BF2E
:1074E000A011002038B50E4B1878C0B1FFF7CEFFC1
:1074F0000C4904460A78824211D060B10A4D95F8D1
:107500002C310BB900F08CF895F82C01012804D12E
:1075100000F032FA01E0FFF7D1FF02490C7038BDEC
:10752000C50F0020C40F0020A011002010B5044694
:107530004020FAF7E7FC074B002283F82D21206852
:10754000A060FFF783FF04490870BDE81040FFF713
:10755000C9BF00BFA0110020C50F00200B4B10B504
:10756000187888B1FFF792FF70B1094991F82C2182
:107570000C460AB900F06CF894F82C31012B03D1B9
:10758000BDE8104000F008BA10BD00BFC50F0020D4
:10759000A011002038B5064C05465E21A068FCF716
:1075A000B4FDA0682946BDE83840FCF7AEBD00BF79
:1075B00010170020024B5E219868FCF7A6BD00BFA3
:1075C0001017002010B50A4C5E280146A06805D1AE
:1075D0005D21FCF79AFDA0683E2105E05D2903D1FD
:1075E000FCF793FDA0683D21BDE81040FCF78DBD80
:1075F0001017002010B50446C0B2FFF7E3FFC4F334
:107600000720BDE81040FFF7DDBF0000034B93F8F3
:107610002D0108B900F092BA704700BFA0110020F8
:10762000044B93F82D0118B94FF4165000F078BAB6
:10763000704700BFA011002008B5044B9868FCF704
:1076400074FDD0F1010038BF002008BD10170020E4
:107650002DE9F041FFF7F0FF002800F04081FCF732
:10766000F5FFA04B1A68811A7C2940F23881186016
:107670009D480478651C0570002404F12406F0B2CE
:10768000FFF788FF994B33F91400F9F73FFA984A4E
:1076900005461088F9F73AFA01462846F9F73EFB05
:1076A0009449F9F787FAF9F74BFC013400B2FFF778
:1076B000A1FF032CE1D13020FFF76CFF8E49B1F917
:1076C0000000FFF797FFFFF775FF8748067816F071
:1076D000030629D1894D1020FFF75CFF2B68642435
:1076E00093FBF4F210B2FFF785FF2120FFF752FF62
:1076F000296891FBF4F004FB101484EAE473A3EB13
:10770000E47318B2FFF776FF1420FFF743FF7C4ABB
:10771000B2F90000FFF76EFF1C20FFF73BFF304679
:10772000FFF768FFFFF746FF6F490878430740F00F
:10773000B080744D0220FFF72DFFB5F900300A2507
:1077400093FBF5F0FFF756FF0220FAF7DBFB00286A
:1077500047D06D4F6D4E3878347840F63401B4FB25
:10776000F0F26B4C4A4321882A2391FBF0F800FB8E
:107770001810B2FBF3F24FEA001399B241EA022C5F
:107780001FFA8CFEC2F303224EEA02080620FFF71E
:1077900001FF0FFA88F0FFF72DFF20883F78431C88
:1077A0009AB292FBF7F107FB1120367820806E2405
:1077B0007443152394FBF3F43A206427FFF7EAFEA1
:1077C000B4FBF7F63046FFF715FF3B20FFF7E2FE6C
:1077D00007FB164291B24C1D94FBF5F000B2FFF787
:1077E00009FF2020FFF7DAFA002850D0494C132077
:1077F000FFF7D0FE2568484F002DB8BF6D4295FBBE
:10780000F7F630B2FFF7F6FE1B20FFF7C3FE236842
:107810000A26002BB8BF5B4293FBF6F142F21075CB
:1078200091FBF5F205FB121000B2FFF7E3FE2320F7
:10783000FFF7B0FE2368002BACBF4E205320FFF7AC
:10784000D9FE1220FFF7A6FE61680029B8BF4942A1
:1078500091FBF7F210B2FFF7CDFE1A20FFF79AFE68
:1078600060680028B8BF404290FBF6F696FBF5F33F
:1078700005FB136108B2FFF7BDFE2220FFF78AFE69
:107880006268002AACBF45205720FFF7B3FEFFF720
:1078900091FE15480378282B21D100240470FCF7B1
:1078A000D5FE4FF47A753C24B0FBF5F61720FFF7B0
:1078B00071FEB6FBF4F5B5FBF4F104FB11521002B6
:1078C00000B2FFF797FE1820FFF764FE04FB156374
:1078D00018B2FFF78FFEBDE8F041FFF76BBEBDE8C1
:1078E000F08100BFCC0F0020C60F0020241600201E
:1078F0004800002000007A44A40B00207C0B0020EC
:10790000F61500204C15002040000020CC1000206F
:10791000C80F002098150020A0860100154B2DE906
:10792000F04180460F4698680221FCF712FC0024C3
:107930002646781E84420F4D0DDA18F80410A86808
:107940008E190134FCF7E1FB4FF47A70B6B2FCF704
:1079500083FEE4B2EDE7F1B2A868FCF7D6FB4FF482
:107960007A70FCF779FEA8680121BDE8F041FCF7C8
:10797000F0BB00BF10170020024B01219868FCF7F4
:10798000E8BB00BF10170020024B03219868FCF7EA
:10799000E0BB00BF10170020F8B5544CA068FCF7FE
:1079A000C4FB002800F0A080A068FCF7C3FB0546DC
:1079B0000520FCF75CFE8A2D21D08E2DEDD14C4C9C
:1079C00000212E22204605F033F94A4A7C232370F9
:1079D0001378E0207D21E07084F82C1014204FF4FF
:1079E000FA71A37723754822782320766076618325
:1079F0006570628484F8243020462E2171E02020B6
:107A0000FFF7CCF90028C8D03B4C00212C2220469F
:107A100005F00EF9A021E170384B39497C207D2218
:107A2000207084F82B201878CA7A6570A076002A16
:107A300052D0344934480F686625FE0F97FBF0FC9E
:107A40006672324E5FFA8CFC06FB0C7284F8295089
:107A500006256A4342F21073B2FBF3FE03FB1E27B6
:107A60004968277391FBF0F03F0AC0B26773CF0FEC
:107A700006FB00116943B1FBF3F5642203FB151308
:107A8000E9B202FB0010010AE07321482174018869
:107A90005FFA8EFE63741B0A02FB0CECA374B1FB4D
:107AA000F2F224235A4390B21A4A010A1388E07171
:107AB0002172180A1849207518480A8801884FEA67
:107AC0001C2EE374130A84F80AC084F80BE0A77331
:107AD0006275A375217702E0202384F829300648D7
:107AE0002C21FFF71BFF58E7F8BD00BF101700203F
:107AF000FC0F0020CC100020D00F0020B615002075
:107B00008B16002098150020A08601006079FEFFEA
:107B1000581500207A1500204E15002084150020ED
:107B200008B50246032303480021FCF73FFC024B43
:107B3000186008BD0038014010170020024B18687B
:107B40000068FFF7EDBF00BF2C10002008B5044B04
:107B50001860FFF7F3FFBDE8084001F0EFB800BF81
:107B60002C100020034B187808B100F0F1BE01F092
:107B70005FB900BF30100020232801D100F0E8BE1B
:107B8000044B19688A7A824202D10120FCF734BE84
:107B9000704700BF2C10002070B50646B6FBF2F40B
:107BA0000846154614B12046FFF7F6FF05FB14649E
:107BB000024B195D00F8011B70BD00BF18E50008FD
:107BC0002DE9F041027803460130202AFAD0092A33
:107BD000F8D02D2A02D10346414D04E02B2A08BFDC
:107BE00003464FF07E551E460024334616F8010B1F
:107BF000A0F13007F9B209290DD83A492046F8F723
:107C0000D9FF04463846F8F781FF01462046F8F7C9
:107C1000C9FE0446E9E72E2817D1324F334616F83D
:107C2000010B3038C2B2092A0FD8F8F76FFF394676
:107C3000F9F774F801462046F8F7B4FE29490446DE
:107C40003846F8F7B7FF0746E8E71878652801D007
:107C5000452839D15E782D2E02D19F1C012605E0E2
:107C60002B2E01D05F1C00E09F1C00267B1E0027EE
:107C700013F8012F303AD1B2092903D80A2000FBAA
:107C80000727F5E7B7F59A7F28BF4FF49A77B846EC
:107C90004FF07E51B8F1070F07D908461249F8F79F
:107CA00089FFA8F108080146F4E707F0070737B194
:107CB00008460C49F8F77EFF013F0146F7E72EB171
:107CC0002046F9F72BF804E04FF07E512046F8F7F4
:107CD00071FF01462846F8F76DFFBDE8F08100BF4F
:107CE000000080BF0000204120BCBE4C10B5441EE7
:107CF00014F8011F21B1034B1868FCF706FAF7E7E7
:107D000010BD00BF101700200148FFF7EFBF00BFF4
:107D10003DE5000810B50748FFF7E8FF0024064BD3
:107D200006481A19E15852680C34FAF7C7FBC02C00
:107D3000F5D110BD6BE500083CE4000881E50008C2
:107D400070B5FCF783FC244C244B4FF47A71B0FBE4
:107D5000F1F11A7822482378FAF7B0FBFFF738F8E8
:107D600005462048204902682048B2FBF1F1FAF7A5
:107D7000A5FB00241E4B53F8241051B1012000FA3A
:107D800004F0284202D01B48FAF798FB0134E4B211
:107D9000F0E70220FFF702F868B1174A174B117895
:107DA000174853F82110FAF789FB1648017A11B1E8
:107DB0001548FAF783FB154C1548FFF797FF248801
:107DC000FCF762F90246134821464FF46673BDE89A
:107DD0007040FAF773BB00BF40000020CC100020B9
:107DE00089E500088801002040420F00C7E500082F
:107DF0005CF30008E5E5000866070020FCE40008E5
:107E0000E9E50008D0150020F3E500082C07002064
:107E1000A6E80008F7E5000838B50C6805462046D6
:107E200005F09EF8024628682146BDE8384005F076
:107E3000C7B8000008B50548FFF758FF0A20FCF74F
:107E400016FC0020BDE80840FCF7D6BC29E6000877
:107E500008B50748FFF74AFF064B93F89403F9F774
:107E6000F3FFFAF701F8BDE80840FFF7E3BF00BFF2
:107E700038E60008A01100207FB5044605F070F830
:107E8000082825D100231F49E25C086885186E7810
:107E900006F00301022908BF203AE2540133082BFF
:107EA000F1D10025665D1848314604F07DFF28B108
:107EB00001356019314604F077FF18B11348FFF718
:107EC00015FF1DE0082DEDD120461149FFF772F88E
:107ED0001048FFF70BFF00230F4A04A9981890F8E9
:107EE00008218818084A995C0133082B00F80C1CFB
:107EF000F2D100208DF80C0001A90848FAF7DEFA4B
:107F00007FBD00BFA401002094E3000842E6000802
:107F1000A812002062E60008A011002084E50008F5
:107F200008B5FDF793FF01300CBF03480348BDE8D7
:107F30000840FFF7DBBE00BF77E600089DE60008BB
:107F40002DE9F041054605F00BF80446FAF780F9F3
:107F5000064694B92A48FFF7C9FE2A4951F8241069
:107F600049B1012202FA04F2324202D02648FAF75D
:107F7000A5FA0134F1E7254821E0284624492246A4
:107F800005F01EF858B92348FFF7B0FE224C54F80C
:107F9000041F0029EFD01C48FAF790FAF7E72B7876
:107FA0002D2B04D10135013C4FF0010801E04FF0C9
:107FB00000080026134850F8267027B91748BDE876
:107FC000F041FFF793BE28463946224604F0F8FFF9
:107FD000A0B9012000FA06F0B8F1000F03D0FAF7BB
:107FE0002FF90F4802E0F9F797FF0E48FFF77EFEE2
:107FF0000D483946BDE8F041FAF760BA0136D9E7D5
:10800000BBE60008A0E30008E5E50008A6E80008D4
:1080100066F10008CEE600089CE30008E3E60008ED
:10802000FDE6000807E7000884E5000810B50446EF
:108030000848FFF75BFE084A084809490023036027
:1080400013700B70FDF790F82046BDE81040FFF765
:10805000FFBE00BF10E700083110002064100020B0
:108060003010002008B50448FFF740FEF9F75CFF28
:10807000BDE80840FFF7DEBE28E70008F8B5074670
:1080800004F06EFF044638B91A491B4B4A791B4865
:10809000511E53F8211028E038461949224604F0B1
:1080A0008FFF60B91748FFF721FE174C54F8041FE3
:1080B00019B11648FAF702FAF8E7154805E0002565
:1080C0000D4B53F8256026B91248BDE8F840FFF77C
:1080D0000DBE38463146224604F072FF01350028B5
:1080E000EED10448314645710B48BDE8F840FAF737
:1080F000E5B900BFA0110020E0E3000841E7000857
:1081000066F1000855E70008DCE30008E5E5000833
:10811000A6E8000868E7000880E7000810B50446F4
:10812000204604F01DFF10F0FF0F07D10B490C484B
:1081300091F89413BDE81040FAF7C0B9204604F056
:108140002DFC022808D8054B064C83F89403F9F758
:108150008BFEF9F745FEE3E710BD00BFA01100203C
:1081600092E70008B6EA000870B5044604F0F8FE8D
:1081700008B9204830E020461F4905F069FB00247B
:108180002646254678B12CB1012C06D104F006FC18
:10819000064602E004F002FC0546002016490134C0
:1081A00005F056FBEEE70B2D05D914480C21BDE870
:1081B0007040FAF783B9012C08DC114A114832F9F2
:1081C00015202946BDE87040FAF778B9A6F57A730C
:1081D000B3F57A7F04D90C48BDE87040FAF76EB960
:1081E0000A4829463246FAF769F9054820F8156029
:1081F00070BD00BFA8E7000880EA0008E2E70008B9
:108200005416002008E8000820E8000842E80008AA
:1082100038B5054604F0A4FEC0B268B90446124958
:10822000124801EB4402B2F8422021460134FAF729
:1082300045F9152CF3D138BD284604F0AFFB1428BE
:1082400004460BDC2021284604F0AEFD04F0A6FB1A
:10825000054B03EB4404A4F8420038BD0448152143
:10826000BDE83840FAF72AB9D41000205BE80008CE
:1082700067E80008931E222B88BF0A22031E10B550
:108280000C4603DA2D2001F8010B5842FFF784FC5D
:1082900000210170204610BD30B587B005460C4660
:1082A00003A800210C2204F0C3FC28460021F8F7A3
:1082B0003DFE20B128462949F8F774FB03E0284623
:1082C0002649F8F76DFB2649F8F774FCF8F738FEF5
:1082D000054685EAE570A0EBE5700A226946FFF7DE
:1082E000C9FF002D01DB202300E02D2368468DF817
:1082F0000C3004F035FE012807D130228DF80D2016
:108300008DF80E208DF80F200CE0022805D13021C9
:108310008DF80D108DF80E1004E0032802D13020E6
:108320008DF80D00694603A804F018FD03A804F0B9
:1083300017FEC51EEDB22A4603A9204604F0AEFE84
:10834000002363552046074904F008FD03A9204691
:10835000491904F003FD204607B030BD6F12033AFF
:1083600000007A4436E6000837B5037904460D4626
:10837000052B34D8DFE803F003060A0D11148168D9
:1083800009782DE0806890F9001029E08368198849
:1083900026E08268B2F9001022E0816809681FE0D7
:1083A000806869460068FFF777FF01461148FAF7D1
:1083B00085F8F5B1E068F8F7A9FB6946FFF76CFFAF
:1083C00001460D48FAF77AF82069F8F79FFB6946ED
:1083D000FFF762FF01460848FAF770F809E000214C
:1083E0000648FAF76BF825B10548E1682269FAF703
:1083F00065F83EBDF0E50008EFE5000891E80008EB
:108400008DE800082DE9F047064604F0A9FD054671
:1084100020B1012819D133782A2B16D14748FFF70C
:1084200065FC002414266643454F4648F159FAF787
:1084300045F8B8192946FFF797FF01344248FFF77E
:1084400055FC6F2CEED1BDE8F08730463D2104F09D
:10845000ABFC002857D0441C204604F09FFA82460B
:108460002046FFF7ADFB0027054614247C43DFF8C8
:10847000D09054F80980404604F072FD414602460F
:10848000304604F09DFD002835D14C44E068F8F7F3
:108490003DFB01462846F8F73FFD002829D020691A
:1084A000F8F734FB01462846F8F72CFD002820D0C9
:1084B00020792279052818BF5546052A0FD8DFE80C
:1084C00002F003030606090CA1680D7007E0A2681C
:1084D000158004E0A068056001E0A1680D604146D8
:1084E0001A48F9F7EBFF20460021BDE8F047FFF7F7
:1084F0003BBF174803E001376F2FB6D11548BDE8E1
:10850000F047FFF7F3BB0446142565430C4F314693
:1085100055F80780404605F025F850B10948414616
:10852000F9F7CCFF78190021FFF71EFF0648F9F78D
:10853000C5FF01346F2CE7D1BDE8F08794E800084F
:108540007CF3000873E90008A6E80008A9E8000821
:10855000B4E80008D9E800082DE9F043584885B090
:10856000584CF9F7ABFF5848FFF752FE6279574B6A
:10857000511E574853F82110F9F7A0FF2069002138
:10858000F8F7ACFC002858D10025266900213046B8
:10859000F8F7A4FC00284CD101354E482946D4F800
:1085A0001490D4F81880E769F9F788FF3046002165
:1085B000F8F79EFC10B14848F9F780FF694630464D
:1085C000FFF76AFE01464548F9F778FF4846002163
:1085D000F8F78EFC10B14048F9F770FF694648463D
:1085E000FFF75AFE01463D48F9F768FF4046002173
:1085F000F8F77EFC10B13848F9F760FF694640464D
:10860000FFF74AFE01463548F9F758FF3846002182
:10861000F8F76EFC10B13048F9F750FF694638465C
:10862000FFF73AFE01462E48F9F748FF10340C2DAB
:10863000ABD12C48691CF9F741FFF9F709FE2A4C28
:10864000064654F8041F19B12848F9F737FFF8E730
:108650000D46274850F8251049B1012202FA05F2CB
:10866000324202D02348F9F729FF0135F1E7154BD3
:10867000214ACE1896F808418B5C04A801310519EF
:10868000082905F8103CF2D100241C4869468DF8F1
:108690000840F9F713FF14256543194E1948A959E5
:1086A000F9F70CFF00217019FFF75EFE0134164840
:1086B000FFF71CFB6F2CEED105B0BDE8F08300BFC7
:1086C000F6E80008A0110020B6EA0008E0E3000880
:1086D00026E9000831E9000880EA0008F0E5000812
:1086E00084E5000839E900089CE300084BE900082C
:1086F000A0E3000859E9000894E3000866E90008CF
:108700007CF300086FE90008A6E800082DE9F043B3
:1087100089B0044604F024FCC6B2002E6AD1794820
:10872000FFF7E4FA784C20690021F8F7D7FB38BB53
:10873000013676483146F9F7C1FE206904A9FFF7F2
:10874000ABFD01467248F9F7B9FE606904A9FFF76D
:10875000A3FD01466E48F9F7B1FEA06904A9FFF731
:108760009BFD01466A48F9F7A9FEE06904A9FFF7F5
:1087700093FD01466748F9F7A1FE10340C2ED2D1C3
:108780000025654C2F46A8464FF000091034B1452E
:1087900014DA404654F8101CF8F704F954F80C1C8D
:1087A00080462846F8F7FEF854F8081C0546384677
:1087B000F8F7F8F809F101090746E7E75748CDF857
:1087C000048002950397FFF791FA002401A823582B
:1087D000534923F00040F8F7A9FB5249524A0434A8
:1087E000002814BF10460846FFF780FA0C2CEDD184
:1087F0004E4870E020464E49052204F0E1FB38B9AE
:10880000414B0022C1181030C0280A61F8D176E02F
:1088100020464849042204F0D3FB0546204605BB08
:10882000202104F0C1FA002869D0461C304604F02B
:1088300097FB2C460746404850F824500DB93F4856
:1088400049E030462946FAB204F0BAFB38B920466E
:10885000FCF728FD3A482946F9F730FE47E0013495
:10886000E9E704F09BF8461E0B2E074643DC204642
:10887000202104F099FA054640B1451C2846FFF72F
:108880009FF9214B3F01D851012400E004462846BE
:10889000202104F089FA054640B1451C2846FFF71F
:1088A0008FF91949013401EB061250612846202145
:1088B00004F07AFA054640B1451C2846FFF780F9D6
:1088C000114B013403EB061188612846202104F086
:1088D0006BFA18B91B48FFF709FA10E00130FFF7EF
:1088E0006FF9094A032C02EB0616F061F2D1164823
:1088F000FFF70CFF03E015480C21F9F7DFFD09B085
:10890000BDE8F08381E90008A0110020ACE900086F
:10891000B2E9000884E50008B4110020B6E90008B7
:108920000AD7233C7DE9000879E90008A6E8000899
:10893000C5E90008CBE90008E0E3000868E70008A3
:10894000D0E90008E3E90008B6EA00081DEA0008DB
:10895000F0B5694B87B01A783AB9012018706748AA
:10896000FFF7C4F96648FFF7C1F9664C2068FBF7CA
:10897000DCFB002800F0BD802068FBF7DBFB09284A
:108980000146614A01D03F2851D1002517685F4C4C
:108990002E462FB15E4821683A4604F011FB10B90B
:1089A000254606B926465B490C348C42F1D3C6B144
:1089B0003468D5F800E03B46E05C1EF803108142C5
:1089C0000DD1534A41B92D2B06D820244E48D454FA
:1089D00001330360D15404E0D0540133ECE74A4939
:1089E0000B60494A14681CB1AE4201D13C4612E00A
:1089F0004948FFF77BF9AE4209D856F80C0BFFF750
:108A000075F9404B09211868FBF77FFBF3E73C48F9
:108A1000FFF76CF900243C4B18688442A5D2394911
:108A20003B4A0868115DFBF770FB0134F3E71368FC
:108A30002BB9042838D13648FFF7F8FA59E00C284A
:108A400001D136488CE70A2901D00D2948D12E4D95
:108A50003348FFF74BF92E4C2A6832490023A354C0
:108A60000493009103A8294910220C23039403F0D6
:108A700099FF054638B1006804F072FA0130AA681F
:108A80002018904702E02848FFF730F900213022F3
:108A90001F4804F0CDF818481B4B027800211960DC
:108AA000002A7FF45FAF24E00C28CAD07F2903D1CD
:108AB0005BE72F2B3FF659AF1F297FF656AF7E2974
:108AC0003FF653AF13B920293FF44FAF104C0E4877
:108AD0000C4AE154013303601068FBF716FB44E7CE
:108AE0007F29E6D10A485C1E0021015514600F4819
:108AF00039E707B0F0BD00BF3010002045EA00089C
:108B00007DEA000810170020641000203CE40008F3
:108B100031100020FCE4000882EA000887EA00081F
:108B2000A6E80008197E000892EA0008B3EA0008E7
:108B3000F8B5174E174C184D0746C1B23068217072
:108B4000FBF7E3FA22782B78C7F3072182EA0300C8
:108B5000287030682170FBF7D8FA21782A783068BD
:108B600081EA0203C7F307412B702170FBF7CDFAAE
:108B70002078297880EA0102390E306821702A7045
:108B8000FBF7C3FA2B78207880EA03012970F8BD3F
:108B90001017002069100020C5100020F8B50D4EF8
:108BA0000D4D0E4CC1B2074630682970FBF7ADFA87
:108BB0002A782378391282EA0300207029703068FD
:108BC000C9B2FBF7A2FA23782A7882EA0300207060
:108BD000F8BD00BF101700206C100020C510002049
:108BE000054B10B5044621461868FBF78EFA03487A
:108BF00002785440047010BD10170020C5100020EA
:108C0000034B04491A78885C01321A70704700BF20
:108C10006A1000208510002010B5FFF7F1FF044610
:108C2000FFF7EEFF04EB002080B210BD10B5FFF798
:108C3000F3FF0446FFF7F0FF04EB004010BD000017
:108C400038B5044624200D46FFF7CAFF4D20FFF734
:108C5000C7FF002C0CBF3E202120FFF7C1FF064BB1
:108C6000002228461A70FFF7BBFF04480078BDE8D1
:108C70003840FFF7B5BF00BFC51000206F100020BF
:108C800001460020FFF7DCBF01460120FFF7D8BFF7
:108C9000014B1878FFF7A4BFC510002070B505463A
:108CA00008460E46FFF7ECFF2C467219D0B2E3B22D
:108CB000984204D014F8010BFFF792FFF5E770BD5E
:108CC00010B5441E14F8010F10B1FFF789FFF9E742
:108CD00010BD00002DE9F843002701240025144BA6
:108CE000187885421CDA1349134B15F801800C22C1
:108CF00002FB0830406804F033F981460CB13F189C
:108D00000CE026464E4509DA0B4A0C2101FB0823EC
:108D10005868805DFFF764FF0136F3E70135DEE751
:108D200024B1F8B2FFF7ACFF0024D7E7BDE8F88321
:108D30006D100020701000206C00002070B5394DBF
:108D4000FF211522284603F073FF002302202B7019
:108D5000FEF724F8012418B102206C70A8700324D7
:108D60000420FEF71BF868B12E4E03214FF400508B
:108D70003155651CF9F7C6F818B104227255023452
:108D800000E02C460220FEF709F848B1254B0520EB
:108D90001E190621072518557170B570033404E0BB
:108DA0000820FDF7FBFF0028F0D12020F9F7AAF8F2
:108DB00018B11C4B08221A5501344FF48070F9F792
:108DC000A1F830B117480A2601190B2506554D7038
:108DD0000234154A134B5079082801D00E2802D1CD
:108DE0000C261E5501340D2104201955651CF9F778
:108DF00089F818B10B4811224255A51C0A491323C2
:108E000091F82E21074E6C1C101C18BF01207355C1
:108E1000F9F778F810B114203055AC1C034B1C70D6
:108E200070BD00BF70100020A01100206D10002048
:108E3000F8B5B54C2068FBF778F9002800F04785B5
:108E40002068FBF777F9B14A0346117871B9B0F1A0
:108E50002404634253EB040111700029E9D1AC4AA8
:108E60005478002CE5D1FEF787FEE2E7012904D112
:108E70004D280CBF0223002321E0022904D13C2805
:108E80000CBF032300231AE003290FD140284FF021
:108E9000000101D91170CCE79E489F4C03709F4898
:108EA000217001709E490B70042308E0042908D149
:108EB0009B499C480C78037063400B70052313702A
:108EC000B7E70529B5D19448924C017822788A42B7
:108ED000934A07D914785C401470934A53544B1C3E
:108EE0000370A6E71078984240F0EC848D4B197817
:108EF0007B2900F0318300F2C5806E2900F07B836E
:108F000060D8682900F0448325D8652900F01082D4
:108F100019D8642940F0D1840720844CFFF7B0FEB3
:108F2000E620FFF75DFE6079FFF75AFE0020FFF7AD
:108F300057FE94F819017E4B7E4A00280CBF10465C
:108F4000184600F06BBC662900F07082672940F07B
:108F5000B48479481DE36B2900F02B8323D8692959
:108F600000F01B836A2940F0A8841020FFF788FED8
:108F70006748724CC07AFFF733FE71490878FFF7F3
:108F80002FFE2068FFF7D4FD6068FFF7D1FD6D4A22
:108F9000B2F90000FFF702FE6B4BB3F90000FFF7D8
:108FA000FDFD6A4A24E36C2900F015836D2940F029
:108FB00084840620FFF764FE65490868FFF7B8FD62
:108FC000644A15E3732900F083833CD8702900F0CC
:108FD0004183C0F02183712900F04F83722940F052
:108FE0006C84524C1620FFF74BFE0020FFF7D6FD95
:108FF000B4F9D000FFF7D2FD574DB4F9D200FFF716
:10900000CDFDB4F9D400FFF7C9FDB5F9B600FFF7FF
:10901000C5FD0020FFF7C2FD0020FFF789FDB5F96F
:1090200028000A2390FBF3F0FFF7B8FD94F8040141
:10903000FFF7D6FD94F80601FFF7D2FD94F805017D
:10904000FFF7CEFD73E3762900F04D830DD8742928
:1090500000F02B83752940F030842F20FFF710FE9D
:109060003E48FFF72DFE00F02BBC772900F020834F
:10907000782940F02284384C3820FFF701FE04F1B3
:10908000400537E2D02900F0878300F2CA80CA2960
:1090900000F00F816CD8A42900F0EE8310D8A0292D
:1090A00040F00B840C20FFF7EBFD2D492D4C086898
:1090B000FFF73EFD2C4A1068FFF73AFD2068ADE34C
:1090C000C82900F0ED80C92940F0F783FFF798FD2B
:1090D0000F4B1A4CD872FFF793FD19490870FFF730
:1090E000A5FD2060FFF7A2FD6060FFF795FD154A22
:1090F0001080FFF791FD144B18801C48017841F057
:1091000002040470E4E000BF101700206810002083
:109110008B1600206B1000206E1000206A100020BB
:10912000C51000206F10002085100020A011002025
:109130001C000080140000805800002098150020BA
:10914000B61500204E15002058150020CA06002034
:109150001C160020A40B0020D410002028FC0008BE
:10916000E8F7FF1FF0F7FF1FECF7FF1FFC060020DA
:10917000CD2900F01B8322D8CB2900F0AB80CC296D
:1091800040F09B83FFF73CFDC74CE077FFF738FDCD
:1091900084F82000FFF734FD84F82300FFF730FD4A
:1091A00084F82400FFF72CFD84F82500FFF728FD44
:1091B00084F82100FFF724FD84F8220088E0CE29FE
:1091C00000F0FE82CF2940F07883FFF725FDFFF7FE
:1091D00023FDB64CB44DA4F8D000FFF71DFDA4F854
:1091E000D200FFF719FDA4F8D400FFF715FDA5F88C
:1091F000B600FFF711FDFFF719FDFFF70DFD0A237C
:1092000058432885FFF7FCFC84F80401FFF7F8FCBD
:1092100084F80601FFF7F4FC84F80501FFF7F0FC81
:1092200056E0D52900F0A6810FD8D2296BD0C0F026
:109230008282D32977D0D42940F03F839A4C0020F2
:10924000FFF71EFD04F1400568E1F02900F0D98226
:109250000CD8D6294ED0EF2940F02F83FFF7DCFC45
:10926000914CA085FFF7D8FC608531E0FA2900F029
:10927000AF82FE2940F021830820FFF701FD8C4CCE
:109280008C488D4B01682068B1FBF3F2B0FBF3F31F
:109290004FF47A7101FB0234884AD4800024A8E29A
:1092A0000024FFF7B9FC864A10530234102CF8D181
:1092B0000EE0844C04F10A05FFF7A2FC0134607053
:1092C000FFF79EFCE072FFF79BFCAC426075F3D1A8
:1092D00000208BE200247C4801788C42F8D27B4D40
:1092E000655DFFF799FC704A013402EB4505A5F86E
:1092F0004200F0E70024FFF78FFC754A1053023458
:10930000102CF8D1E4E7734C6478002CE0D1FFF71F
:1093100077FC6649022881F8940388BF81F894435A
:10932000F8F7A2FD3FE2FFF777FC6B490880CFE733
:109330006A4D0B20FFF7A4FCB5F90000FFF72EFCE7
:10934000FAF7A2FE00B2FFF729FC0220FDF726FD86
:1093500005460420FDF722FD04460820FDF71EFD0A
:10936000820042EA4401294320208CB2FDF716FD19
:1093700044EAC00084B21020FDF710FD44EA001357
:1093800018B2FFF70BFC534A1079D1788400537858
:10939000907944EA4101194341EAC0045179537A72
:1093A00044EA411040EA83144D48C17944EAC113AC
:1093B000047A417A43EA042343EA4124D379117AB7
:1093C00044EA8324927A44EAC123417B43EA02348B
:1093D000827B44EA4133017C43EA8234027944EAE5
:1093E0000143417C43EA0214827C44EA4143C17C4C
:1093F00043EA8244007D44EAC142334B42EA0054CE
:109400000020197803468B420AD2304D01225D5D5F
:1094100002FA05F525421CBF9A4010430133F2E7DA
:10942000224CFFF785FB94F8940381E11220FFF7AB
:1094300027FC2C490C88B4F5806F2B4CB4F9000044
:1094400008D8FFF7ABFBB4F90200FFF7A7FBB4F9AC
:1094500004000EE0082590FBF5F0FFF79FFBB4F940
:10946000020090FBF5F0FFF799FBB4F9043093FB91
:10947000F5F01E4CFFF792FBB4F90000FFF78EFBEE
:10948000B4F90200FFF78AFBB4F90400184CFFF7A7
:1094900085FBB4F90000FFF781FBB4F90200FFF788
:1094A0007DFBB4F90400B6E1D4100020A011002027
:1094B000880100208401002040420F006415002034
:1094C000CC160020D31000206D100020701000205A
:1094D000541600208B160020F41500202C070020C5
:1094E0009C16002048000020241600209A0B002023
:1094F000DC150020B4F97400FFF750FBB4F97600D6
:10950000FFF74CFBB4F97800FFF748FB94F87A00BA
:109510000834FFF765FBAC42ECD1D1E1FFF77CFBEF
:10952000A4F87400FFF778FBA4F87600FFF774FB4B
:10953000A0F57A72072893B298BF84F87B00B3F540
:109540007A7F98BFA4F87800FFF75AFB84F87A0076
:109550000834AC42E2D1B3E10820FFF791FB0024CC
:10956000B04AA31893F87B000834FFF739FB402C6E
:10957000F6D1A5E10020FFF783FB0024FFF740FBB5
:10958000A84AA3180834402C83F87B00F6D197E151
:10959000A5481021FFF782FB92E11020FFF770FB36
:1095A0000024A248005F0234FFF7F8FA102CF8D12B
:1095B00086E10520FFF764FB9D4BB3F90000FFF740
:1095C000EDFA9C48B0F90000FFF7E8FA9A490A78EA
:1095D00002F00100ACE0994C0620FFF751FBB4F912
:1095E0000000FFF7DBFAB4F90200FFF7D7FA944A5C
:1095F000B2F900000FE10720FFF742FB9148007825
:10960000FFF7EEFA0020FFF7C9FA8F4BB3F900001D
:10961000FFF7C4FA0020FEE0824C0720FFF730FB82
:10962000E07FFFF7DDFA94F82000FFF7D9FA94F80D
:109630002300FFF7D5FA94F82400FFF7D1FA94F845
:109640002500FFF7CDFA94F82100FFF7C9FA94F846
:1096500022006DE01E20FFF713FB7C4C04F10A058D
:1096600001346078FFF7BCFAE07AFFF7B9FA607D61
:10967000FFF7B6FAAC42F3D122E175490A785400FB
:1096800004F0FE00FFF7FCFA0024714803789C42C6
:1096900080F016816F496348625C013400EB42033D
:1096A000B3F94200FFF77AFAEFE7FFF713FB07E1A0
:1096B000674900240878FFF7E3FA654A1078844286
:1096C00080F0FE80634B185DFFF78AFA0134F4E7FF
:1096D0000820FFF7D5FA0124E0B20134FFF780FA41
:1096E000092CF9D1ECE0FFF78BFA06461220FFF7C0
:1096F000C7FA0EB9584902E0102E03D157490D6838
:109700004C6801E0002425463046FFF769FA2846F8
:10971000FFF70EFA2046FFF70BFA514A1068FFF7E1
:1097200007FA0020FFF73AFA0020FFF737FA002087
:10973000FFF756FAC4E0FFF763FA0546FFF776FA3B
:109740000746FFF773FA0646FFF770FA0446FFF77D
:1097500063FAFFF761FAFFF753FA65B93E484149EA
:10976000012207604660CD710A73002C3FF4B0AD52
:109770003B4B1C60ACE5102D7FF4AAAD3748076069
:1097800046600CB1364A1460374B344802211970D8
:10979000011DFCF79BFB9BE53248417800297FF4D3
:1097A00097ADF8F7C1FBF8F71BFB91E52D4C6378FB
:1097B000002B7FF48DAD2D494FF4C870088087E5EC
:1097C0002848417800297FF483AD012282737FE528
:1097D000244B5C78002C70D1254991F89403F8F75C
:1097E00033FBF8F741FBF8F7FBFA2046FFF748FA9E
:1097F00066E02048005F0234FFF7D0F9082CF8D16A
:109800005EE0084C0420FFF73BFAB4F92C00FFF7A8
:10981000C5F9B4F92A00FFF7C1F951E0FFF788F95B
:109820004EE000BFD41000203C160020CC160020D3
:109830007A15002084150020FC060020780B0020FB
:10984000F6150020CC100020B4150020D310002005
:109850006D100020701000207C1500205C15002089
:10986000201600208B16002008070020600700202B
:10987000A011002064150020154C23789800411C8D
:10988000C8B2FFF7FDF92078FFF7AAF90024104AC3
:1098900013789C4214D20F48005DFFF7A1F90E49DE
:1098A000085DFFF79DF90D4A105DFFF799F90C4B24
:1098B000185DFFF795F90134E9E70020FFF7E4F9B7
:1098C000FFF7E6F9074900200870FFF7B2BAF8BDC4
:1098D000B71500203C15002086150020A01500209B
:1098E000C0150020681000202DE9F0410746884689
:1098F00016460024B44213D00025BD420AD0094BBD
:109900000135DA68EDB282F48050D8604046FAF74B
:10991000AEFEF2E73C200134FAF7A9FEE4B2E9E733
:10992000BDE8F081001001400F4B1A6842F00100C1
:10993000186059680D4A0A405A60186820F084710E
:1099400021F480321A60186820F4802119605A6866
:109950004FF41F0122F4FE0058609960044B4FF051
:1099600000629A60704700BF001002400000FFF8DC
:1099700000ED00E0164A174B516801F00C00042876
:1099800003D0082805D0144801E01449086818607D
:1099900011E051685068C1F383410231C00301D422
:1099A0000F4A06E052680D4812F4003F026818BFE3
:1099B000520851431960064B0A485A68054BC2F3D6
:1099C0000311415C1A6822FA01F21A60704700BF65
:1099D000001002408801002000127A00840100205B
:1099E00000093D00740100201FB50023574C4FF4BF
:1099F000E0110093019302930391226842F48033B3
:109A00002360A16941F01002A261504C236803F465
:109A100000310191009A531C0093019919B9009AE1
:109A2000B2F5A06FF1D12168484B11F4003401D098
:109A3000022416E01A6842F0010119600094434BB9
:109A40001C6804F00202019200994C1C0094019AD7
:109A50001AB90099B1F5A06FF1D11B6899073BD5F0
:109A600001243B4902940A6842F010030B600C6821
:109A700024F003020A600B6843F002040C60A1F5B5
:109A80008053596859605A685A605C68314A44F496
:109A900080615960146824F0704111602E4C2F4988
:109AA0000C605C6824F47C145C60146844F000442E
:109AB0001460946824F400449460043A9268120498
:109AC00049BF274A4FF4E0120A604FF48012039214
:109AD0000299012901D119E0FEE702291AD168B1E2
:109AE0000398B0F5801F02D14FF4A01205E0039B4C
:109AF000B3F5E01F02D14FF400120392134B5968E3
:109B0000039841EA000242F4803002E0596841F4CF
:109B1000601058600D4B1A68184642F08071196049
:109B200002680A4B9201FBD5596821F00300586086
:109B30005A6842F002015960044B586800F00C0268
:109B4000082AF9D1FFF716FF1FBD00BF0010024021
:109B5000002002400410014000127A00840100201D
:109B6000001BB700CB78F0B5DA0648BF8A780988C1
:109B700003F00F0548BF154311F0FF0F1ED0046816
:109B80000022012707FA02F707EA0106BE4211D1B7
:109B900097004FF00F0C0CFA07FC05FA07F724EAC0
:109BA0000C04282B44EA070401D1466102E0482B4B
:109BB00008BF06610132082AE3D10460FF2920D9D9
:109BC0004468002202F10806012707FA06F707EAAF
:109BD0000106BE4211D197004FF00F0C0CFA07FCA2
:109BE00005FA07F724EA0C04282B44EA070401D1FC
:109BF000466102E0482B08BF06610132082AE1D124
:109C00004460F0BD08B5154B98420BD101214FF4CB
:109C1000805000F0ADFD4FF480500021BDE80840B9
:109C200000F0A6BD0E49884207D14FF480400121C3
:109C300000F0AAFD4FF4804009E00A4A90420BD19F
:109C40004FF40040012100F09FFD4FF4004000213F
:109C5000BDE8084000F098BD08BD00BF00300140DD
:109C600000380040003C00400B8810B54C8802884A
:109C700023438C8802F441522343CC8823430C892C
:109C800023434C8923438C892343CC89098A23436A
:109C90001A4393B20380828B22F400631A04130CDC
:109CA0008383018210BD038819B199B241F040034A
:109CB00003E023F040010A04130C03807047818104
:109CC0007047808980B27047038919420CBF002019
:109CD00001207047426810B522F470230A6823F40B
:109CE000807444EA02030C7943EA04224260CB68A0
:109CF0008A6884681A43084B234013434A7943EA2D
:109D000042038360097CC26A4B1E22F47002D9B2FE
:109D100042EA0152C26210BDFDF7F1FF836811B142
:109D200043F0010101E023F0010181607047836885
:109D300011B143F4807101E023F4807181607047B8
:109D4000836843F00801816070478068C0F3C000F9
:109D50007047836843F00401816070478068C0F3F6
:109D600080007047836811B143F4A00101E023F43F
:109D7000A00181607047092970B54FF003040CD928
:109D80004C4307251E3C05FA04F503FA04F3C668A4
:109D900026EA05052B43C3600BE04C43072505FA73
:109DA00004F503FA04F3066926EA050545EA030407
:109DB0000461062A4FF005030DD8013A53431F22D0
:109DC00002FA03F201FA03F1446B24EA020242EAC6
:109DD0000103436370BD0C2A0DD853431F22233B5C
:109DE00002FA03F201FA03F1046B24EA020242EAE6
:109DF0000103036370BD53431F22413B02FA03F288
:109E000001FA03F1C46A24EA02021143C16270BD7F
:109E100040F0BF60024B40F40031D960704700BF92
:109E200000ED00E0C37810B503B3164CE168CB43F6
:109E3000C3F302244178C4F1040201FA02F10F22B3
:109E400022FA04F28478037822400A43110103F1D4
:109E50006043CAB203F5614181F800230078012212
:109E600000F01F03410902FA03F007E00078012225
:109E700000F01F03410902FA03F02031024B43F8BE
:109E8000210010BD00ED00E000E100E030B5048CE1
:109E900024F001052C04250C0584048BA5B225F0C3
:109EA000F3052A4342EA0313114A048C9042A4B2F8
:109EB0009DB215D002F50063984211D0B0F1804FE9
:109EC0000ED0A3F5983290420AD002F580639842F2
:109ED00006D003F58062904218BF24F00A0401D135
:109EE00024F0020444F0010421430583018430BDC1
:109EF000002C014030B5048C24F010052C04250CF6
:109F00000584048B058C24F440742405240D44EA54
:109F1000022242EA0333144AADB290429BB212D0FD
:109F200002F5006290420ED0B0F1804F0BD0A2F546
:109F30009832904207D002F58062904203D002F539
:109F40008062904207D125F0200242F0100545EAD8
:109F5000011189B204E025F0A00545F01005294360
:109F60000383018430BD00BF002C0140224A0388D6
:109F700090429BB212D002F5006290420ED0B0F136
:109F8000804F0BD0A2F59832904207D002F5806244
:109F9000904203D002F58062904203D14A8823F0B8
:109FA00070031343154A904208D002F58062904234
:109FB00004D023F44073CA889BB2134303808B8878
:109FC0000A8883850C4B028598420FD003F5006206
:109FD00090420BD002F54063984207D003F58062AF
:109FE000904203D002F58063984201D1097A01863C
:109FF00001228282704700BF002C01400010004007
:10A00000038C70B523F001021404250C0584068C22
:10A010008388028B9CB222F073052B040D881A0CE6
:10A0200026F0020633042A434E880D891B0C354363
:10A03000ADB22B43134DA8420FD005F50065A842E1
:10A040000BD005F54065A84207D005F58065A8420C
:10A0500003D005F58065A8420ED123F008064B8990
:10A060008D881E4326F004032B43CE898D8924F46A
:10A0700040743543ADB22C43C98884800283818605
:10A08000038470BD002C0140038C30B523F0100216
:10A090001404250C0584038C8288048B23F0200390
:10A0A00024F4E6452C040D88240C44EA05241D0400
:10A0B0002B0C0D8992B243EA05134D88A4B243EAF2
:10A0C0000513124D9BB2A84203D005F50065A842C6
:10A0D00015D14D8923F080039BB243EA05134FF657
:10A0E000BF751D408B8822F4406245EA0315ABB270
:10A0F0008D8942EA8502CD8942EA850292B2C988F9
:10A10000828004830187038430BD00BF002C01409E
:10A11000038C30B523F480721404250C0584038C61
:10A120008288848B23F4007324F073052C040D883B
:10A13000240C2C431D042B0C0D8992B243EA0523F9
:10A140004D8843EA0523124D9BB2A84203D005F582
:10A150000065A84215D14D8923F400639BB243EA00
:10A1600005234FF6FF351D408B8822F4405245EA07
:10A170000325ABB28D8942EA0512CD8942EA051268
:10A1800092B2C988828084838187038430BD00BFF6
:10A19000002C0140038C30B523F480521404250CAC
:10A1A0000584038C8288858B94B225F4E6421504DD
:10A1B0002A0C0D8823F4005342EA05221D042B0CBF
:10A1C0000D8992B243EA05334D8843EA05330A4DBF
:10A1D0009BB2A84203D005F50065A84205D18D8940
:10A1E00024F4804444EA8514A4B2C988848082831C
:10A1F000A0F84010038430BD002C014000214FF630
:10A20000FF7383800180C1804180017270470388A1
:10A2100019B199B241F0010303E023F001010A04EE
:10A22000130C03807047B0F8443029B16FEA434300
:10A230006FEA53418AB201E059044A0CA0F8442065
:10A24000704783899BB20AB1194301E023EA0101F7
:10A2500081817047038B23F0080213041A0C114309
:10A2600001837047038B23F4006213041A0C42EA43
:10A2700001218BB203837047838B23F00802130400
:10A280001A0C114381837047838B23F400621304FB
:10A290001A0C42EA01218BB283837047038B23F0AF
:10A2A0000C0213041A0C0283038B9AB2114301832C
:10A2B0007047038B23F4406213041A0C0283038B50
:10A2C0009AB242EA01218BB203837047838B23F059
:10A2D0000C0213041A0C8283838B9AB2114381837C
:10A2E0007047838B23F4406213041A0C8283838BA0
:10A2F0009AB242EA01218BB283837047F8B50B888A
:10A300000D4604464988AA8843B92B89FFF7BEFD4C
:10A31000E9882046BDE8F840FFF7C0BF042B08D10C
:10A320002B89FFF7E7FDE9882046BDE8F840FFF7F5
:10A33000C0BF082B0E462F89008C3BD120F48073C0
:10A340001804030C2384A08B83B223F0F30343EAA5
:10A350000717374B208CBFB29C4280B247EA0202FB
:10A3600012D003F500639C420ED0B4F1804F0BD0A5
:10A37000A3F598339C4207D003F580639C4203D039
:10A3800003F580639C4207D120F4007040EA062167
:10A390008BB243F4807305E020F4206041F48071B7
:10A3A00040EA0103E9882046A2832384BDE8F840FF
:10A3B000FFF78CBF20F480531804030C2384A38B75
:10A3C000208C23F440731B051B0D43EA022242EA52
:10A3D0000733174A80B294429BB212D002F5006252
:10A3E00094420ED0B4F1804F0BD0A2F59832944233
:10A3F00007D002F58062944203D002F58062944255
:10A4000007D120F4005040EA063291B241F4805264
:10A4100005E047F6FF52024041F480510A43E988C3
:10A420002046A3832284BDE8F840FFF75ABF00BF4F
:10A43000002C0140808E80B27047008F80B2704740
:10A44000808F80B27047B0F8400080B27047038AB6
:10A45000828911EA030092B203D011420CBF00209E
:10A4600001207047C9438AB202827047038A30B51F
:10A470000D460446EA8898B220F4405111432182E7
:10A48000A3892889A98823F4B05340EA0102688986
:10A4900023F00C0102430804030C1A4391B2A1817A
:10A4A000A08AAA8983B223F4407187B01143A182A4
:10A4B00001A800F0EBF81848A38984420CBF049867
:10A4C000039819B200294FF019032A6803FB00F022
:10A4D00001DA510000E09100B0FBF1F16423B1FB1F
:10A4E000F3F21201100903FB1011A08900B2002839
:10A4F00006DAC9003231B1FBF3F303F0070005E0DF
:10A5000009013231B1FBF3F303F00F00024390B2C3
:10A51000208107B030BD00BF00380140838919B1E8
:10A5200099B241F4005303E023F400510A04130CE0
:10A5300083817047C1F3421310B5012401F01F015C
:10A54000A34204FA01F101D10C3004E0022B01D145
:10A55000103000E01430036812B143EA010201E058
:10A5600023EA0102026010BD838A9BB20AB119433B
:10A5700001E023EA0101818270470000034A044B95
:10A5800002F188305A605860704700BF2301674568
:10A5900000200240024B1A6942F0800018617047A7
:10A5A00000200240014BD860704700BF00200240ED
:10A5B000084BDA68D20709D4D868400708D4D968AC
:10A5C00011F0100F0CBF04200320704701207047CA
:10A5D000022070470020024010B50446FFF7E8FF54
:10A5E000012806D11CB1FFF7E3FF013CF8E7052085
:10A5F00010BD002C08BF052010BD000073B500235E
:10A6000006464FF400500D460193FFF7E5FF04287E
:10A610001AD10E4CAAB2206940F0010121614FF419
:10A6200000503280FFF7D8FF042808D10236019687
:10A63000019B2D0C1D804FF40050FFF7CDFF2169C9
:10A6400041F6FE720A4022617CBD00BF002002403C
:10A6500038B505464FF43020FFF7BEFF042812D16D
:10A66000094C236943F002002061656121694FF4C0
:10A67000302041F040022261FFF7AEFF216941F630
:10A68000FD730B40236138BD00200240204B10B504
:10A690005A6802F00C01042903D0082905D01D4B8B
:10A6A00001E01D4C2368036011E05C685968C4F345
:10A6B0008342941CC90301D4184A06E016495B681A
:10A6C0000A6813F4003F18BF520854430460104B4B
:10A6D0005968C1F3031212498C5C026822FA04F231
:10A6E00042605C68C4F302240C5D22FA04F48460C6
:10A6F0005C68C4F3C224095D22FA01F2C2605B689F
:10A700000849C3F38133CB5CB2FBF3F2026110BDA5
:10A710000010024000127A008401002000093D0070
:10A72000900100208C010020044B5A6909B11043AC
:10A7300001E022EA00005861704700BF00100240AB
:10A74000044B9A6909B1104301E022EA00009861C4
:10A75000704700BF00100240044BDA6909B1104392
:10A7600001E022EA0000D861704700BF00100240FB
:10A77000044BDA6809B1104301E022EA0000D86016
:10A78000704700BF00100240044B1A6909B1104322
:10A7900001E022EA00001861704700BF001002408B
:10A7A000024B5A6A42F080705862704700100240B3
:10A7B00008B50B4B984207D14FF400100121FFF769
:10A7C000E3FF4FF4001006E04FF480000121FFF793
:10A7D000DBFF4FF480000021BDE80840FFF7D4BF45
:10A7E00000540040F0B58688044687B026F03F004C
:10A7F0000D46010401A80E0CFFF748FF2C4A0399EF
:10A80000B1FBF2F087B23E43A680238823F0010219
:10A8100013041A0C22802B68264A93420AD85B0044
:10A82000B1FBF3F0013783B2BFB22784032B98BF8B
:10A83000042320E0EE884BF6FF72964204D10322F7
:10A840005343B1FBF3F305E019225343B1FBF3F19A
:10A8500041F4804399B20A054FF4967208BF41F063
:10A860000101504341F400434FF47A7190FBF1F041
:10A87000421C91B22184A383228891B241F001034A
:10A880002380208820F4816222F002010B04AA8830
:10A890006989180C41EA02032989AA89184380B200
:10A8A00041EA0203208098B2208107B0F0BD00BFCA
:10A8B00040420F00A086010041F28833002103606E
:10A8C0004BF6FF724FF480438180C2800181418149
:10A8D00083817047038819B199B241F0010303E005
:10A8E00023F001010A04130C03807047038819B197
:10A8F00099B241F4807303E023F480710A04130CCD
:10A9000003807047038819B199B241F4007303E0E2
:10A9100023F400710A04130C03807047038819B1F3
:10A9200099B241F4806303E023F480610A04130CBC
:10A930000380704783889BB20AB1194301E023EA80
:10A9400001018180704701827047008AC0B2704760
:10A9500012B141F0010101E001F0FE0101827047F6
:10A9600002684FF6FE73134003602D4B002198429E
:10A97000016041608160C16022D02A49884229D0AB
:10A98000294B984230D02949884237D0284B9842E9
:10A990003ED0284B984206D153F8681C41F4700011
:10A9A00043F8680C70472449884206D151F87C0C62
:10A9B00040F0706241F87C2C7047204B984206D1E1
:10A9C00053F8042C42F00F0143F8041C70471C4953
:10A9D000884206D151F8183C43F0F00041F8180CB9
:10A9E0007047184B984206D153F82C2C42F47061F2
:10A9F00043F82C1C70471449884206D151F8403C5A
:10AA000043F4704041F8400C7047104B984205D118
:10AA100053F8542C42F4702143F8541C704700BF83
:10AA2000080002401C000240300002404400024086
:10AA3000580002406C0002408000024008040240BE
:10AA40001C04024030040240440402405804024006
:10AA500070B506688C680D6A26F4FF4222F0700615
:10AA60000A6945EA04034C6913438A692343CC69A4
:10AA700013431C434B6A44EA03028B6A1A43324372
:10AA80000260CB680A68496843608260C16070BD3B
:10AA90000023036043608360C3600361436183619B
:10AAA000C361036243628362704719B1016841F078
:10AAB000010303E002684FF6FE7313400360704722
:10AAC00003680AB1194301E023EA010101607047FC
:10AAD00041607047406880B270470000C3004CBFBF
:10AAE000014B024B586070470004024000000240D6
:10AAF00000B540F6D87320F00042C3F649739A427D
:10AB000083B0014615DDB2F1FF4F03DBF5F748FFD7
:10AB100003B000BD694600F095FB00F00302012A76
:10AB2000009801990ED0022A07D082B900F0A0FD4A
:10AB3000EEE7002100F09CFDEAE700F099FD00F14E
:10AB40000040E5E701F040FC00F10040E0E70122B1
:10AB500001F03AFCDCE700BF30B5C0F3C754A4F104
:10AB60007F031E2B83B0014621DC581C1DDBCD0F5B
:10AB7000162B0CDD21F07F4323F4000040F400008D
:10AB8000963C00FA04F005B1404203B030BD1148D4
:10AB900050F825402046F5F705FF01902146019821
:10ABA000F5F7FEFE20F0004121B90020EDE7F6F7B1
:10ABB000C7F9EAE720F07F4222F40003C0F3C75050
:10ABC00043F40001C0F1960221FA02F0002DDCD01E
:10ABD000DAE700BF08FD000800B540F6D87320F0A2
:10ABE0000042C3F649739A4283B0014616DDB2F1C2
:10ABF000FF4F03DBF5F7D4FE03B000BD694600F05C
:10AC000021FB00F00300012815D002280BD0B8B9B1
:10AC100000980199012201F0D7FBEDE70021002205
:10AC200001F0D2FBE8E700980199012201F0CCFB8A
:10AC300000F10040E0E70098019900F019FDDBE722
:10AC40000098019900F014FD00F10040D4E700BF26
:10AC500070B58AB0064600F09BF8224C054694F980
:10AC60000030013303D0304601F0B0FD10B9284662
:10AC70000AB070BD304601F05BFD4FF07E51F6F733
:10AC800055F90028F3D0184A0121002530460192D9
:10AC900000910895F5F7CAFB02460B461348CDE92B
:10ACA0000423CDE9022301F011FC94F90030CDE931
:10ACB0000601022B0BD0684601F006FC38B108985B
:10ACC00050B9DDE90601F5F717FE0546CFE701F0BB
:10ACD00089FE21210160F2E701F084FE089A0260FA
:10ACE000EFE700BFA001002010FD000818FD0008DC
:10ACF00000F002BA70B58AB0054600F04FFC224C55
:10AD0000064694F90030013308D0284601F05EFD74
:10AD100020B128460021F6F7EBF810B930460AB00A
:10AD200070BD1A4A0121284600260091019208961A
:10AD3000F5F77CFB2478CDE90401CDE902017CB96B
:10AD400000220023CDE90623684601F0BDFB88B14F
:10AD50000898A0B9DDE90601F5F7CEFD0646DDE766
:10AD60000020002102460B46F5F7DEFC022CCDE95F
:10AD70000601E9D101F036FE21230360E8E701F086
:10AD800031FE08990160E5E7A00100201CFD0008E4
:10AD9000F8B520F00043B3F17E5F044613D00BDC1E
:10ADA000B3F17C5F14DAB3F10C5F00F3A48040F6DA
:10ADB000DB70C3F6C970F8BD0146F5F7F1FD014639
:10ADC000F5F7ACFFF8BD002840F30E810020F8BD78
:10ADD0000028C0F20E8101464FF07E50F5F7E0FDED
:10ADE0004FF07C51F5F7E6FE044600F0D7FB4EF637
:10ADF0000871064620F47F65C3F611012046F5F779
:10AE0000D9FE47F60471C3F64F21F5F7CBFD214675
:10AE1000F5F7D0FE41F24611C3F62451F5F7C0FD17
:10AE20002146F5F7C7FE40F6A821C3F64E61F5F7B7
:10AE3000B9FD2146F5F7BEFE4BF29001C3F6A661BF
:10AE4000F5F7AEFD2146F5F7B5FE4AF6AB21C3F6A0
:10AE50002A61F5F7A7FD2146F5F7ACFE4CF22E610D
:10AE60000746C3F69D512046F5F7A4FE43F2613133
:10AE7000C3F63071F5F794FD2146F5F79BFE45F2D8
:10AE80002D71C4F20101F5F78DFD2146F5F792FE13
:10AE90004DF23911C4F21901F5F782FD2146F5F79B
:10AEA00089FE4FF07E51F5F77DFD01463846F5F7F6
:10AEB00035FF3146F5F77EFE25F00F05074629469A
:10AEC0002846F5F777FE01462046F5F769FD294645
:10AED00004463046F5F766FD01462046F5F71EFFAD
:10AEE00001463846F5F75EFD2946F5F75BFD01465C
:10AEF000F5F758FDF8BD0146F5F75CFE4EF6087112
:10AF0000C3F611010546F5F755FE47F60471C3F681
:10AF10004F21F5F747FD2946F5F74CFE41F2461162
:10AF2000C3F62451F5F73CFD2946F5F743FE40F6FC
:10AF3000A821C3F64E61F5F735FD2946F5F73AFE2F
:10AF40004BF29001C3F6A661F5F72AFD2946F5F705
:10AF500031FE4AF6AB21C3F62A61F5F723FD2946F7
:10AF6000F5F728FE4CF22E610646C3F69D512846A1
:10AF7000F5F720FE43F26131C3F63071F5F710FDAD
:10AF80002946F5F717FE45F22D71C4F20101F5F7D8
:10AF900009FD2946F5F70EFE4DF23911C4F21901EB
:10AFA000F5F7FEFC2946F5F705FE4FF07E51F5F763
:10AFB000F9FC01463046F5F7B1FE01462046F5F7AB
:10AFC000F9FD014642F26810C3F2A230F5F7E8FC41
:10AFD00001462046F5F7E4FC014640F6DA70C3F678
:10AFE000C970F5F7DDFCF8BD40F6DB70C4F249002E
:10AFF000F8BD4FF07E51F5F7D5FC4FF07C51F5F7D9
:10B00000D9FD4EF60871C3F611010446F5F7D2FDDD
:10B0100047F60471C3F64F21F5F7C4FC2146F5F756
:10B02000C9FD41F24611C3F62451F5F7B9FC21469A
:10B03000F5F7C0FD40F6A821C3F64E61F5F7B2FC66
:10B040002146F5F7B7FD4BF29001C3F6A661F5F77F
:10B05000A7FC2146F5F7AEFD4AF6AB21C3F62A61FF
:10B06000F5F7A0FC2146F5F7A5FD0646204600F0C1
:10B0700095FA4CF22E610546C3F69D512046F5F730
:10B0800099FD43F26131C3F63071F5F789FC214631
:10B09000F5F790FD45F22D71C4F20101F5F782FC40
:10B0A0002146F5F787FD4DF23911C4F21901F5F784
:10B0B00077FC2146F5F77EFD4FF07E51F5F772FCE7
:10B0C00001463046F5F72AFE2946F5F773FD42F2B0
:10B0D0006811C3F2A231F5F763FC01462846F5F783
:10B0E00061FC0146F5F75EFC014640F6DA70C4F2F9
:10B0F0004900F5F755FCF8BDF8B521F00044B4F16E
:10B10000FF4F034617DC20F00045B5F1FF4F064620
:10B1100011DCB1F17E5F42D08F1707F0020040EAE8
:10B12000D37775B9022F35D0032F08D140F6DB73E2
:10B13000CCF2490303E01846F5F734FC0346184601
:10B14000F8BDD4B1B4F1FF4F2DD0B5F1FF4F14D0FD
:10B150002C1BE4153C2C18DC002952DB1846F5F7B3
:10B16000DDFD01F0E5FA01F0B7F9012F46D0022F1D
:10B1700035D0002F25D10346E1E7002E40F6DB73E2
:10B180001CDBC3F6C9731846F8BD40F6DB70C3F686
:10B19000C970EAE740F6DB73C4F24903CFE7BDE8C4
:10B1A000F84001F099B9B5F1FF4F2FD0022FF1D03F
:10B1B000032FBBD0012F34D00023C0E7CBF6C973D7
:10B1C000BDE74BF62E51C3F2BB31F5F7EBFB40F672
:10B1D000DB71C4F24901F5F7E3FB0346AFE74BF639
:10B1E0002E51C3F2BB31F5F7DDFB014640F6DB70B3
:10B1F000C4F24900F5F7D4FB0346A0E700F1004391
:10B200009DE714F13C0FA9DA0020AEE7022F13D01E
:10B21000032F0CD0012F40F6DB7305D0C3F6497322
:10B220008DE74FF000438AE7CBF6497387E74CF68A
:10B23000E433CCF2160382E74CF6E433C4F216038F
:10B240007DE700BF2DE9F04F40F6D87320F00044B1
:10B25000C3F649739C4289B006460D4640F38B8085
:10B260004CF6E331C4F216018C4226DC4FF47861CF
:10B270000028C3F6C97140F32B81F5F791FB4FF419
:10B280007D6224F00F04C3F6C9729442064600F0B2
:10B29000818044F24341C3F23571F5F781FB0146E9
:10B2A00028603046F5F77CFB44F24341C3F2357128
:10B2B000F5F776FB0127686061E04FF47867C4F228
:10B2C0004937BC4240F38180B4F1FF4F5BDA4FEA6B
:10B2D000E459A9F18609A4EBC9542046F5F730FEDC
:10B2E000F5F714FC0246014620460592F5F758FB97
:10B2F0004FF08741F5F75EFC0746F5F721FEF5F7BD
:10B3000005FC0146044638460694F5F749FB4FF024
:10B310008741F5F74FFC00210790F5F7DFFD002886
:10B3200000F0F6800327204600210DF11808013FA8
:10B33000F5F7D4FD40B158F8044D00212046013FF7
:10B34000F5F7CCFD0028F6D1924B02200090019336
:10B3500005A83B4629464A4600F066FA002E0746F5
:10B360000DDA95E80C0002F1004103F1004229607A
:10B370006A60474203E00023286000274B6038469C
:10B3800009B0BDE8F08F0146F5F70AFB00276860B9
:10B390002860F4E74FF48841C3F23571F5F700FBFC
:10B3A0004AF20831C2F685610446F5F7F9FA01461A
:10B3B00028602046F5F7F4FA4AF20831C2F68561B2
:10B3C000F5F7EEFA01276860D9E701F0B1F94FF619
:10B3D0008411C3F622718046F5F7ECFB4FF07C51E7
:10B3E000F5F7E0FAF5F7ACFD0746F5F78FFB4FF4FC
:10B3F0007861C3F6C9718346F5F7DCFB0146404628
:10B40000F5F7CEFA44F243418146C3F2357158460E
:10B41000F5F7D0FB1F2F8246514648461FDC5E4B96
:10B420007A1E53F8223024F0FF029A4217D0F5F723
:10B43000B7FA8046C5F8008041464846F5F7B0FAAD
:10B440005146F5F7ADFA002E686098DA08F1004829
:10B4500000F10041C5F8008069607F428FE7F5F791
:10B460009FFAE3158046C0F3C750191A0829E1DD99
:10B470004FF48841C3F2357158460393F5F79AFBB0
:10B48000824651464846F5F78BFA0446214648461F
:10B49000F5F786FA5146F5F783FA4AF20831814604
:10B4A000C2F685615846F5F785FB4946F5F778FA07
:10B4B000824651462046F5F773FA039BC0F3C75204
:10B4C0008046981A192841DCC5F80080A146B3E7E8
:10B4D000F5F768FA4FF47D6724F00F04C3F6C977D7
:10B4E000BC42064616D044F24341C3F23571F5F72B
:10B4F00059FA014628603046F5F752FA44F24341C2
:10B50000C3F23571F5F74EFA4FF0FF37686036E752
:10B51000032719E74FF48841C3F23571F5F742FA72
:10B520004AF20831C2F685610446F5F73BFA014656
:10B5300028602046F5F734FA4AF20831C2F68561F0
:10B54000F5F730FA4FF0FF37686018E74FF4234102
:10B55000C2F685615846F5F72DFB804641462046E8
:10B56000F5F71EFA814649462046F5F719FA414695
:10B57000F5F716FA43F232110446C2F28D415846ED
:10B58000F5F718FB2146F5F70BFA82465146484677
:10B590004DE700BFA4FD000824FD000820F0004294
:10B5A000B2F1FF4FF8B50446034646D2002A42D016
:10B5B000002852DBC415B2F5000F09D210F40005C3
:10B5C00053D15B0001351902FBD5C5F101002418E8
:10B5D00023F07F417F3C21F40006E20746F400009F
:10B5E00048BF400043004FF08072002760109A422D
:10B5F0003C462CDD5B004FF400021825A6185108CC
:10B600009E4205F1FF3502DCB4189B1BBF185B009E
:10B6100062189A4202DC9B1A54187F185B004A0891
:10B62000013DEBD113B107F001017F187C1004F14B
:10B630007C5303EBC0542046F8BD0146F5F7BAFA37
:10B6400001462046F5F7AEF904462046F8BD4FF016
:10B65000007403F17F431746CCE70146F5F7A0F9E4
:10B660000146F5F75BFB0446E5E70120AFE700BFC5
:10B670002DE9F84320F00046B6F1485F05460F4635
:10B680005BDAF5F75DFC002800F0CA802946284601
:10B69000F5F790FA4DF24E71CAF647510446F5F7A8
:10B6A00089FA47F2F641C3F20F11F5F77BF921460B
:10B6B000F5F780FA4FF27C21C3F29341F5F770F968
:10B6C0002146F5F777FA40F60151C3F2D071F5F74C
:10B6D00069F92146F5F76EFA40F66131C3F6B621F5
:10B6E000F5F75EF92146F5F765FA4AF6AB21C3F6A0
:10B6F0002A51F5F757F92146F5F75CFA80462046BE
:10B700004FF07C51F5F756FA414606462046F5F7CC
:10B7100051FA394604462846F5F74CFA01462046C8
:10B72000F5F73EF901463046F5F73AF901464FF094
:10B730007E50F5F735F9BDE8F8830146F5F73AFA9A
:10B740004DF24E71CAF647510446F5F733FA47F207
:10B75000F641C3F20F11F5F725F92146F5F72AFA5C
:10B760004FF27C21C3F29341F5F71AF92146F5F720
:10B7700021FA40F60151C3F2D071F5F713F92146D1
:10B78000F5F718FA40F66131C3F6B621F5F708F976
:10B790002146F5F70FFA4AF6AB21C3F62A51F5F721
:10B7A00001F92146F5F706FA49F69913C3F69963AC
:10B7B0009E428046A3DD0020C3F64870864227DC07
:10B7C00006F17F464FF07E503146F5F7E9F88146A5
:10B7D00020464FF07C51F5F7EDF93146F5F7E0F8EA
:10B7E000414606462046F5F7E5F93946044628461F
:10B7F000F5F7E0F901462046F5F7D2F80146304664
:10B80000F5F7CEF801464846F5F7CAF8BDE8F883E3
:10B810004FF000090026C3F63879C3F69066D7E7E3
:10B820004FF07E50BDE8F8832DE9F04FDFB00C9368
:10B830000C9D224B689C0A91691ED61E48BF161D9E
:10B84000834653F82400F71027EAE7730890049121
:10B8500004980D93089DDC43DDF834C002EBC4026C
:10B8600041190792C0EB0C0750D47E18699BC7EBB7
:10B8700006090136002F03EB870522AC09F0010A07
:10B88000C0F2FE822868F5F741F90137B74220601F
:10B890004FF004083AD0BAF1000F26D0002FC0F2C2
:10B8A000F18255F80800F5F731F90137B74244F84D
:10B8B000080008F1040818D128E000BFBC00010806
:10B8C00055F80800F5F722F9013708F1040944F8A2
:10B8D000080013D455F80900F5F718F90137B742F5
:10B8E00044F8090009F1040810D0002FE8DA00201C
:10B8F000013708F1040944F80800EBD501370020AE
:10B90000B74244F8090009F10408EED1089A002A68
:10B91000C0F2458508990C9E8D004AAB5C190395D1
:10B9200049AF02944FEA860A049A002AC0F296822E
:10B930000DF1880808EB860555F8041CAAF10403EC
:10B94000DBF80000C3F38009F5F734F90146002065
:10B95000F5F728F80424043D544580462BD0B9F16E
:10B96000000F0DD055F8041DDBF80400F5F722F99F
:10B9700001464046F5F716F80824544580461AD08B
:10B9800055F8041C5BF80400F5F714F9014640462D
:10B99000F5F708F80434804655F8081C5BF80400F5
:10B9A000F5F708F901464046F4F7FCFF0434083D7A
:10B9B00054458046E4D1029847F8048F0136874207
:10B9C000B2D1039F0EA9CE190996089EB2005EABB4
:10B9D0009D18002E029255F8509C7DDD0DF5947C4B
:10B9E0004FF06E5148460DACA7180CEB0205F5F769
:10B9F000E1F8F5F7A5FAF5F789F84FF087410190DE
:10BA0000F5F7D8F801464846F4F7CAFFF5F798FA73
:10BA10000EAC20600198014655F8040DF4F7C2FF02
:10BA2000BC428146C7F3800156D0E9B14FF06E5158
:10BA3000F5F7C0F8F5F784FAF5F768F84FF08741A5
:10BA40000190F5F7B7F801464846F4F7A9FFF5F776
:10BA500077FA019A0FAC2060114655F8040DF4F7FF
:10BA6000A1FFBC42814637D04FF06E514846F5F7F2
:10BA7000A1F8F5F765FAF5F749F84FF087418046E8
:10BA8000F5F798F801464846F4F78AFFF5F758FAB3
:10BA90004146606055F8040DF4F784FF4FF06E5195
:10BAA0008146F5F787F8F5F74BFAF5F72FF84FF0E1
:10BAB00087418046F5F77EF801464846F4F770FF67
:10BAC000F5F73EFA4146A06055F8040DF4F76AFF19
:10BAD0000834BC428146C7D10799484600F0A2FE0F
:10BAE0004FF078510546F5F765F800F025FE4FF068
:10BAF0008241F5F75FF801462846F4F751FF074603
:10BB0000F5F71EFA8146F5F701F801463846F4F7D5
:10BB100047FF07990746002940F33981721E0EAC92
:10BB2000079D54F82230C5F1080043FA00F101FAEC
:10BB300000F0C5F107041B1A43FA04F40DF1380CA8
:10BB400089444CF82230002C55DD002E09F1010902
:10BB500040F39481029D0EABDDF808C053F8042B2E
:10BB6000281F0DF1380E00250EEB0C01C0F38000EC
:10BB700022B1C2F5807243F8042C01258B4226D0F5
:10BB800060B10F9A0433002D40F0F38022B1C2F56A
:10BB9000807543F8045C01258B4218D053F8042BC0
:10BBA000002D40F0EC80C2F5807012B143F8040C17
:10BBB000012553F8042B002D40F0DB80C2F5807086
:10BBC000002AE9D001258B4243F8040CE6D10799FD
:10BBD00000290DDD012900F0E280022908D1701E44
:10BBE0000DF1380E5EF8202002F03F034EF82030B1
:10BBF000022C00F0E08038460021F5F76FF90028AC
:10BC000000F0F3800898751EA84225DC029B0DF118
:10BC1000380E0EEB03010B46DDF824C053F8042D5B
:10BC2000CCEB0100011F6345C1F3800011D030B19E
:10BC300053F8041DDDF824E00A43734509D0099F39
:10BC400053F8040D53F8041D0243BB4242EA0102BB
:10BC5000F6D1002A40F01A81089F0EAD781E55F8E3
:10BC60002020002A40F0108105EB8004012354F8C5
:10BC7000041D01330029FAD0F018771C87420B907D
:10BC800075DCDDF810E00D9D0B9B0C9C0EEB0702A4
:10BC9000DDF808C0699F991B06EB05094AA8A6199B
:10BCA00022AB07EB890900EB0C05571C8A0003EB5C
:10BCB0008601029506920591002659F8040FF4F7C3
:10BCC00025FF059CA051049800285EDB22AD05EB02
:10BCD0008702AAF10403C3F3800452F8041CDBF8C2
:10BCE00000000394141FF4F765FF01460020F4F7E9
:10BCF00059FE4FF00408D04505462DD0039971B187
:10BD000054F8041DDBF80400F4F754FF01462846FC
:10BD1000F4F748FE4FF00808D04505461CD054F80B
:10BD2000041C5BF80800F4F745FF01462846F4F7C9
:10BD300039FE08F10408054654F8081C5BF80800B1
:10BD4000F4F738FF01462846F4F72CFE08F1040802
:10BD5000083CD0450546E2D1DDF808E006980436F7
:10BD60004EF8045F01378642CDF808E0A5D10B9E5E
:10BD70002CE6C2F1FF0243F8042C01250CE7C2F1C6
:10BD8000FF0543F8045C012513E70025E4E75ED1D5
:10BD9000701E0DF1380E5EF820301C12D3E6711EB5
:10BDA0000DF1380C5CF82100022C00F07F024CF8F9
:10BDB00021207FF420AF39464FF07E50F4F7F0FD9C
:10BDC0000746002D3FF417AF07994FF07E5000F063
:10BDD00029FD01463846F4F7E3FD074638460021C1
:10BDE000F5F77CF800287FF40DAF0294079C3846E5
:10BDF0006142CDF8109000F015FD4FF087410546E7
:10BE0000F5F78AF8002800F0D2824FF06E512846EC
:10BE1000F4F7D0FEF5F794F8F4F778FE4FF0874189
:10BE20000746F4F7C7FE01462846F4F7B9FDF5F7D3
:10BE300087F80EA941F826003846F5F781F8079AE9
:10BE4000013608320EAC079244F8260034E04FF079
:10BE50007C51F5F761F858B90024CCE64FF00008A2
:10BE6000029847F8048F013687427FF45DADA8E55C
:10BE70000224002E09F101093FF76CAE0025A6E669
:10BE8000002002E5002010E50123F5E6079A0EAE3A
:10BE900056F82530083ACDF8109002940792002BFE
:10BEA00040F08E8206EB85042E4654F8045D013E78
:10BEB000083A002DF9D007924FF07E50079900F014
:10BEC000B1FC002E0446C0F2AC804FEA860AC6EBF5
:10BED000867B0EAF4FEA8B095744C9F100034AA98C
:10BEE000386801EB0A08C3F3800BF4F70FFE214614
:10BEF000F4F760FE4FF06E51C8F800002046F4F7EA
:10BF000059FEA9F104096FF0030ACA45054631D06C
:10BF1000BBF1000F0BD057F8040CF4F7F7FD2946DE
:10BF2000F4F748FE6FF0070A48F8040C1AE057F8D7
:10BF30000A00F4F7EBFD2946F4F73CFE4FF06E5192
:10BF400048F80A002846F4F735FEAAF1040405462D
:10BF50003859F4F7DBFD2946F4F72CFEAAF1080A5C
:10BF600048F8040028464FF06E51F4F723FECA4506
:10BF70000546DCD1701CDFF84C94DDF820A003905E
:10BF800000270596BAF1000FC0F20582002FC0F21B
:10BF90000282002600241AF0010F354620D0D8F87E
:10BFA0000010D9F80000F4F705FE01462046F4F72A
:10BFB000F9FC0125AA45044626DB0426BD420FDD17
:10BFC00022E0BB4520DC58F8021059F80200F4F7D3
:10BFD000F1FD01462046F4F7E5FCBD42044613DCC2
:10BFE00058F8061059F80600F4F7E4FD014620461B
:10BFF000F4F7D8FC05F1010B06F104020235DA452D
:10C00000044602F10406DCDA5EABDDF80CC003EB9B
:10C0100087010137674541F8A04CA8F10408B1D168
:10C02000059E689C032C16D8DFE814F085011F01DB
:10C030001F011B0000230299002900F00B81379C8F
:10C04000369804F100420A9C00F1004503F10043D8
:10C0500025606260A360049D05F007005FB0BDE845
:10C06000F08F002EE6DD06F1FF3836AF07EB8809CA
:10C070004D4655F804290DF1D40AD5F808B01046FC
:10C0800059460192F4F78EFC804641460198F4F738
:10C0900087FC01465846F4F785FC5545C9F38003F3
:10C0A000A860C5F8048044D0BBB155F80429D5F880
:10C0B00008B0104659460192F4F774FC0199804685
:10C0C00008464146F4F76CFC01465846F4F76AFC12
:10C0D0005545C5F80480A8602BD02C4654F8043987
:10C0E000D4F808B0184659460193F4F75BFC804633
:10C0F00041460198F4F754FC01465846F4F752FCC7
:10C10000C4F80480A06055F804BC251FD5F8088049
:10C1100058464146F4F746FC044621465846F4F793
:10C120003FFC01464046F4F73DFC55456C60A86075
:10C13000D3D1012E7FF77EAF4D4655F804B9C7EB3A
:10C14000090ED5F808A058465146AEF10409F4F797
:10C1500029FC804641465846F4F722FC01465046E9
:10C16000F4F720FCBD42C9F38009C5F80480A8603B
:10C1700043D0B9F1000F15D055F804A9D5F80890AF
:10C1800050464946F4F70EFC804641465046F4F7C7
:10C1900007FC01464846F4F705FCBD42C5F804809B
:10C1A000A8602AD02C4654F804A9D4F80890504628
:10C1B0004946F4F7F7FB804641465046F4F7F0FB5A
:10C1C00001464846F4F7EEFBC4F80480A06055F839
:10C1D000049C251FD5F8088048464146F4F7E2FB49
:10C1E000044621464846F4F7DBFB01464046F4F797
:10C1F000D9FBBD426C60A860D4D1013607EB86073D
:10C2000008353E467A1B131F56F8041D0020C3F361
:10C210008007F4F7C7FBAE4203463FF40CAF3FB1D3
:10C2200056F8041DF4F7BEFBAE4203463FF403AFDD
:10C23000184656F8041C341FF4F7B4FB083E54F8B3
:10C24000041CF4F7AFFBAE42F3D102990346002978
:10C250007FF4F5AEDDF828C036993798CCF8001099
:10C26000CCF80400CCF80830F5E60023002E29DBDA
:10C2700036AF751C07EB85042546E21B55F8041DF7
:10C28000A2F1040E0020CEF38008F4F78BFBBD4230
:10C29000034617D0B8F1000F06D055F8041DF4F787
:10C2A00081FBBD4203460DD0184655F8041C2C1FD7
:10C2B000F4F778FB083D54F8041CF4F773FBBD4217
:10C2C000F3D103460299002967D003F10040DDF85D
:10C2D00028C01946CCF800003698F4F761FB002E10
:10C2E000034621DD36AF07EB8606F51B2A1F37997B
:10C2F000C2F38007F4F756FB37ACB442034613D0C1
:10C3000037B16168F4F74EFB38ACB44203460BD04A
:10C31000184654F8041FF4F745FB54F8041FF4F7CB
:10C3200041FBB442F5D10346029909B103F1004340
:10C330000A9C63608FE6002E40DB36AF013607EBC8
:10C3400086000546C21B55F8041D0020141FF4F793
:10C3500029FBBD42C4F38006034615D036B155F81B
:10C36000041DF4F71FFBBD4203460DD0184655F8D7
:10C37000041C2C1FF4F716FB083D54F8041CF4F7BA
:10C3800011FBBD42F3D10346029909B103F1004309
:10C390000A9C23605FE6002436E6184697E7DDF83E
:10C3A00030E0900003904FEA8E0AFFF70ABB284660
:10C3B000F4F7C6FD0EAB43F826007DE50023E3E766
:10C3C0002E4679E5C80001082DE9F84320F0004326
:10C3D000B3F1485F04460F46904603DAF4F7B0FD28
:10C3E000002859D021462046F4F7E4FB21460546B3
:10C3F000F4F7E0FB4CF6D311C2F62E710646284640
:10C40000F4F7D8FB42F63471C3F2D721F4F7C8FA37
:10C410002946F4F7CFFB4EF61B71C3F23861F4F7EF
:10C42000C1FA2946F4F7C6FB40F60151C3F6501194
:10C43000F4F7B6FA2946F4F7BDFB48F68901C3F6CE
:10C440000841F4F7AFFA8146B8F1000F27D04FF05A
:10C450007C513846F4F7AEFB494680463046F4F747
:10C46000A9FB01464046F4F79BFA2946F4F7A2FBE4
:10C470003946F4F795FA4AF6AB210546C3F62A6128
:10C480003046F4F797FB01462846F4F78BFA01464D
:10C490002046F4F785FA04462046BDE8F8830146B5
:10C4A0002846F4F787FB4AF6AB21C3F62A61F4F776
:10C4B00077FA3146F4F77EFB01462046F4F772FA2C
:10C4C00004462046BDE8F883002070470021002084
:10C4D000C7F6F871704700BF2DE9F04120F0004524
:10C4E000B5F1A14F044606460DDBB5F1FF4F00F351
:10C4F0009C80002840F6DB7440F3D480C3F6C974F6
:10C500002046BDE8F0814FF6FF73C3F6DF639D421E
:10C5100000F3A280B5F1445FC0F28E804FF0FF3788
:10C5200021462046F4F746FB01468046F4F742FBDD
:10C5300046F6D711C3F685410546F4F73BFB4DF6A9
:10C540005921C3F64B51F4F72DFA2946F4F732FB83
:10C5500046F63531C3F68851F4F724FA2946F4F744
:10C5600029FB42F66E61C3F6BA51F4F71BFA29466D
:10C57000F4F720FB44F62511C3F61261F4F712FA22
:10C580002946F4F717FB4AF6AB21C3F6AA61F4F784
:10C5900009FA4146F4F70EFB4AF221218046CBF618
:10C5A00015512846F4F706FB4FF26B11C3F66E5196
:10C5B000F4F7F6F92946F4F7FDFA48F29571C3F657
:10C5C0009D51F4F7EDF92946F4F7F4FA48F638618D
:10C5D000C3F6E351F4F7E4F92946F4F7EBFA4CF625
:10C5E000CD41C3F64C61F4F7DBF92946F4F7E2FAE2
:10C5F0007B1C0146404658D0F4F7D4F92146F4F7A5
:10C60000D9FA494B53F82710F4F7CAF92146F4F741
:10C61000C7F90146454850F82700F4F7C1F9002E44
:10C620003DDB04462046BDE8F0810146F4F7BAF947
:10C6300004462046BDE8F0814FF2CA21C7F24911F5
:10C64000F4F7B0F94FF07E51F4F770FC00283FF496
:10C6500065AF2046BDE8F08100F06AF84FF6FF7143
:10C66000C3F697718D4204464FF6FF7228DCC3F67D
:10C670002F72954246DC0146F4F794F94FF07E5153
:10C68000F4F78EF94FF0804105462046F4F78AF919
:10C6900001462846F4F742FB0027044640E700F134
:10C6A00000442DE7CBF6C9742AE7F4F77BF921465D
:10C6B000F4F780FA01462046F4F772F904461FE7C2
:10C6C000C4F21B02954214DC4FF07F51F4F768F975
:10C6D0004FF07F5105462046F4F76CFA4FF07E513B
:10C6E000F4F760F901462846F4F718FB02270446E0
:10C6F00016E700202146CBF68070F4F70FFB0327E6
:10C7000004460DE74FF07E51F4F74AF94FF07E51A1
:10C7100007462046F4F746F901463846F4F7FEFA94
:10C7200001270446FCE600BFF400010804010108EB
:10C7300020F00040704700BFF8B520F00046F50D2E
:10C740007F3D162D014604461BDC002D074620DBED
:10C750004FF6FF73C0F27F0343FA05F606420ED090
:10C760004FF2CA21C7F24911F4F71CF90021F4F77E
:10C77000DDFB18B1002C1BDB27EA06042146084626
:10C78000F8BDB6F1FF4FFAD3F4F70CF901460846AD
:10C79000F8BD4FF2CA21C7F24911F4F703F900219D
:10C7A000F4F7C4FB0028E9D0002C07DB0024E5E700
:10C7B0004FF4000040FA05F56719DDE70021CBF6DC
:10C7C0008071002E18BF0C46D8E700BF08B90220C0
:10C7D0007047B0F1004FFAD0A0F500026FF00143AE
:10C7E0009A4201D80420704700F1FF419942F9D9DB
:10C7F0004FF6FE73421EC0F27F039A4201D8032017
:10C80000704700F100414A1E9A42F8D9B0F1FF4F3B
:10C8100005D010F5000F14BF002001207047012043
:10C82000704700BF38B530F00044034602460D465D
:10C830000FD0B4F1FF4F0ED2B4F5000F11D3E40DB9
:10C840006419FE2C33DC002C1BDD22F0FF4141EA91
:10C85000C453184638BD0146F4F7A4F803461846F9
:10C8600038BD4FF09841F4F7A5F943F6B041CFF643
:10C87000FF718D42034612DBC0F3C7540246193CD8
:10C88000DEE714F1160F21DA4CF2503295421946C8
:10C890000EDC44F26020C0F6A25000F023F844F20F
:10C8A0006021C0F6A251F4F785F90346D1E7194695
:10C8B0004FF2CA20C7F2491000F014F84FF2CA2113
:10C8C000C7F24911F4F776F90346C2E722F0FF43B5
:10C8D00004F1190043EAC0504FF04C51F4F76AF9E3
:10C8E0000346B6E701F0004120F0004008437047DE
:10C8F0002DE9F041274C84B025680746D5F848411A
:10C90000002C41D066681F2E1CDD234810B94FF063
:10C91000FF301FE04FF4C870039102920193AFF310
:10C92000008003990446029A019B0028EFD0D5F8B5
:10C930004861002060602660C5F84841C4F888015D
:10C94000C4F88C01656847B9A81C013544F820106B
:10C950006560002004B0BDE8F081012000FA05F018
:10C96000D4F8886104EB85080643022FC8F88820B4
:10C97000C4F88861C8F80831E6D1D4F88C3143EAAC
:10C980000002C4F88C21DFE705F5A674C5F848411C
:10C99000B8E700BF1C0201080000000000210A22C5
:10C9A00001F028B82DE9F84FDDF828B081468A4615
:10C9B00098469AB193B11646002503E00FD0651C46
:10C9C000AE420BD97419640808FB04A748463946DF
:10C9D000D8470028F2DA2646AE42F3D80027384678
:10C9E000BDE8F88F40F2D053C2F2000318687047D8
:10C9F000114B124A70B5981A831018D0591E02EBC9
:10CA000083040D4654F8042D01F00106904775B1DA
:10CA100026B154F8040D8047013D08D054F8043D78
:10CA20009847013D54F8041D8847013DF6D1BDE803
:10CA3000704003F0FBBB00BF440201084002010844
:10CA4000F8B5204F204C381B871017D07A1E23686A
:10CA5000012502F001069847AF420FD02EB154F8DD
:10CA6000041F02258847AF4208D06068804702351E
:10CA7000A268261D90470834AF42F6D1134F144CDC
:10CA800003F0CEFB3B1B9F1018D07D1E216805F0E4
:10CA9000010601258847AF4211D02EB154F8040F8A
:10CAA00002258047AF420BD0626890470235A368E9
:10CAB000261D98470834AF42F6D1F8BDF8BDF8BD41
:10CAC000F8BD00BF38020108380201084002010821
:10CAD000380201080F2A2DE9F00340F2A18041EA53
:10CAE00000039B0740F09E800C68A2F110050460D3
:10CAF0004B68AC4643608C68BCF10F0F8460CC6817
:10CB0000C5F30015C46000F1100301F110042BD926
:10CB100075B12568ACF1100C1D6065685D60A56895
:10CB20009D60E5681034DD601033BCF10F0F1BD938
:10CB3000276804F110061F60676803F110055F6045
:10CB4000A768ACF1200C9F60E768DF6024691C6176
:10CB5000776806F110046F60B7682033AF60F6683D
:10CB6000BCF10F0FEE60E3D8A2F1100828F00F031C
:10CB700002F00F0403F1100C032C00EB0C0301EB8B
:10CB80000C0851D9211F4FEA9109444608EB890C42
:10CB900054F8046BC8EB0C010CF1040C1D46644501
:10CBA00045F8046BC1F3800112D029B154F8041B7D
:10CBB000644545F8041B0BD0274657F8041B2E4646
:10CBC00046F8041B64686C603C1D351D6445F3D158
:10CBD00009F1010C4FEA8C0902F0030208EB09018C
:10CBE0004B44D2B10D789A18DC4303F8015B141959
:10CBF000934204F0010410D02CB111F8014F03F856
:10CC0000014B934209D04D781C4604F8015B8D78A6
:10CC100002315D70631C9342F5D1BDE8F0037047AB
:10CC20000346DEE70346DDE741462246D9E700BF7B
:10CC3000F0B48407034600F08D80541E002A00F0F3
:10CC40008780E507CEB211D41A4602F8016B13466D
:10CC50001546920710D0621E002C79D003F8016BA4
:10CC600014469A071D4607D0013CEDE7034603F83A
:10CC7000016B9A071D46F7D1032C52D9CEB246EA72
:10CC800006270F2C47EA07432DD9A4F110021746B7
:10CC90000F2FC2F300162B606B60AB60EB6005F1E9
:10CCA000100216D93EB1103F136053609360D360F9
:10CCB00010320F2F0DD9203F02F110061360536080
:10CCC0009360D360136153619361D36120320F2F5E
:10CCD000F1D8A4F1100222F00F0204F00F04103278
:10CCE000032C15441DD9271F3E462A46032E42F821
:10CCF000043BC7F380070DD927B1043E032E42F849
:10CD0000043B07D9174647F8043B083E53603A1DD9
:10CD1000032EF7D8231F23F00302131D04F003048E
:10CD2000ED18ACB1C9B2EA432C1905F8011BA318E0
:10CD3000A54203F001020BD01AB105F8011BA54270
:10CD400006D02B4603F8011B69705D1CA542F8D183
:10CD5000F0BC7047054614468EE700BF830770B5E8
:10CD6000064614D10368A3F1013222EA030010F051
:10CD7000803F0CD1331D1A4653F8044BA4F1013502
:10CD800025EA040414F0803FF5D0104600E0304658
:10CD900003782BB1421C147810460132002CFAD1D2
:10CDA00000F080F8304670BDC9B2F0B400294BD015
:10CDB00082070FD00278002A71D0914242D0431CE2
:10CDC00005E013F8012B002A3BD091423AD09A0794
:10CDD0001846F6D1036841EA0127A3F1013222EA9D
:10CDE000030212F0803F47EA07471CD17B40A3F1C2
:10CDF000013222EA030313F0803F14D1021D02E046
:10CE000014F0803F0FD1104652F8043BA3F10136D5
:10CE100087EA030426EA0303A4F1013513F0803FF7
:10CE200025EA0404ECD00278002A38D0914209D0D7
:10CE3000431C01E0914205D0184613F8012B002A4B
:10CE4000F8D11046F0BC704783070BD00278002A57
:10CE5000F8D0431C03E0017801330029F2D0990790
:10CE60001846F8D10168A1F1013323EA010212F05A
:10CE7000803F0AD1031D184653F8041BA1F1013469
:10CE800024EA010212F0803FF5D00378002BD9D0BC
:10CE9000421C1178104601320029FAD1D2E710461F
:10CEA000D0E700BF80EA0102844612F0030F4FD1A1
:10CEB00011F0030F32D14DF8044D11F0040F51F869
:10CEC000043B0BD0A3F101329A4312F0803F04BF20
:10CED0004CF8043B51F8043B16D100BF51F8044B09
:10CEE000A3F101329A4312F0803FA4F101320BD139
:10CEF0004CF8043BA24312F0803F04BF51F8043BBE
:10CF00004CF8044BEAD023460CF8013B13F0FF0F1A
:10CF10004FEA3323F8D15DF8044B704711F0010F4D
:10CF200006D011F8012B0CF8012B002A08BF70471E
:10CF300011F0020FBFD031F8022B12F0FF0F16BF15
:10CF40002CF8022B8CF8002012F47F4FB3D17047DD
:10CF500011F8012B0CF8012B002AF9D1704700BF02
:10CF600020F0030110F00300C0F1000051F8043B71
:10CF700000F1040C4FEACC0C6FF000021CBF22FA47
:10CF80000CF213434FF0010C4CEA0C2C4CEA0C4C05
:10CF9000A3EB0C0222EA030212EACC1204BF51F8FE
:10CFA000043B0430F4D013F0FF0F1FBF013013F423
:10CFB0007F4F013013F47F0F18BF0130704700BF5F
:10CFC000F0B4002A63D0344B04461B6814F8010BFC
:10CFD000571E1D186E7807F0010706F00305012D96
:10CFE00058D011F8015B5E19767806F00306012E21
:10CFF00008BF2035401B4BD1002D49D0013A47D006
:10D000002FB314F8010B1D186E7806F00305012DDF
:10D0100011F8015B08BF20305E19767806F0030630
:10D02000012E08BF2035401B32D18DB3013A0ED1FD
:10D030002EE011F8012B9E18767806F00306012EDB
:10D0400008BF2032801A23D112B36A1E20D014F8F0
:10D05000010B1D186E7806F00305012D11F8015B18
:10D0600008BF20305E19767806F00306012E08BF4F
:10D070002035401B0CD15DB114F8010B551E1A1858
:10D08000567806F00302012AD3D12030D1E71046AA
:10D09000F0BC70472030A4E7A401002041EA00035F
:10D0A0009B07F0B474D1032A72D90C4654F8045B80
:10D0B000161FA5F1013727EA050717F0803F034641
:10D0C000C6F3800C31D10346032E324643F8045B8D
:10D0D0002AD9BCF1000F0AD0214654F8045BA5F10F
:10D0E000013626EA050616F0803F18D01DE02646D8
:10D0F00056F8045B2146A5F1013727EA050717F02A
:10D10000803F12D143F8045B65683146A5F10136D2
:10D1100026EA0506043A0C1D16F0803F05D1043AB4
:10D12000032A43F8045BE2D821467AB30D78013A2A
:10D1300003F8015B9DB112F0010F1C462AD1234672
:10D1400022B311F8015F013A03F8015B3DB111F818
:10D15000015F013A65705C1C2346002DEFD1AAB136
:10D1600000219C18DA4303F8011BA218A34202F025
:10D1700001020BD01AB103F8011BA34206D01A46D4
:10D1800002F8011B5970531CA342F8D1F0BC704740
:10D190000346CAE711F8015F1C4604F8015B013A37
:10D1A0002346002DCBD1DAE72DE9F00701273C46D5
:10D1B00000254FF0FF3663198B4200EB060C0DD2B1
:10D1C0001CF804A010F80380D0452ED201241D467F
:10D1D0009F1B63198B4200EB060CF1D34FF0010A41
:10D1E0001760544600254FF0FF3C6319994200EB4D
:10D1F0000C080ED918F8048010F80390C1451AD90C
:10D2000001241D46CCEB030A6319994200EB0C087C
:10D21000F0D80CF101000136B0423CBFBA463046AE
:10D22000C2F800A0BDE8F00770470BD001272E46DA
:10D230003C46ED19BFE709D04FF0010AAC46544611
:10D240005544D2E7BC4205D00134B4E7544505D07B
:10D250000134CAE727461D460124ACE7A2461D4615
:10D260000124C2E72DE9F04FADF2244D15460646E4
:10D2700089461046194607AA1C46FFF795FF07ABDB
:10D2800082460DF21C411A1D5C6008338B425460CB
:10D29000F9D114B301232F78611E08A8A34240F8E6
:10D2A000271001EA030218D032B16A7802234F1E18
:10D2B000A34240F8227010D0B046A4465C1C15F87A
:10D2C00003E0CE1A2A5D02330F1B634540F82E603F
:10D2D00040F82270F2D146466446079928466918FC
:10D2E000524600F045FC002840F0B6800AF1FF3EAF
:10D2F00005EB0E0CCDF808E0CAF1010E834604F1EF
:10D30000FF38CDF80CC0CDF814E00746CDF810A0DA
:10D310004A460095019408E027B1079FBB4201D21D
:10D320000199CB1B9B4400272246019CB0185C440A
:10D330000021A21A00F07CFB002840F08780002C1E
:10D3400000F08480301910F8013C08A951F823300E
:10D35000002BE1D1049B9F4228BF3B46434527D287
:10D36000DDF8009006EB0B0119F80350CA5C09EBDD
:10D370000300954266D1DD43454415F0010F024696
:10D3800013D00133434513D24078CD5C013285423E
:10D390000BD057E012F8010FCD5C854252D101331A
:10D3A00012F8010FCD5C85424CD101334345F1D3D6
:10D3B000DDF81090029B4F4528BF4B4639D2DDF86F
:10D3C00008C0DDF8009006EB0B0519F80C1015F8F5
:10D3D0000C00814240F0C080DDF80CE009EB070A48
:10D3E000CAEB0E01C80772461ED5DDF8089009F198
:10D3F000FF31DDF80C90685C19F801CC09F1FF32BF
:10D40000844516D10B460FE012F8019C15F800E098
:10D410004A1EF1450DD10346013815F800C011F838
:10D42000011C614505D10346581E524502F1FF31EA
:10D43000EAD101379F4200F29180079F019ABB44D5
:10D44000D71B71E7DDF814E0F3446BE7002009B067
:10D450000DF5806DBDE8F08FCAEB0400504538BF74
:10D460005046CAF10102431C0AF1FF3C05EB0A07D2
:10D4700004F1FF3B019200944A460793B1464FF0F6
:10D48000000864463E46009909EB020008EB0107DC
:10D49000BA1A002100F0CCFA0028D7D1002FD5D03D
:10D4A00009EB070010F8013C08AA52F823000028F5
:10D4B0004AD1DA4509EB08002AD210F80A3031784F
:10D4C000994218BF534642D16FEA0A0303EB0B019E
:10D4D000C9073246534618D50AF101035B4517D2F6
:10D4E000324612F8011F10F803E08E450DD02EE0F1
:10D4F00012F8011F10F803C08C4528D1013312F82F
:10D50000011F10F803E08E4521D101335B45EFD3B5
:10D51000621C23469BD0295D025D914213D1E10735
:10D5200009D5631EE95CC25C914204D00BE0E95C62
:10D53000C25C914207D15A1E002B88D0A95C825C44
:10D54000023B9142F3D0079880443A469BE7DDF8CE
:10D5500004C0E0449844F8E7049B6AE706EB0B003C
:10D5600075E700BF2DE9F04F037889B080460D467E
:10D57000002B00F065810A789AB1844601310126BA
:10D5800002E011F8012B5AB1934214BF002606F0B5
:10D5900001061CF8013F0C46002BF2D1207820B97F
:10D5A00036B1404609B0BDE8F08F4FF00008F8E70B
:10D5B00008F101002978FFF7F7FB641B06460028F5
:10D5C000F3D0012C00F0B580A044404594BFC0EBDF
:10D5D000080701271F2C06D939462A462346FFF79C
:10D5E00041FE8046DDE7214607AA2846FFF7DCFD1D
:10D5F0000799039069182846039A00F0B9FA0028A1
:10D6000040F09980DDF80CC0DDF80C900CF1FF3E85
:10D6100005EB0E01C9F1010C8346CDF808E0804608
:10D620000491CDF814C03A46B146019508EB0406C2
:10D6300009EB02000021B21A00F0FAF90028B4D177
:10D64000002EB2D0039B9B4528BF5B469C4227D946
:10D65000019D09EB030010F80820E95CE8189142ED
:10D660005FD1DD432D1915F0010F024609EB0801CA
:10D6700013D001339C4213D94078CD5C01328542EE
:10D680000BD04EE012F8010FCD5C854249D1013339
:10D6900012F8010FCD5C854243D101339C42F1D891
:10D6A000DDF80CE0029ADE4540F2CD80019B09EBEB
:10D6B0000805995CA85C814240F0C580DDF804A0B3
:10D6C000049BDA44CAEB0301C8071AD5029FDDF8B0
:10D6D00010C0791E685C1CF8017C0CF1FF33874296
:10D6E00014D10A460DE013F801EC2F5C4B1EBE4529
:10D6F0000CD1024601382F5C11F8011CB94205D14A
:10D700000246501E534503F1FF31ECD10BF1010BE2
:10D71000934500F29A80079A9044C2EB040B32467C
:10D7200084E7059D05EB080B0BEB03084FF0000B9E
:10D73000F5E7804635E7DDF80CA00399CAEB040352
:10D74000534538BF5346CAF1010B581C06EB0A0279
:10D7500005EB0A08CDF808B03B4607904FF00009EA
:10D76000019201F1FF3B37468A4609EB0406F8189F
:10D770000021F21A00F05CF900287FF416AF002EA9
:10D780003FF413AF544598BF07EB09002CD9DDF8DF
:10D7900004E098F800001EF8093098424AD16FEA78
:10D7A0000A021119C9074246534607EB090018D56A
:10D7B0000AF101039C4217D9424612F8011F10F8E2
:10D7C00003C08C450DD036E012F8011F10F803E0BD
:10D7D0008E4530D1013312F8011F10F803C08C457B
:10D7E00029D101339C42EFD8BBF1FF3F5B463FF4A8
:10D7F000F8AE15F80B1010F80B20914216D11BF063
:10D80000010F0AD00BF1FF33E95CC25C914204D0F6
:10D810000CE0E95CC25C914208D15A1E002B3FF437
:10D82000E0AEA95C825C023B9142F2D00798814451
:10D8300033469AE75346DDF808E0F1449944F7E7A8
:10D840000C460126AAE6039A60E74E46C844A8E6BD
:10D8500040F2D053C2F200031A6801235C3200F098
:10D8600001B800BFF0B4002825D0074638463E78FE
:10D870000D46013715F8014B3CB1A642FAD1002BF9
:10D88000F4D1176007F8013C11E0C6B13D4600E055
:10D890001BB915F8016B0C46284614F8013B9E4253
:10D8A000F6D136B1002105F8011C1060781EF0BCDD
:10D8B00070473046F9E710680028D6D1F7E71660C0
:10D8C0003046F4E72DE9F00F494C82B0D4F800C09F
:10D8D00001900F463C4614F8015B0CEB05004678BE
:10D8E000274606F00800C6B2002EF3D12D2D61D0D8
:10D8F0002B2D04BF244614F8015BB346002B41D105
:10D90000302D43D00A239A46BBF1000F0CBF6FF0B5
:10D9100000474FF00047B7FBFAF90AFB1970009077
:10D92000002080460CE0303DAB421BDD461C05D09C
:10D93000C84539D835D00AFB0858012014F8015BD6
:10D940000CEB0506767806F00407FFB2002FEAD14B
:10D9500016F0030606D0012E14BF57263726AD1B3E
:10D96000AB42E3DC431C2AD0BBF1000F01D0C8F16D
:10D970000008002A31D0D0B94046116002B0BDE89D
:10D98000F00F7047102BBED1302DBCD12578782DEB
:10D9900025D0582D23D043BB4FF0080A30255346DD
:10D9A000B2E700988542C6DD4FF0FF30C6E740463B
:10D9B000611EE2E714F8015B4FF0010B9EE7BBF13B
:10D9C000000F01990CBF6FF000404FF00040222380
:10D9D0000B60002AD2D0611ECFE74046CEE74FF061
:10D9E000100A6578534602348EE79A4630258BE755
:10D9F000A401002070B440F2D054C2F200040646E4
:10DA00000D462068134631462A4670BCFFF75ABFC0
:10DA1000024B13B1024800F005B870470000000047
:10DA2000F1C900080146002002460346FEF760BF28
:10DA30008307F0B4C9B200F09680531E002A00F0AC
:10DA4000948002788A420BD0421CD8071AD512F073
:10DA5000030F10461CD01478013B01328C4211D1C7
:10DA6000F0BC7047002B7CD01278013B8A42F7D083
:10DA700014F0030F204604F1010209D02478013B81
:10DA80008C42EDD012F0030F104602F10104E9D1EF
:10DA9000032B3FD9046841EA012545EA054585EA9B
:10DAA0000407A7F1013222EA07021E1F041D12F02B
:10DAB000803FC6F380072DD1032E334629D967B1A5
:10DAC0002668204685EA0602A2F1013626EA02020D
:10DAD000043412F0803F19D01CE020462468061D53
:10DAE00085EA0402A2F1013424EA020212F0803F26
:10DAF00010D13468043B85EA0402A2F1013424EA1F
:10DB00000202341D12F0803F304603D1043B032B48
:10DB1000E3D820465D1E23B303788B42A0D0431C7C
:10DB20000022E80714D51C781846012201338C42E4
:10DB300096D09542184603F1010402F102020ED07C
:10DB40001B788B428CD020462478431C8C4287D093
:10DB50009542184603F1010402F10202F0D10020BF
:10DB60007EE718467CE7134692E7104678E700BF49
:10DB7000032AF0B431D941EA00039C072ED106688C
:10DB80000F68151F031D0C1DBE42C5F3800C24D168
:10DB9000032D2A461FD9BCF1000F08D01E68256846
:10DBA0002146184604340433AE4211D015E0214614
:10DBB00018461C680B68051D0E1D9C420DD1314690
:10DBC00028462E680D68043A031D0C1DAE4204D190
:10DBD000043A032AEBD8214618461AB303780C7886
:10DBE000A3420AD1551E0022EB0714D510F8013FBD
:10DBF00011F8014F0122A3420DD0181B10E010F8BC
:10DC0000013F11F8014FA342F7D110F8013F11F87D
:10DC1000014FA342F1D1AA4202F10202EFD100204A
:10DC2000F0BC70471046FBE71E1E646464646464C5
:10DC30000010014000101002000801400080100296
:10DC400034080040380800403C08004040080040CC
:10DC500034040040380400403C04004040040040CC
:10DC6000D00732003200320032003200320032007F
:10DC7000C800640000004145545231323334000082
:10DC800015260008992600085926000835260008A0
:10DC900071260008F52600082126000837420008F2
:10DCA0005F41000807420008BD41000875410008B7
:10DCB0005D4100080000803F00000000A8AAAA3FC4
:10DCC0000000803F0000803F000080BFB0AA2ABF54
:10DCD000000080BF0000803F0000803FB0AA2ABF44
:10DCE000000080BF0000803F00000000A8AAAA3FFB
:10DCF000000080BF0000803F000080BFB0AA2ABFA4
:10DD00000000803F0000803F0000803FB0AA2ABF93
:10DD10000000803F0000803F00000000A8AAAA3F4A
:10DD2000000000000000803F000080BFB0AA2ABFB2
:10DD3000000000000000803F0000803FB0AA2ABF22
:10DD4000000000000000803F000080BF0000803F16
:10DD5000000080BF0000803F000080BF000080BF47
:10DD60000000803F0000803F0000803F0000803FB7
:10DD70000000803F0000803F0000803F000080BF27
:10DD8000000080BF0000803F000000000000000095
:10DD9000000000000000803F0000000000000000C4
:10DDA000000000000000803F000000000000803FF5
:10DDB0000000803F0000803F000080BF000080BF67
:10DDC000000000000000803F000000000000803FD5
:10DDD000000080BF0000803F0000803F000080BF47
:10DDE000000000800000803F000000000000803F35
:10DDF000000080BF0000803F000080BF00000000E6
:10DE00000000803F0000803F0000803F00000000D5
:10DE10000000803F0000803F00000000000080BF45
:10DE2000000080BF000000000000000003010000AF
:10DE300014DD000804000000E4DD00080400000018
:10DE40001CE0000802010000BCDF00080001000027
:10DE50000000000006000000B4DC0008060000001E
:10DE60005CDF000801010000000000000400000069
:10DE7000DCDF000806000000DCE00008080000000D
:10DE80003CE1000808000000DCDE0008080000009B
:10DE90005CE000080101000000000000000100003B
:10DEA000000000000001000000000000040000006D
:10DEB000A4DD00080600000044DD000800010000A9
:10DEC0000000000002010000BCE1000801010000A8
:10DED0000000000000000000000000000000803F83
:10DEE000F704353FF70435BF0000803F0000803F56
:10DEF000F70435BFF70435BF0000803F0000803FC6
:10DF0000F70435BFF704353F0000803F0000803F35
:10DF1000F704353FF704353F0000803F0000803FA5
:10DF200000000000000080BF000080BF0000803FB4
:10DF3000000080BF00000000000080BF0000803FA4
:10DF4000000000000000803F000080BF0000803F14
:10DF50000000803F00000000000080BF0000803F04
:10DF6000D0B35DBF0000003F0000803F0000803F55
:10DF7000D0B35DBF000000BF000080BF0000803F45
:10DF8000D0B35D3F0000003F0000803F0000803FB5
:10DF9000D0B35D3F000000BF000080BF0000803FA5
:10DFA00000000000000080BF0000803F0000803FB4
:10DFB000000000000000803F000080BF0000803FA4
:10DFC0000000803F00000000000000000000803FD3
:10DFD000000080BF00000000000000000000803F43
:10DFE000000000000000803F000080BF0000803F74
:10DFF000000080BF000080BF000000000000803FE4
:10E00000000000000000803F0000803F0000803FD3
:10E010000000803F000080BF000000000000803F43
:10E02000000080BF0000803F000080BF0000803FF4
:10E03000000080BF000080BF0000803F0000803FE4
:10E040000000803F0000803F0000803F0000803FD4
:10E050000000803F000080BF000080BF0000803FC4
:10E060000000803F000000BF0000803F0000803FB4
:10E07000000000BF000080BF0000803F0000803F24
:10E08000000080BF0000003F0000803F0000803F94
:10E090000000003F0000803F0000803F0000803F04
:10E0A0000000003F000080BF000080BF0000803FF4
:10E0B000000080BF000000BF000080BF0000803F64
:10E0C000000000BF0000803F000080BF0000803FD4
:10E0D0000000803F0000003F000080BF0000803F44
:10E0E000000000BFD0B35D3F0000803F0000803FD4
:10E0F000000000BFD0B35DBF0000803F0000803F44
:10E100000000003FD0B35D3F000080BF0000803FB3
:10E110000000003FD0B35DBF000080BF0000803F23
:10E12000000080BF00000000000080BF0000803FB2
:10E130000000803F000000000000803F0000803FA2
:10E14000000080BF0000803F000080BF0000803FD3
:10E15000000080BF000080BF0000803F0000803FC3
:10E160000000803F0000803F0000803F0000803FB3
:10E170000000803F000080BF000080BF0000803FA3
:10E18000000080BF0000803F0000803F0000803F13
:10E19000000080BF000080BF000080BF0000803F03
:10E1A0000000803F0000803F000080BF0000803FF3
:10E1B0000000803F000080BF0000803F0000803FE3
:10E1C0000000000000000000000080BF0000803F51
:10E1D00000000000000000000000803F2450554275
:10E1E000582C34312C312C303030332C303030310D
:10E1F0002C3131353230302C302A31450D0A002493
:10E20000504D544B3235312C3131353230302A318A
:10E21000460D0A0024505542582C34312C312C30F4
:10E220003030332C303030312C35373630302C30E4
:10E230002A32440D0A0024504D544B3235312C35CE
:10E24000373630302A32430D0A0024505542582CBC
:10E2500034312C312C303030332C303030312C33C1
:10E26000383430302C302A32360D0A0024504D54C8
:10E270004B3235312C33383430302A32370D0A00E6
:10E2800024505542582C34312C312C303030332C22
:10E29000303030312C31393230302C302A32330D9D
:10E2A0000A0024504D544B3235312C313932303044
:10E2B0002A32320D0A00B56206010300F00500FFA4
:10E2C00019B56206010300F00300FD15B5620601F1
:10E2D0000300F00100FB11B56206010300F000002D
:10E2E000FA0FB56206010300F00200FC13B56206E6
:10E2F000010300F00400FE17B562060103000102ED
:10E30000010E47B562060103000103010F49B56222
:10E3100006010300010601124FB562060103000168
:10E3200012011E67B56206160800030703005108B4
:10E3300000008A41B56206080600C800010001001D
:10E34000DE6A00000000000000C20100DCE10008FD
:10E35000FFE100080100000000E1000014E20008F5
:10E3600036E2000802000000009600004AE20008C1
:10E370006CE2000803000000004B000080E200088F
:10E38000A2E200080400000080250000B6EA0008B0
:10E39000B6EA0008414552543132333400000000DF
:10E3A000E7F20008EBF20008F0F2000801F30008C1
:10E3B0000AF3000815F3000820F300082BF3000807
:10E3C00009F2000834F3000803F200083DF30008E6
:10E3D00047F3000852F3000858F30008000000005B
:10E3E00039F200083DF2000843F2000849F2000843
:10E3F0004CF2000853F2000856F200085BF20008E5
:10E4000067F200086AF2000870F2000877F200086C
:10E4100081F200088BF2000894F20008A2F20008D2
:10E42000AEF20008B5F20008BBF20008C8F200081E
:10E43000D3F20008E0F20008000000004BF00008F2
:10E440004FF000081182000876F000087BF0000809
:10E450000D8700088FF0000898F00008658000081C
:10E46000B5F00008BAF0000859850008E9F0000886
:10E47000B6EA00082D800008EEF00008F6F000086B
:10E48000417F00080AF1000819F10008217F000807
:10E4900033F10008B6EA0008157D000838F10008DD
:10E4A0003CF10008797E000889F0000858F1000866
:10E4B0007D8000086BF1000871F100086981000897
:10E4C0008CF1000894F100081D810008A3F10008F8
:10E4D000A8F10008517E0008C7E90008B8F100085B
:10E4E00005840008E6F10008DAF10008417D000823
:10E4F000EDF10008B6EA0008097D0008B6EA000858
:10E5000015F200081DF2000825F200082DF200089F
:10E5100034F2000800000000303132333435363731
:10E5200038394142434445464748494A4B4C4D4E91
:10E530004F505152535455565758595A00416672CC
:10E540006F333220434C492076657273696F6E20B9
:10E55000322E32204170722032312032303134205C
:10E560002F2032303A33373A303900417661696CC6
:10E5700061626C6520636F6D6D616E64733A0D0A44
:10E580000025730925730D0A0053797374656D2096
:10E59000557074696D653A202564207365636F6EEC
:10E5A00064732C20566F6C746167653A2025642073
:10E5B0002A20302E3156202825645320626174743D
:10E5C000657279290D0A004350552025644D487A1B
:10E5D0002C2064657465637465642073656E736F65
:10E5E00072733A20002573200041434348573A2074
:10E5F0002573002E2563004379636C652054696D93
:10E60000653A2025642C20493243204572726F728E
:10E61000733A2025642C20636F6E666967207369E6
:10E620007A653A2025640D0A000D0A5265626F6F03
:10E6300074696E672E2E2E00536176696E672E2EDA
:10E640002E004D75737420626520616E79206F72A3
:10E65000646572206F662041455452313233340D67
:10E660000A0043757272656E742061737369676E18
:10E670006D656E743A20004572726F723A20456E75
:10E6800061626C6520616E6420706C756720696ED4
:10E69000204750532066697273740D0A00456E61FD
:10E6A000626C696E672047505320706173737468A1
:10E6B000726F7567682E2E2E0D0A00456E61626CB2
:10E6C00065642066656174757265733A20004176F1
:10E6D00061696C61626C65206665617475726573F1
:10E6E0003A2000496E76616C6964206665617475D4
:10E6F0007265206E616D652E2E2E0D0A00446973C1
:10E7000061626C65642000456E61626C6564200026
:10E710000D0A4C656176696E6720434C49206D6F28
:10E7200064652E2E2E0D0A00526573657474696E31
:10E730006720746F2064656661756C74732E2E2E6D
:10E740000043757272656E74206D697865723A2047
:10E7500025730D0A00417661696C61626C65206DFC
:10E7600069786572733A2000496E76616C6964203D
:10E770006D6978657220747970652E2E2E0D0A00F1
:10E780004D697865722073657420746F2025730D50
:10E790000A0043757272656E742070726F66696CE0
:10E7A000653A2025640D0A0055736167653A0D0AC4
:10E7B0006D6F746F7220696E646578205B76616C32
:10E7C00075655D202D2073686F77205B6F722073F5
:10E7D00065745D206D6F746F722076616C75650D68
:10E7E0000A004E6F2073756368206D6F746F722C12
:10E7F000207573652061206E756D626572205B30D7
:10E800002C2025645D0D0A004D6F746F7220256405
:10E81000206973207365742061742025640D0A00DB
:10E82000496E76616C6964206D6F746F72207661D9
:10E830006C75652C20313030302E2E323030300D5A
:10E840000A0053657474696E67206D6F746F72206F
:10E85000256420746F2025640D0A006175782025D9
:10E86000752025750D0A00496E76616C6964204635
:10E8700065617475726520696E6465783A206D759E
:10E880007374206265203C2025750D0A00202564E4
:10E890002025640043757272656E7420736574740C
:10E8A000696E67733A200D0A002573207365742022
:10E8B000746F20004552523A2056616C7565206194
:10E8C000737369676E6D656E74206F7574206F6603
:10E8D0002072616E67650D0A004552523A20556EEE
:10E8E0006B6E6F776E207661726961626C65206E07
:10E8F000616D650D0A0043757272656E7420436F19
:10E900006E6669673A20436F707920657665727923
:10E910007468696E672062656C6F772068657265E0
:10E920002E2E2E0D0A006D697865722025730D0A52
:10E9300000636D697820256400636D697820256423
:10E9400020302030203020300D0A0066656174755B
:10E950007265202D25730D0A0066656174757265F8
:10E960002025730D0A006D61702025730D0A007358
:10E970006574202573203D20004E4709004F4B0948
:10E9800000437573746F6D206D697865723A200D60
:10E990000A4D6F746F720954687209526F6C6C097A
:10E9A0005069746368095961770D0A002325643A38
:10E9B00009002573090053616E69747920636865E5
:10E9C000636B3A09007265736574006C6F61640073
:10E9D0004C6F61646564202573206D69782E2E2E3E
:10E9E0000D0A0057726F6E67206E756D626572203A
:10E9F0006F6620617267756D656E74732C206E652D
:10EA0000656473206964782074687220726F6C6C1E
:10EA1000207069746368207961770D0A004D6F7406
:10EA20006F72206E756D626572206D7573742062F1
:10EA300065206265747765656E203120616E6420A3
:10EA400025640D0A000D0A456E746572696E6720B3
:10EA5000434C49204D6F64652C20747970652027E4
:10EA6000657869742720746F2072657475726E2CD6
:10EA7000206F72202768656C70270D0A000D0A232D
:10EA800020000D1B5B4B001B5B324A1B5B313B3193
:10EA900048004552523A20556E6B6E6F776E206378
:10EAA0006F6D6D616E642C20747279202768656CBF
:10EAB000702700082008006C6F6F7074696D650026
:10EAC000656D665F61766F6964616E6365006D692F
:10EAD000647263006D696E7468726F74746C650043
:10EAE0006D61787468726F74746C65006D696E63C3
:10EAF0006F6D6D616E64006D696E636865636B0058
:10EB00006D6178636865636B006465616462616E02
:10EB10006433645F6C6F77006465616462616E6426
:10EB200033645F68696768006E65757472616C3321
:10EB300064006465616462616E6433645F7468720A
:10EB40006F74746C65006D6F746F725F70776D5F5A
:10EB50007261746500736572766F5F70776D5F7256
:10EB60006174650072657461726465645F61726D81
:10EB700000666C6170735F737065656400666978C8
:10EB8000656477696E675F616C74686F6C645F64FD
:10EB90006972007265626F6F745F6368617261634E
:10EBA00074657200736F667473657269616C5F621D
:10EBB0006175647261746500736F66747365726900
:10EBC000616C5F315F696E76657274656400736F46
:10EBD000667473657269616C5F325F696E766572C7
:10EBE000746564006770735F747970650067707333
:10EBF0005F62617564726174650073657269616CEE
:10EC000072785F747970650074656C656D65747297
:10EC1000795F70726F76696465720074656C656D9A
:10EC2000657472795F706F72740074656C656D6580
:10EC30007472795F73776974636800766261747364
:10EC400063616C6500766261746D617863656C6C9C
:10EC5000766F6C7461676500766261746D696E636E
:10EC6000656C6C766F6C7461676500706F77657248
:10EC70005F6164635F6368616E6E656C00616C699F
:10EC8000676E5F6779726F00616C69676E5F616361
:10EC90006300616C69676E5F6D616700616C6967D5
:10ECA0006E5F626F6172645F726F6C6C00616C6941
:10ECB000676E5F626F6172645F7069746368006140
:10ECC0006C69676E5F626F6172645F79617700790A
:10ECD00061775F636F6E74726F6C5F646972656396
:10ECE00074696F6E006163635F68617264776172FB
:10ECF00065006D61785F616E676C655F696E636CFE
:10ED0000696E6174696F6E006D6F726F6E5F7468AB
:10ED1000726573686F6C64006779726F5F6C7066A0
:10ED2000006779726F5F636D70665F666163746FB1
:10ED300072006779726F5F636D70666D5F666163A5
:10ED4000746F72007069645F636F6E74726F6C6C65
:10ED50006572007961776465616462616E64006107
:10ED60006C745F686F6C645F7468726F74746C65E8
:10ED70005F6E65757472616C00616C745F686F6C56
:10ED8000645F666173745F6368616E676500746871
:10ED9000726F74746C655F636F7272656374696FB0
:10EDA0006E5F76616C7565007468726F74746C6503
:10EDB0005F636F7272656374696F6E5F616E676CBB
:10EDC000650072635F726174650072635F6578707D
:10EDD0006F007468725F6D6964007468725F657853
:10EDE000706F00726F6C6C5F70697463685F7261E2
:10EDF0007465007961777261746500747061726125
:10EE00007465007470615F627265616B706F696ECA
:10EE100074006661696C736166655F64656C6179D5
:10EE2000006661696C736166655F6F66665F6465E5
:10EE30006C6179006661696C736166655F746872A4
:10EE40006F74746C65006661696C736166655F649C
:10EE500065746563745F7468726573686F6C640071
:10EE6000727373695F6175785F6368616E6E656CFC
:10EE7000007961775F646972656374696F6E0074AD
:10EE800072695F756E61726D65645F736572766FCE
:10EE90000067696D62616C5F666C616773006163D6
:10EEA000635F6C70665F666163746F720061636359
:10EEB00078795F6465616462616E64006163637A3E
:10EEC0005F6465616462616E64006163635F756E57
:10EED00061726D656463616C006163635F74726924
:10EEE0006D5F7069746368006163635F7472696DFC
:10EEF0005F726F6C6C006261726F5F7461625F73EE
:10EF0000697A65006261726F5F6E6F6973655F6CCD
:10EF10007066006261726F5F63665F76656C006247
:10EF200061726F5F63665F616C74006D61675F64DF
:10EF300065636C696E6174696F6E006770735F7092
:10EF40006F735F70006770735F706F735F690067E6
:10EF500070735F706F735F64006770735F706F735F
:10EF6000725F70006770735F706F73725F690067C4
:10EF700070735F706F73725F64006770735F6E6150
:10EF8000765F70006770735F6E61765F69006770AF
:10EF9000735F6E61765F64006770735F77705F7236
:10EFA0006164697573006E61765F636F6E74726F12
:10EFB0006C735F68656164696E67006E61765F732C
:10EFC000706565645F6D696E006E61765F73706514
:10EFD00065645F6D6178006E61765F736C65775F05
:10EFE0007261746500705F706974636800695F7056
:10EFF0006974636800705F726F6C6C00695F726F38
:10F000006C6C00705F79617700695F79617700707F
:10F010005F616C7400695F616C7400645F616C7443
:10F0200000705F6C6576656C00695F6C6576656C19
:10F0300000645F6C6576656C00705F76656C006976
:10F040005F76656C00645F76656C0061757800665C
:10F050006561747572655F6E616D65206175786656
:10F060006C6167206F7220626C616E6B20666F72DC
:10F07000206C69737400636D6978006465736967F7
:10F080006E20637573746F6D206D697865720064AE
:10F09000656661756C747300726573657420746F56
:10F0A0002064656661756C747320616E642072659E
:10F0B000626F6F740064756D70007072696E742099
:10F0C000636F6E666967757261626C6520736574E3
:10F0D00074696E677320696E20612070617374615A
:10F0E000626C6520666F726D006578697400666594
:10F0F0006174757265006C697374206F72202D766F
:10F10000616C206F722076616C0067707370617340
:10F11000737468726F756768007061737374687276
:10F120006F7567682067707320746F2073657269EC
:10F13000616C0068656C70006D6170006D6170706D
:10F14000696E67206F66207263206368616E6E650A
:10F150006C206F72646572006D69786572206E61F3
:10F160006D65206F72206C697374006D6F746F72BF
:10F17000006765742F736574206D6F746F72206FF4
:10F1800075747075742076616C75650070726F6649
:10F19000696C6500696E64657820283020746F2082
:10F1A00032290073617665007361766520616E6453
:10F1B000207265626F6F74006E616D653D76616C83
:10F1C0007565206F7220626C616E6B206F72202AF1
:10F1D00020666F72206C6973740073686F77207398
:10F1E000797374656D2073746174757300766572DC
:10F1F00073696F6E004759524F00414343004241CB
:10F20000524F00534F4E4152004750530047505306
:10F210002B4D4147004144584C333435004D505537
:10F2200036303530004D4D413834357800424D414F
:10F23000323830004E6F6E650054524900515541CE
:10F2400044500051554144580042490047494D42FD
:10F25000414C005936004845583600464C59494EF5
:10F26000475F57494E4700593400484558365800C3
:10F270004F43544F5838004F43544F464C4154501D
:10F28000004F43544F464C41545800414952504C52
:10F29000414E450048454C495F3132305F43435051
:10F2A0004D0048454C495F39305F4445470056544E
:10F2B00041494C340048455836480050504D5F5441
:10F2C0004F5F534552564F004455414C434F5054A5
:10F2D00045520053494E474C45434F505445520008
:10F2E000435553544F4D0050504D00564241540029
:10F2F000494E464C494748545F4143435F43414C64
:10F300000053455249414C5258004D4F544F525FA3
:10F3100053544F5000534552564F5F54494C54007C
:10F32000534F465453455249414C004C45445F525B
:10F33000494E47004641494C534146450054454CCF
:10F34000454D4554525900504F5745524D4554452F
:10F350005200564152494F0033440000F5F1000875
:10F36000FAF10008FEF1000811F2000803F20008AB
:10F3700009F200080DF2000800000000B7EA0008DA
:10F3800002000000AC110020000000002823000053
:10F39000C0EA000800000000AE11002000000000DC
:10F3A00001000000CEEA000802000000B2120020B6
:10F3B000B0040000A4060000D4EA00080200000027
:10F3C0007012002000000000D0070000E0EA0008F2
:10F3D000020000007212002000000000D0070000B0
:10F3E000ECEA000802000000741200200000000097
:10F3F000D0070000F7EA000802000000B412002065
:10F4000000000000D007000000EB00080200000030
:10F41000B612002000000000D007000009EB000831
:10F42000020000007612002000000000D00700005B
:10F4300018EB000802000000781200200000000015
:10F44000D007000028EB0008020000007A1200201C
:10F4500000000000D007000032EB000802000000AE
:10F460007C12002000000000D007000046EB0008DE
:10F47000020000007E12002032000000007D00002B
:10F4800055EB00080200000080120020320000004E
:10F49000F201000064EB000800000000B812002038
:10F4A000000000000100000071EB000800000000F7
:10F4B000B912002000000000640000007DEB00088D
:10F4C00001000000BA120020FFFFFFFF0100000052
:10F4D00093EB000800000000CA120020300000007A
:10F4E0007E000000A8EB000804000000C01200200D
:10F4F000B004000000C20100A4EB000804000000FA
:10F50000C4120020B0040000004B0000B8EB00085B
:10F5100000000000C81200200000000001000000F0
:10F52000CEEB000800000000C9120020000000001F
:10F5300001000000E4EB000800000000BC12002005
:10F540000000000004000000EDEB000801000000D6
:10F55000BD1200200000000004000000FAEB0008CB
:10F5600000000000B01200200000000003000000B6
:10F5700008EC000800000000CC1200200000000091
:10F58000010000001BEC000800000000CD1200206C
:10F5900000000000020000002AEC0008000000004B
:10F5A000CE12002000000000010000003BEC00082B
:10F5B00000000000A41200200A000000C8000000A3
:10F5C00045EC000800000000A51200200A00000021
:10F5D0003200000058EC000800000000A6120020D5
:10F5E0000A000000320000006BEC00080000000080
:10F5F000A712002000000000090000007DEC0008B8
:10F60000000000008212002000000000080000003E
:10F6100088EC0008000000008312002000000000B9
:10F620000800000092EC0008000000008412002096
:10F6300000000000080000009CEC0008030000002F
:10F64000861200204CFFFFFF68010000ADEC0008AF
:10F6500003000000881200204CFFFFFF680100003B
:10F66000BFEC0008030000008A1200204CFFFFFFDF
:10F6700068010000CFEC0008010000008C1200209F
:10F68000FFFFFFFF01000000E5EC000800000000A4
:10F690008D1200200000000005000000F2EC0008C0
:10F6A00002000000961200206400000084030000A5
:10F6B00008ED000800000000941200200000000087
:10F6C0008000000018ED0008020000008E120020EB
:10F6D000000000000001000021ED00080200000011
:10F6E0009012002064000000E803000032ED0008E2
:10F6F000020000009212002064000000E8030000F5
:10F7000044ED000800000000D410002000000000BC
:10F7100001000000B3EE00080000000040110020CE
:10F72000000000002000000053ED00080000000071
:10F730004111002000000000640000005FED00089F
:10F74000000000004211002001000000FA0000004B
:10F7500079ED0008000000004311002000000000C7
:10F76000010000008EED000800000000461100209E
:10F770000000000096000000A8ED00080200000054
:10F78000441100200100000084030000C2ED0008C5
:10F7900000000000F310002000000000FA0000004C
:10F7A000CAED000800000000F41000200000000076
:10F7B00064000000D2ED000800000000F5100020F9
:10F7C0000000000064000000DAED00080000000006
:10F7D000F61000200000000064000000E3ED0008C7
:10F7E00000000000F710002000000000640000008E
:10F7F000F3ED000800000000F810002000000000F9
:10F8000064000000FBED000800000000F91000207B
:10F81000000000006400000003EE00080200000089
:10F82000FA100020E8030000D007000012EE0008E4
:10F83000000000008811002000000000C800000047
:10F8400021EE0008000000008911002000000000E7
:10F85000C800000034EE0008020000008A110020F9
:10F86000E8030000D007000046EE00080200000098
:10F870008C11002064000000D007000060EE00083A
:10F8800001000000BB120020000000000400000086
:10F8900071EE0008010000008E110020FFFFFFFF45
:10F8A000010000007FEE0008010000008F11002021
:10F8B000000000000100000091EE000800000000C0
:10F8C0009011002000000000FF0000009EEE0008E4
:10F8D000000000000211002000000000FA000000FB
:10F8E000ADEE000800000000041100200000000040
:10F8F00064000000BCEE00080000000003110020BE
:10F900000000000064000000CAEE000800000000D3
:10F91000141100200000000001000000D9EE0008D2
:10F920000300000000110020D4FEFFFF2C010000A6
:10F93000E8EE000803000000FE100020D4FEFFFFE8
:10F940002C010000F6EE0008000000000511002068
:10F95000000000003000000004EF00080500000077
:10F9600008110020000000000100000013EF000853
:10F97000050000000C110020000000000100000044
:10F980001FEF00080500000010110020000000001B
:10F99000010000002BEF000803000000FC10002015
:10F9A000B0B9FFFF504600003BEF00080000000028
:10F9B000D910002000000000C800000045EF00083A
:10F9C00000000000E310002000000000C80000005C
:10F9D0004FEF000800000000ED10002000000000C4
:10F9E000C800000059EF000800000000DA100020F5
:10F9F00000000000C800000064EF000800000000E4
:10FA0000E410002000000000C80000006FEF0008B4
:10FA100000000000EE10002000000000C800000000
:10FA20007AEF000800000000DB100020000000005A
:10FA3000C800000084EF000800000000E51000206E
:10FA400000000000C80000008EEF00080000000069
:10FA5000EF10002000000000C800000098EF000830
:10FA6000020000009211002000000000D0070000FA
:10FA7000A6EF000800000000961100200000000022
:10FA800001000000BBEF00080200000098110020F8
:10FA90000A000000D0070000C9EF000802000000C3
:10FAA0009A1100200A000000D0070000D7EF0008DC
:10FAB000000000009511002000000000640000001C
:10FAC000E5EF000800000000D61000200000000054
:10FAD000C8000000EDEF000800000000E01000206A
:10FAE00000000000C8000000B7EC000800000000A3
:10FAF000EA10002000000000C8000000F5EF000838
:10FB000000000000D510002000000000C800000028
:10FB1000FCEF000800000000DF10002000000000E3
:10FB2000C8000000A6EC000800000000E91000205A
:10FB300000000000C800000003F000080000000002
:10FB4000D710002000000000C800000009F00008E5
:10FB500000000000E110002000000000C8000000CC
:10FB6000C9EC000800000000EB10002000000000BD
:10FB7000C80000000FF0000800000000D8100020AE
:10FB800000000000C800000015F0000800000000A0
:10FB9000E210002000000000C80000001BF0000878
:10FBA00000000000EC10002000000000C800000071
:10FBB00021F0000800000000DC1000200000000020
:10FBC000C800000029F0000800000000E610002036
:10FBD00000000000C800000031F000080000000034
:10FBE000F010002000000000C800000039F00008FC
:10FBF00000000000DE10002000000000C80000002F
:10FC00003FF0000800000000E810002000000000A5
:10FC1000C800000045F0000800000000F2100020BD
:10FC200000000000C8000000524F4C4C3B504954AB
:10FC300043483B5941573B414C543B506F733B50F9
:10FC40006F73523B4E6176523B4C4556454C3B4D93
:10FC500041473B56454C3B0041524D3B00414E47CE
:10FC60004C453B00484F52495A4F4E3B004241528F
:10FC70004F3B00564152494F3B004D41473B0048E6
:10FC8000454144465245453B004845414441444A6C
:10FC90003B0043414D535441423B0043414D54527C
:10FCA00049473B0047505320484F4D453B00475084
:10FCB0005320484F4C443B005041535354485255F5
:10FCC0003B004245455045523B004C45444D415850
:10FCD0003B004C45444C4F573B004C4C4947485423
:10FCE000533B0043414C49423B00474F5645524E1F
:10FCF0004F523B004F53442053573B0054454C4513
:10FD00004D455452593B00000000004B000000CB11
:10FD100061636F736600000000000000737172740D
:10FD200066000000000FC93F000F494000CB96401D
:10FD3000000FC9400053FB4000CB164100ED2F419E
:10FD4000000F49410031624100537B41003A8A4132
:10FD500000CB9641005CA34100EDAF41007EBC4169
:10FD6000000FC94100A0D5410031E24100C2EE417F
:10FD70000053FB4100F20342003A0A420083104262
:10FD800000CB164200141D42005C234200A529420C
:10FD900000ED2F4200363642007E3C4200C7424210
:10FDA000000F4942A2000000F9000000830000009B
:10FDB0006E0000004E00000044000000150000002E
:10FDC00029000000FC000000270000005700000090
:10FDD000D1000000F500000034000000DD0000004C
:10FDE000C0000000DB000000620000009500000081
:10FDF000990000003C00000043000000900000005B
:10FE000041000000FE0000005100000063000000FF
:10FE1000AB000000DE000000BB000000C5000000D9
:10FE200061000000B7000000240000006E00000028
:10FE30003A000000420000004D000000D200000027
:10FE4000E000000006000000490000002E00000055
:10FE5000EA00000009000000D1000000920000004C
:10FE60001C000000FE0000001D000000EB00000070
:10FE70001C000000B100000029000000A7000000E5
:10FE80003E000000E8000000820000003500000095
:10FE9000F50000002E000000BB0000004400000040
:10FEA00084000000E90000009C00000070000000D9
:10FEB00026000000B40000005F0000007E0000008B
:10FEC000410000003900000091000000D600000051
:10FED00039000000830000005300000039000000DA
:10FEE000F40000009C000000840000005F0000009F
:10FEF0008B000000BD000000F90000002800000099
:10FF00003B0000001F000000F80000009700000008
:10FF1000FF000000DE000000050000009800000067
:10FF20000F000000EF0000002F0000001100000093
:10FF30008B0000005A0000000A0000006D00000065
:10FF40001F0000006D000000360000007E00000071
:10FF5000CF00000027000000CB00000009000000D7
:10FF6000B70000004F000000460000003F00000006
:10FF7000660000009E0000005F000000EA00000034
:10FF80002D0000007500000027000000BA000000EE
:10FF9000C7000000EB000000E5000000F1000000D9
:10FFA0007B0000003D000000070000003900000059
:10FFB000F70000008A0000005200000092000000DC
:10FFC000EA0000006B000000FB0000005F00000082
:10FFD000B10000001F0000008D0000005D00000067
:10FFE0000800000056000000030000003000000080
:10FFF00046000000FC0000007B0000006B000000D9
:020000040801F1
:10000000AB000000F0000000CF000000BC000000CA
:10001000200000009A000000F400000036000000FC
:100020001D000000A9000000E30000009100000096
:10003000610000005E000000E60000001B00000000
:100040000800000065000000990000008500000025
:100050005F00000014000000A00000006800000025
:10006000400000008D000000FF000000D8000000EC
:10007000800000004D000000730000002700000019
:10008000310000000600000006000000150000001E
:1000900056000000CA00000073000000A800000025
:1000A000C900000060000000E20000007B000000CA
:1000B000C00000008C0000006B0000000400000085
:1000C00007000000090000000000C93F0000F039EF
:1000D0000000DA370000A2330000842E0000502B0D
:1000E0000000C2270000D0220000C41F0000C61B71
:1000F000000044176937AC3168212233B40F143340
:100100006821A2333863ED3EDA0F493F5E987B3FAA
:10011000DA0FC93F0020202020202020202028287E
:1001200028282820202020202020202020202020B7
:1001300020202020208810101010101010101010F7
:100140001010101010040404040404040404041027
:1001500010101010101041414141414101010101B5
:10016000010101010101010101010101010101017F
:10017000101010101010424242424242020202028B
:10018000020202020202020202020202020202024F
:1001900010101010200000000000000000000000FF
:1001A000000000000000000000000000000000004F
:1001B000000000000000000000000000000000003F
:1001C000000000000000000000000000000000002F
:1001D000000000000000000000000000000000001F
:1001E000000000000000000000000000000000000F
:1001F00000000000000000000000000000000000FF
:1002000000000000000000000000000000000000EE
:10021000000000000000000043000000A8010020D2
:10022000F8B500BFF8BC08BC9E467047F8B500BFE3
:08023000F8BC08BC9E467047B3
:0802380011DA0008350100088D
:0402400011010008A0
:100244000000004000000200000000400400040020
:100254000000004008000800000000400C001000EE
:1002640000040040000002000004004004000400F8
:100274000004004008000800000400400C001000C6
:1002840003010100A5290008000100000000803FCF
:100294000000000000000000DC05DC05DC05DC05D6
:1002A400DC05DC05DC05DC050000803F0000000007
:1002B40058FC000800000000010000005DFC00087C
:1002C400010000000200000064FC000802000000BD
:1002D400030000006DFC000803000000040000009F
:1002E40073FC000804000000050000007AFC00080C
:1002F40005000000060000007FFC00080600000066
:100304000700000089FC0008070000000800000046
:1003140092FC000808000000090000009BFC000893
:10032400090000000A000000A4FC00080A00000004
:100334000B000000AEFC00080B0000000C000000E5
:10034400B8FC00080C0000000D000000C2FC00080E
:100354000D0000000E000000CAFC00080E000000A2
:100364000F000000D2FC00080F0000001000000085
:10037400DAFC00081000000011000000E3FC000893
:100384001100000012000000EAFC00081200000046
:1003940013000000F4FC0008130000001400000027
:1003A400FCFC000814000000150000000000000020
:1003B400FF00000000000000000000000102030430
:1003C4000607080900127A0000A24A04020406087B
:1003D40000000000010203040102030406070809E7
:1003E4000100000014010108000000009404002032
:1003F400FC04002064050020000000000000000050
:1004040000000000000000000000000000000000E8
:1004140000000000000000000000000018020108B5
:1004240000000000000000000000000000000000C8
:1004340000000000000000000000000000000000B8
:1004440000000000000000000000000000000000A8
:100454000000000000000000000000000000000098
:100464000000000000000000000000000000000088
:100474000000000000000000000000000000000078
:100484000000000000000000000000000000000068
:1004940001000000000000000E33CDAB34126DE605
:1004A400ECDE05000B00000000000000000000006E
:1004B4000000000000000000000000000000000038
:1004C4000000000000000000000000000000000028
:1004D4000000000000000000000000000000000018
:1004E4000000000000000000000000000000000008
:04081400A801002017
:0400000508000000EF
:00000001FF
